:1000000000800020BD01000071D4000029D4000050
:1000100029D4000029D4000029D4000029D40000EC
:1000200029D4000029D4000029D4000071D4000094
:1000300071D4000029D40000F1CA0000F5CB000003
:1000400071D4000071D4000071D4000071D400009C
:1000500071D4000071D4000071D4000071D400008C
:1000600071D4000071D4000071D4000071D400007C
:1000700071D4000071D4000071D4000071D400006C
:1000800071D4000071D4000071D4000071D400005C
:1000900071D4000071D4000071D4000071D400004C
:1000A0002DB0000039B0000071D4000071D4000000
:1000B00071D4000071D4000071D4000071D400002C
:1000C00071D4000071D4000071D4000071D400001C
:1000D00071D4000071D4000071D4000071D400000C
:1000E00071D4000071D4000071D4000071D40000FC
:1000F00071D40000DDF4000071D4000009F60000A6
:1001000071D4000049DE000071D4000071D40000F9
:1001100071D4000071D4000071D4000071D40000CB
:1001200071D4000071D4000071D4000071D40000BB
:1001300071D4000071D4000071D4000071D40000AB
:1001400071D4000071D4000071D4000071D400009B
:10015000E1CC0000F5CC000009CD00001DCD000071
:1001600071D4000065E1000071D4000071D400007A
:1001700071D4000071D4000071D4000071D400006B
:1001800071D4000071D4000071D4000071D400005B
:1001900071D4000071D4000071D4000071D400004B
:1001A00071D4000071D4000071D4000071D400003B
:1001B00071D4000071D4000071D40000564B4CF291
:1001C000205210B51A804DF628121A8000BF00BFC9
:1001D0000DF052F9514B4FF010621A60504A9A607C
:1001E000504ADA60504A136813F4807304D14F49BF
:1001F0000B604FF4A85313604D4B1A78110703D5C9
:100200001A7842F008021A704A4B4B492A221A7097
:100210004A4A4B4B8B4204D252F8040F43F8040B6A
:10022000F8E7484B484900228B4202D243F8042B9E
:10023000FAE74649464A002352F8230041F82300D2
:1002400001336F2BF8D1434B434A802103F8011B44
:100250009342FBD1414B3D4A1A60414B8A221A70AE
:10026000A3F5805324225A70A0221A709A7992071B
:10027000FCD59A79D406FCD43A4A937903F00C035E
:10028000082B384BF9D103221A7140225A719A79FE
:100290009006FCD5334A9179324B4906FBD5324A58
:1002A000324911600221516020221A709A7902F0BD
:1002B0000C020C2AFAD12E4B2E4A1A602E4B2F4AD2
:1002C0001A6000225A60072243F8042C2C4AC3F813
:1002D0000C2D62B60DF080FC144B1B68DA0705D5B7
:1002E00028480DF04DFA284B284A1A60284B1B78F5
:1002F0005B0609D5244C254B22689A4204D121483B
:100300000DF03EFA0023236010F036FC0DF0BAF831
:100310000CF0E8FFFEE700BF0E20054030800440EF
:10032000823F04000100002B10D0034014D0034092
:1003300002D0074000E00740DC9BFF1F1C45010086
:100340004088FF1FDC9BFF1FF4A3FF1F0082FF1FDD
:100350000000000000E400E05FE400E008ED00E0E1
:100360000050064000400640448004400000030165
:1003700004800440C010050014E000E0FF76010096
:1003800000002020BB02825F1CE00340A5C3945AFA
:1003900000F00740FFFFFFFFFFFFFFFFFFFFFFFF32
:1003A000FFFFFFFFFFFFFFFFFFFFFFFFFFFFFFFF5D
:1003B000FFFFFFFFFFFFFFFFFFFFFFFFFFFFFFFF4D
:1003C000FFFFFFFFFFFFFFFFFFFFFFFFFFFFFFFF3D
:1003D000FFFFFFFFFFFFFFFFFFFFFFFFFFFFFFFF2D
:1003E000FFFFFFFFFFFFFFFFFFFFFFFFFFFFFFFF1D
:1003F000FFFFFFFFFFFFFFFFFFFFFFFFFFFFFFFF0D
:10040000FFFFFFFFFFFFFFFFFFFFFFFFDEF9FFFF23
:1004100010B5054C237833B9044B13B10448AFF33E
:1004200000800123237010BDDC9BFF1F0000000033
:1004300020450100084B10B51BB108490848AFF32F
:1004400000800848036803B910BD074B002BFBD0A0
:10045000BDE81040184700BF00000000E09BFF1FF0
:1004600020450100DC9BFF1F0000000038B504465A
:10047000104621700A491D4610F060F901464FF000
:100480007E5010F00FFA074910F058F9E5606060EF
:10049000256165610DF030FBE061204638BD00BF8D
:1004A000DB0FC9400024744938B50446104621705A
:1004B00009491D4610F042F901464FF07E5010F0F8
:1004C000F1F9064910F03AF9E5606060256165616F
:1004D0000DF012FBE06138BDDB0FC9400024744908
:1004E00038B503780446032B20D8DFE803F01A1848
:1004F0001002C168406910F017F80D4905466068A0
:1005000010F0D0F90146284610F0CCF938BD084962
:10051000406810F0C7F9E16810F010F938BDC06804
:1005200038BDC16840690FF0FFFF38BD002038BDFD
:100530000024744970B504460E460DF0DDFA0546F8
:10054000E069281A10F0A6F8E3682361E5616661A6
:10055000A0610146606810F0A5F90146A06010484E
:1005600010F0A0F90FF076FC0FF016F90FF088FFED
:10057000054601464FF07E500FF0D6FF616910F03E
:10058000DDF821690646284610F0D8F801463046C5
:100590000FF0CCFFE0602046BDE87040FFF7A0BF41
:1005A000000080BF08B50E200CF076FD114B1B88B3
:1005B000012B19D0104B1B88984213DB40F6FF71BA
:1005C0008842D4BFC3EB0001C3EB0101C1EB013191
:1005D000C3F57F630F33282091FBF3F1BDE808409A
:1005E0000DF0E0B80021F3E70146BDE80840142013
:1005F0000DF0D8B8309EFF1FC49CFF1F10B50446F5
:100600000CF04CFB204610BD70B44C88A04220D9A1
:1006100001230133DBB21CB2660031F8144084427E
:100620001D46F6D3A04211D005F10045013D965B71
:1006300031F8151032F81530401AF21A00FB02F0AA
:10064000641A90FBF4F4E01870BC7047905B70BCC7
:10065000704702260125E5E700280CDA064A4342E6
:1006600082FB0320DA17C2EB600000EB4000A3EB33
:100670008000C0F10C007047ABAAAA2A38B5234B02
:100680001B78002B2CD015200CF006FD204B186099
:10069000204B1B88984203DA1F4C237863BB38BD7C
:1006A0001E4A1488A042A4EB0302A8BF20467F2A5A
:1006B0001CDDC01AC001541C90FBF4F4002CEBD0DC
:1006C000154B1A780AB901221A70154D2B689C42F5
:1006D00004D0144BE1B2187808F07AFD2C6038BDD4
:1006E00011200DF01DFC0A4B1860D1E7C01AC0EBB9
:1006F000C01090FBF2F4E1E70A4B0021187808F0F3
:1007000067FD0023064A2370136038BD429EFF1F19
:10071000089CFF1F7E9CFF1FB09EFF1F5C9EFF1F5B
:10072000AC9EFF1F549CFF1F38B50F200DF0F8FB47
:100730001B4A1C4B12881860C0F53B600830904281
:1007400020DB194B1B889842A3EB0204A8BF184674
:10075000801A7F2CC6BFC0010134C0EBC01090FBD3
:10076000F4F47CB1114B1A780AB901221A70104DB9
:100770002B689C4204D00F4BE1B2187808F028FD9A
:100780002C6038BD094C237803B938BD094B0021D2
:10079000187808F01DFD0023054A2370136038BD4A
:1007A000C89CFF1FD89DFF1F489EFF1F6C9EFF1F08
:1007B000889CFF1F769CFF1FF0B40E8886420DD2E6
:1007C00003F10043013B31F81350854202D9F0BCDC
:1007D000FFF71ABF32F81300F0BC70471088F0BC66
:1007E000704700BF094B1B880C2B09D8084A80B200
:1007F00052F8232028B143F6FE73984203D9108C97
:100800007047108870470349FFF7FEBE2E9CFF1FFC
:10081000A01F01003C2101004B4B4C4A2DE9F04741
:100820001E8814684A4BB442B3F80080494B33DB4E
:100830004445A8BF4446A6421C60C8BF00202DDD29
:10084000C6EB0807B7F5804F33DB80037B1C90FBBA
:10085000F3F0FFF7C7FF404A404B15881B88C0F3F1
:10086000C61909FB05F57F2D8246A8BF7F252BB34E
:10087000A64253DC4445D4BFC6EB0404C6EB0804CF
:100880009F42CCBF03FB04445C43354BC8BF0137D8
:1008900094FBF7F71F6013E034461E60C6EB0807B1
:1008A000A045D4BFC6EB0800C6EB0400B7F5804FE7
:1008B000CBDAC0EB803090FBF7F0CAE7284A136030
:1008C000284C2368994508D0274B1B88002B34D12E
:1008D000264B1B886BBBC4F80090254C23689A45B7
:1008E00006D0214B1B885A1F032A19D9C4F800A02F
:1008F000204C23689D420FD01F4B188848B11A4BDB
:100900001E4A1B88D35C834203D0C0B2E9B208F010
:100910005FFC2560BDE8F087BDE8F0870024AFE705
:10092000164AD05C2030C0B20AF07F0108F050FCBB
:10093000DCE7484608F0C0FCCDE7104A4946D05CE9
:1009400008F046FCC4E700BFC49CFF1F2C9EFF1F9D
:100950008C9EFF1F009CFF1F109CFF1F129CFF1FFF
:10096000909EFF1F709CFF1F129EFF1FBA9CFF1FCF
:10097000289CFF1FBC9CFF1F229EFF1F9C89FF1FFE
:100980002DE9F04F17208BB00DF0CAFADFF870B3E5
:10099000DFF870A3CBF8000016200DF0C1FABA4BB7
:1009A000CAF800001B880C2B00F05E82B74EB84AD4
:1009B0003188B84B52F8214000221A70B64BB74A22
:1009C0001B88B7491288013B012A31F9133005937E
:1009D00000F0AE81B34B0193B34B0293B34FDFF8FA
:1009E000288300230093B24B1B88012B00F0F48175
:1009F000DFF81893AF4B0393D9F80050AE4B049334
:100A00000023AE4A1288013A032A00F24982DFE845
:100A100012F0A500ED000400C900284605930FF070
:100A200039FEA7490FF08AFE059B054618460FF0D0
:100A300031FEA4490FF082FE014628460FF076FDF4
:100A400010F042F80546C9F8005038680FF022FE51
:100A50009B490FF073FE814600980FF01BFE9949E9
:100A60000FF06CFE014648460FF060FD10F02CF8C8
:100A70003860954A954B17881988954BDBF800200C
:100A80001B88DFF88CE2C7EB050C3D44039FC7F8D9
:100A900000C0471A084404990D6001990F6002993B
:100AA000BEF8007008609A4280F2E7800025C3EB30
:100AB000070E7445DAF8000080F2D380611C98427A
:100AC00005FB01F50EF1010E95FBFEF5C0F25F830B
:100AD0008742A8BF0746FF1A01FB07F494FBFEF408
:100AE0009A4200F3A780984200F3A480794C2068D2
:100AF0000FF0D0FD78490FF021FE78490FF016FD78
:100B00000FF0E2FFA0F5FF531C3B082B98BF4FF4FA
:100B10000050D8F80030184400282060C0F29F80B0
:100B2000B0F5804F80F2F6806D4B1B781BB1B0F5AD
:100B3000005F40F0F7806B4D2B78002B40F0AB81CD
:100B4000694D20682B68634C984204D080B208F04D
:100B50001DFC23682B600BB0BDE8F08F2846059381
:100B60000FF098FD61490FF0E9FD059B0546184619
:100B70000FF090FD5E490FF0E1FD014628460FF0B1
:100B8000D5FC0FF0A1FF0546C9F8005038680FF0FA
:100B900081FD56490FF0D2FD814600980FF07AFD95
:100BA00053495DE7284605930FF074FD4A490FF05D
:100BB000C5FD059B054618460FF06CFD4D490FF02D
:100BC000BDFD014628460FF0B1FC0FF07DFF054644
:100BD000C9F8005038680FF05DFD3F490FF0AEFDD9
:100BE000814600980FF056FD424939E728460593A3
:100BF0000FF050FD40490FF0A1FD059B054618463A
:100C00000FF048FD3D490FF099FD014628460FF0D1
:100C10008DFC0FF059FF0546C9F8005038680FF0F9
:100C200039FD35490FF08AFD814600980FF032FDFD
:100C3000324915E73388002B3FF458AF2B1B002BAC
:100C4000B8BF5B42092B00F32D81D8F80030214C4E
:100C50004FF40050184400282060BFF661AF002216
:100C60005AE0984205FB04F5B8BF002195FBFEF55C
:100C700080F2848291FBFEF432E7BA42D4BFC3EB28
:100C80000205C3EB070512E75E9EFF1F649CFF1F72
:100C90005889FF1F069CFF1F2089FF1F329EFF1FE0
:100CA000A8230100589CFF1F989CFF1FF89BFF1F63
:100CB000C09DFF1F509EFF1FC49DFF1F2E89FF1F59
:100CC000CDCC4C3FCDCC4C3EA889FF1F2C89FF1FBB
:100CD000289EFF1F9089FF1F9A99193FCDCC4C4544
:100CE000629FFF1FB99CFF1F2489FF1F3333733F8F
:100CF000CDCC4C3DCDCCCC3E6666663FCDCCCC3D1C
:100D0000609CFF1F249CFF1F689EFF1F4C9EFF1FBF
:100D1000409CFF1F43F6FF72C04B22601B78002BE4
:100D20003FF409AF05F020FCBD4B01221A7007E724
:100D3000BC4BBD4A1B88BD491278013B31F91350A9
:100D4000002A40F0C78011200DF0EAF80090B84B5F
:100D50000193D3F80080009B984540F3C080B54BC9
:100D6000B54F1B88B54A012B3B68B2F80090B44AD6
:100D700002922046A3EB050500F0E2800FF08AFC0A
:100D8000029A52F829100FF0D9FC014600200FF00A
:100D9000CBFB0FF099FE009BC8EB05029D42B8BF4C
:100DA0001D469042C8EB050580F2DE8000FB05552C
:100DB000013295FBF2F5A34BDFF8B4820293D8F829
:100DC00000302B4403EBD3735B10C8F800309E4B0C
:100DD0001B88012B7FF40CAE9C4B03931D460F2008
:100DE0000DF09EF82A6804929042034680F2CC806F
:100DF000904A1288012A00F03F81904A0790128899
:100E00008F4D069220460FF045FC069ADFF864925B
:100E100055F82210D9F800500FF090FC0146002040
:100E20000FF082FB059BEA1A05920FF04DFE059A22
:100E3000079B04999A42C1EB020EB8BF1A4670454F
:100E400080F24481521A00FB02220EF1010192FB52
:100E5000F1F2D8F800107E4804900A4402EBD272F6
:100E60005210C8F80020CCE57A4B1B78002B3FF4D9
:100E70009DAD794E794A3188794B52F82100012293
:100E80001A700FF007FC4FF07C510FF057FC0FF079
:100E90001BFE044692E505F063FB00232B704FE632
:100EA0003868E6E505F500500130001B0FF0F2FB55
:100EB0006C496D4C0FF042FC054620680FF0EAFBD0
:100EC0006A490FF03BFC014628460FF02FFB0FF05C
:100ED000FBFD1EE615200CF0DFF8009037E7594BBC
:100EE0000293D3F80080009B984542DA514B524F51
:100EF0001B88524A012B3B68B2F80090504A03927B
:100F000020461D4400F0E9800FF0C4FB039A52F81C
:100F100029100FF013FC0FF0D7FD009B9D42C8EB8A
:100F20000502A8BF1D46C8EB05059042BABF00FBED
:100F300005550132454395FBF2F5DFF834813EE774
:100F40000FF0A8FB029A52F829100FF0F7FB0FF0F0
:100F5000BBFD009BC8EB05029D42B8BF1D46824207
:100F6000C8EB05053FF722AF00FB05F595FBF2F551
:100F700021E7DFF8FC80304FD8F8003003EBD37363
:100F80005B10C8F800302EE5314A049212680692D0
:100F9000904237DD274A1288012A00F0BC80274A98
:100FA00009901188264A0891204607920FF072FB9B
:100FB000079A0899DFF8BC9052F82110D9F8005030
:100FC0000FF0BCFB059B2B4405930FF07DFD0599AD
:100FD000099B069A9942C2EB010EA8BF19467045BB
:100FE00080F2BE80891A00FB01110EF1010291FB13
:100FF000F2F2D8F800100A4402EBD2725210C8F88C
:101000000020FEE4D8F80020DFF8689002EBD272EE
:101010005210D9F80050C8F80020F2E4629FFF1F78
:10102000B99CFF1FAC89FF1F429EFF1FF4200100E7
:10103000589CFF1F9E9CFF1FF89BFF1F489CFF1F93
:10104000C0230100989CFF1FC09DFF1F509EFF1FE3
:10105000C49DFF1F109EFF1F649CFF1F5889FF1F28
:10106000069CFF1FCDCCCC3E9089FF1F9A99193F5B
:10107000689EFF1F4C9EFF1F464A08901188464AF3
:101080000791204606920FF005FB069A0799DFF8B4
:101090000C9152F82110D9F800500FF04FFB059B2E
:1010A000E91A05910FF010FD0599089B049A9942E1
:1010B000C2EB010EB8BF1946704558DA891A00FB19
:1010C00001110EF1010291FBF2F2C2E60499521AEB
:1010D00000FB02F292FBFEF2BBE60FF0DBFA039A92
:1010E00052F829100FF02AFB014600200FF01CFADD
:1010F0000FF0EAFC009A9542C8EB0503A8BF15461D
:10110000C8EB05059842BABF00FB055501334543BE
:1011100095FBF3F511E71F491F4A089020460D88FB
:1011200007920FF0B7FA079ADFF8709052F825107F
:10113000D9F800500FF002FB014600200FF0F4F93F
:10114000059B2B4405930FF0BFFC0599089B069A5D
:101150009942C2EB010EA8BF19467045FFF642AF97
:10116000069A891A00FB01F191FBFEF241E7049A0D
:10117000891A00FB01F191FBFEF26AE6B842D4BF86
:10118000C3EB0001C3EB070104FB01F172E51F464D
:10119000A1E400BF489CFF1FC02301004C9EFF1F1D
:1011A00008B5244B1B88FBB1234B1B78FBB1234BA9
:1011B0001B78E3B1224B1B78CBB1224B1B78B3B128
:1011C000214B22481A78C2B9214A22490088128844
:1011D00009680244B1EB620F09DD01221A70642034
:1011E000BDE8084005F0D4B9174A117801B908BD27
:1011F0001370BDE8084008F093B8154A16490088F6
:10120000128809680244B1EB620FF0DD00221A7007
:1012100008F086F8642005F0BBF9642005F0B8F901
:10122000642005F0B5F94FF41670BDE808400CF0E5
:1012300085BC00BFD09DFF1FB49EFF1F869EFF1F71
:10124000879EFF1F889EFF1F2C9CFF1F409CFF1F37
:10125000289EFF1F609CFF1F249CFF1F38B5114C68
:10126000232025780BF018FF0F4A42F82500131FA2
:1012700002F1C400002253F8041F83420A44FAD149
:1012800023780A4907480A4C0133DBB2322B81FB31
:10129000025108BF0023D217C2EB21120370226053
:1012A00038BD00BF149CFF1FD49CFF1F1F85EB514E
:1012B000249EFF1F2DE9F04FB84CB94D2068B94F5F
:1012C00083B00FF0E7F9B8490FF038FA064610205E
:1012D0000CF026FE0FF0DEF9B4490FF02FFA31467C
:1012E0000FF024F90FF0F0FB2988206088423B883A
:1012F00043DA9E465B1A7F2B4FF0000247DDD20196
:101300005E1C92FBF6F2AA4EDFF8C882B6F800C067
:10131000C8F80020BCF1190F00F0DF80BCF11A0FF3
:1013200000F01781BCF11E0F00F020810126B146AC
:10133000A04A1288002A00F09D808842C0F20781EE
:101340007045D4BFC1EB0000C1EB0E009A42BABF9A
:1013500002FB00000133504390FBF3F3964A136005
:10136000964B1888C0B9964A1288AAB9954B197835
:1013700001B11A7003B0BDE8F08F9842D4BFC1EB41
:101380000002C1EB03029E465B1A7F2BB7DCC2EB67
:10139000C21292FBF3F2B6E72988D4F800E0DFF836
:1013A0000082DFF8F8A171456CDCDFF818C29CF808
:1013B0000020002A2ED14FF0010B04288CF800B039
:1013C00028D1002E40F094817D4B18880028D1D080
:1013D000B9F1000FCED023682C883A88A34280F25E
:1013E00065810023141B7E2C774DD5BFC3EB83137F
:1013F000C3EBC3135B00013493FBF4F42B6801349B
:10140000A34203D0C0B2E1B207F0E2FE2C6003B009
:10141000BDE8F08F012800F0F680022800F0EB8094
:101420000328D1D1694B1B88092BCDD0002ECBD0FE
:1014300023682E883A88B34280F27B810023961B72
:101440007E2EDFF88CA1D5BFC3EB8313C3EBC31390
:101450005B00013693FBF6F6DAF800300136B34252
:1014600003D0F1B24A2007F0B3FECAF80060ABE740
:1014700016469146BCF11E0F7FF472AF0022DFF8D2
:1014800058817EE04F4B1A78002A3FF473AF002456
:1014900001281C7000F0A480022840F00E81002E6C
:1014A00000F0A3804A4D2B68002B00F09E800420A2
:1014B000214607F08DFE424B2C60188800283FF42F
:1014C00059AFB9F1000F3FF455AFC0B2002107F09A
:1014D0007FFE3D4B00221A604CE7DFF8FC8098F855
:1014E0000020C2B1DFF8D890B9F800A0BAF1000F1F
:1014F00011D0DFF8E89099F800B0934578D05FFA02
:101500008AF07F2107F064FE98F80030B6F800C03A
:1015100089F8003010E0DFF8C49099F800A09245F7
:1015200066D0274B0021187807F052FE98F800305B
:10153000B6F800C089F800301E4B1A88002A97D0F0
:10154000BCF11E0F40F006810026B14619E00020D4
:10155000FCE6DFF8848098F80020002A0BBF012603
:1015600000264FF000094FF00109E1E6DFF868803E
:10157000104B98F800601A88B6FA86F676094FF094
:10158000000998F80030002B3FF4E8AE2988B7F83E
:1015900000E02068C1EB0E03CFE600BF509CFF1FA8
:1015A000D69DFF1FD29DFF1F9A99193FCDCCCC3EEF
:1015B0005E9EFF1F949EFF1FCC9CFF1F5E9CFF1F23
:1015C000709EFF1F659EFF1F349CFF1F129EFF1F12
:1015D000D09CFF1F449EFF1F109EFF1F189CFF1FE3
:1015E0001EB1614D2B68002B7BD1604B188865E7DD
:1015F0000026B1469CE6002E3FF4E6AEDFF868A177
:10160000DAF800202EE0002E3FF4DEAEB7F80080BE
:10161000F045D4BFC1EB0802C1EB0E02C1EB0808D4
:10162000B8F17E0FDFF840A1D5BFC2EB8212C2EB4A
:10163000C212520008F1010892FBF8F8DAF8002013
:1016400008F10108424506D05FFA88F101200093B5
:1016500007F0BEFD009B1888CAF8008002287FF4BE
:10166000DFAE42462168B5F800803888414559DA36
:101670000021C8EB0008B8F17E0FD3BFC1EB811188
:10168000C1EBC11108F10108490091FBF8F808F11C
:101690000108904506D05FFA88F10420009307F016
:1016A00097FD009B1888CAF80080B9E69342D4BF22
:1016B000C4EB0303C4EB020394E6032827D12C4BAD
:1016C0001B88092B91D0002E8FD0274D2B68002B23
:1016D0008BD04A20214607F07BFD244B2C601888D4
:1016E000ECE6214607F074FD204B2C601888E5E6F7
:1016F00040207F218DE80C0007F06AFD019B009AD5
:10170000188858451CD002287FF48AAE76E7042852
:101710007FF46BAF002E3FF468AF2146402007F006
:1017200057FD62E78142D4BFC8EB0101C8EB00015D
:101730009FE79342D4BFC6EB0303C6EB02037EE6EA
:10174000B8F80010DAF800E0B7F800808E45FFF630
:1017500065AF5DE72988B7F800E020680026C1EB97
:101760000E03B146E9E500BFD09CFF1F709EFF1F2E
:10177000129EFF1F08B5114B1B88022B09D0052BA9
:1017800007D0032B15D0042B0BD00D4B01221A7060
:1017900008BD7F21412007F01BFD094B01221A7073
:1017A00008BD7F21092007F013FD054B01221A70A7
:1017B00008BD4021092007F00BFDE6E7CA9CFF1F8A
:1017C000809CFF1F38B5074B074D1B88052B04462F
:1017D00006D02B68834203D0C1B2052007F0F8FC85
:1017E0002C6038BDCA9CFF1F749EFF1F38B5124D78
:1017F000124C2B88052B12D022684AB9022B0ED02E
:10180000033B012B13D90E4A00231370236038BD0C
:101810000021052007F0DCFC2B88022B04D10021DD
:10182000412007F0D5FCEEE7052BE9D1F7E70021D1
:10183000092007F0CDFCE6E7CA9CFF1F749EFF1F3E
:10184000809CFF1F464B1B881D2B70B541D0454D1A
:101850000024454B1B88022B16D0444B1B88022BBF
:1018600054D02888424B002C1B780ADB8442A8BF46
:10187000044634B1002B3AD02046BDE87040FFF753
:10188000A1BF002B2FD170BD3A4B1B78002B37D056
:1018900015200BF001FC384B1860384A1288002ADA
:1018A000DBD0374A186811888142D6DC354B2A884C
:1018B0001B888342A3EB0106A8BF03465B1AB24212
:1018C000BABF02FB03330136534393FBF6F31C44C8
:1018D000C3E72A4B1C888CB12B4B224D1C78002C63
:1018E000B7D02C88B5E7BDE87040FFF77FBFFFF7A2
:1018F00041FF2046BDE87040FFF764BF194DA8E7DF
:1019000011200CF00DFB1C4B1860C6E70F200CF0EB
:1019100007FB1A4B1D4A1B881060002BA1D01C4AE4
:10192000C0F53B63118808338B429ADB194A28883B
:1019300012889342A2EB0105A8BF1346A842A3EB6D
:10194000010306DA00FB0333013593FBF5F31C4476
:1019500088E700FB03F292FBF5F31C4482E700BF2B
:101960005E9EFF1F629EFF1F329EFF1FC09DFF1FD6
:10197000809CFF1F429EFF1F089CFF1FCA9CFF1FE9
:101980007E9CFF1F5C9EFF1F109EFF1FD89DFF1FA8
:10199000C89CFF1F489EFF1F38B510200CF0C0FAEE
:1019A000C830B0F5FA7FC0F2EE80B0F57A6F01462C
:1019B000A8BF4FF47A6101F51673B3F57A6FA8BF2B
:1019C0004FF47A639BB289B28E4A8F4C11802220E9
:1019D000238007F081FD21888C4D8D4C242007F059
:1019E0007BFD0E200BF058FB40F6FF71C83088429B
:1019F000A8BF084620EAE07000F5FA6283B28A4286
:101A0000A8BF0A460220194622802B8007F064FDF9
:101A10002188042007F060FD17200CF081FA0446AD
:101A200016200CF07DFAA042B8BF204600F1C80194
:101A3000B1F5FA7FC0F2A280B1F57A6FA8BF4FF47A
:101A40007A6101F54873B3F57A6FA8BF4FF47A63F2
:101A50009BB289B26F4A704C11800A20238007F034
:101A60003BFD21880C2007F037FD0F200CF058FAC1
:101A7000C0F53F610431B1F5AF6F7CDBB1F5FA6FB2
:101A8000A8BF4FF4FA6189B2644BC0F54360B0F56A
:101A9000AF6F19806CDBB0F5FA6FA8BF4FF4FA6036
:101AA00083B25F4CA420238007F016FDA620218876
:101AB00007F012FD0B200CF00BF8002868D0112065
:101AC0000CF02EFA00F1C801B1F52F7F6EDA40F26A
:101AD00014534FF42F71534A1180534C0620238026
:101AE00007F0FAFC2188082007F0F6FC00244FF4E8
:101AF000AF75E1B24D4809F00DFB01348542A8BF36
:101B000005460C2CF5D101200CF00AFA0446002001
:101B10000CF006FA323CA0F1320345496FF495709F
:101B200000FB03F300FB04F081FB034281FB004157
:101B3000DB17C017C3EB6223C0EB612003F5AF7264
:101B400000F5AF739342A8BF13469D42A8BF1D4640
:101B5000A5F11401312938DC40F26C73322135488B
:101B6000354A018013602A20BDE8384007F0B4BC34
:101B70004FF4AF6395E74FF4AF6185E740F214533C
:101B80004FF4FA7166E740F24C434FF4FA711BE7E9
:101B900015200BF081FA00F59671B1F52F7F96DBD9
:101BA00041F25C2399421FDD194694E741F25C2320
:101BB0009942F9DC1B4A00F5487089B2B0F52F7FD5
:101BC000118019DA4FF42F7387E740F23A72A5F5C6
:101BD000B9751A4B02FB05F583FB0523ED17A5EB41
:101BE000631389B23233BAE70E4A00F5617089B2E5
:101BF000B0F52F7F1180E5DB8342A8BF03469BB27F
:101C00006BE700BFD69DFF1FD29DFF1FC49CFF1F27
:101C10008C9EFF1F289EFF1F409CFF1FC89CFF1F1C
:101C2000489EFF1F7E9CFF1F5C9EFF1FB89CFF1FEE
:101C300067BBCF46849EFF1F9889FF1FB5814E1B4F
:101C40002DE9F84F0C200BF0F3F90C200BF0A8FE57
:101C5000A74914200BF0B4FEA649A74808F0ECFEF3
:101C6000022103200BF042FF022104200BF03EFF73
:101C7000022105200BF03AFF022106200BF036FF6F
:101C800001210A200BF032FF012109200BF02EFF69
:101C900001210D200BF02AFF012128200BF026FF47
:101CA000012114200BF022FF02210B200BF01EFF5C
:101CB00001210C200BF01AFF0C2000210BF002FF79
:101CC00004200BF005FF002836D005200BF000FFA4
:101CD00000283BD00023894D06202B700BF0F8FE26
:101CE000B0FA80F35B090024854A137005F0E0FF29
:101CF0002B78EBB9204607F019FC824B82491B88F0
:101D0000824D0988824A2970A3F5AF7140F23A7377
:101D100003FB01F382FB0312DB177E4E7E48A3EB2D
:101D2000621332335A21336009F030FAA8B9FEE762
:101D3000BDE8F84F08F090BD06200BF0C9FE002862
:101D4000C3D16E4D034628700124CDE703200BF06C
:101D5000BFFEB0FA80F35B09BDE7704A70481268B5
:101D6000DFF804B200230121FEF79EFB0B200BF0ED
:101D7000AFFE011E0CBF012300238BF8003002D1FF
:101D800011200BF0B3FEDFF8A491664FDFF8DC8181
:101D9000654E0023C9F800303B60C8F800304FF0B2
:101DA000040A14E00BF078F93B68184438600AF034
:101DB000010080F0010004F0DBFB3388002B14BF2E
:101DC0004B20DC200BF0BAFEBAF1010A1BD00F2029
:101DD0000CF0A6F8D8F8003003440E20C8F8003004
:101DE0000BF05AF9D9F800309BF800200344C9F8E9
:101DF00000301520002AD5D111200CF091F83B6855
:101E000018443860D3E7D8F80030D9F800204749A3
:101E10003868DFF85CE1DFF85CC1002BB8BF033342
:101E2000002AB8BF033292100A604149414A09882A
:101E300012880028B8BF03309B10801038605F1AEA
:101E40001944CEF80070CCF80010DFF82CE13A4FBE
:101E50003A49C8F80030C2EB000C0244CEF800C08A
:101E60003A600B600CB1FFF797FD33885BB94FF414
:101E7000FA7004F08DFB04F077FB06F04DFA4FF496
:101E8000AF600BF05BFE2E4B012404201C600BF0B6
:101E90001FFE10B92B4B28701C702B4B1B881C2B62
:101EA0001CD02A4C04F1C80523200BF0F5F844F8A7
:101EB000040F01200BF042FEA542F5D1244A254B28
:101EC0001078187007F03CFA04F04AFB45F6BF5250
:101ED00021492248BDE8F84F0AF096BE204B1888E9
:101EE0000028DED01F4BC0B2197807F071F9D8E78F
:101EF000001B374640420F00E490FF1F329CFF1F3B
:101F0000C89DFF1F849EFF1F609EFF1F949CFF1FA4
:101F1000B5814E1B9889FF1FB89CFF1F2889FF1FA2
:101F2000F09DFF1FF89BFF1F1E9EFF1F0C9CFF1FB5
:101F3000A889FF1F2C89FF1F989CFF1F9C9EFF1FD5
:101F4000589EFF1F1C9CFF1F5E9EFF1FD09CFF1F03
:101F5000DC9DFF1FBE9DFF1FA50500007C9EFF1F8F
:101F60009C9CFF1F4C9CFF1F429EFF1F4C9EFF1F0F
:101F7000509EFF1FC49DFF1F589CFF1F2DE9F04F6F
:101F80008BB007ADC04F2C460AAE611BC9B2BF482B
:101F900009F0C0F83B88834294BF0020012004F878
:101FA000010BA642F1D1BA48BA4A9DF81C70BA4951
:101FB00007709DF81E00B94D10709DF820209DF807
:101FC0002430B74EB74C0A709DF8221029700025B6
:101FD0003370257073B9002940F01A81B2491AB1E3
:101FE0000B78002B40F00682002800F0DB810223F2
:101FF000237005E0002A40F0BB800523AA49237026
:10200000DFF8F8B2DFF8F8829DF81D209DF8210076
:10201000DFF8F092DFF8F0A2A44DA54FA54E0B70AB
:102020009DF81FC09DF823109DF827309DF826E0ED
:102030008BF8002088F800009DF8252029700120E9
:102040003A70337089F800C08AF800E00BF068FF3E
:10205000994A9A4B11688842CCBF012200221A701B
:1020600040F38A80964B1B88182B00F28580954A96
:10207000B2F800E00C3B0093BEF1000F40F0858009
:10208000914A9BF800C092F800B098F8008099F847
:1020900000209AF8009094F800A02C78ABEB4C0B41
:1020A000C2EB0B0BA8EB880EDE44C9EB897BC9EBB6
:1020B0008B09DFF81CB2F14497F800E0BBF800B0E0
:1020C00009EB44093478CE4404FB0BEE4FF00C09C5
:1020D0007E4C19FB0AEEC4F800E0B8F1000F0BD0FB
:1020E00036784EB17A4E3688042E0CBF0EF1020EB1
:1020F0000EF1040EC4F800E0764E774CDFF80CB217
:102100003688DBF800B02488DFF804A2DFF80492F8
:10211000BAF800A0B9F80090009BC6EBC6065E4472
:10212000033CDFF8F4B104EB4404DBF800B00EEB41
:1021300084045444C9EBC909DFF8E0A1D944DFF8AD
:10214000E0B15AF826605BF829900C3C1C44A319B6
:102150004B44BCF1000F29D02C783CB3002A5BD152
:10216000B8FA88F85D4C4FEA581884F8008024E0EB
:10217000062323704C4943E7524AB2F800E000239B
:102180000093BEF1000F3FF47BAFBEF1010F47D0CB
:10219000BEF1020F00F0C8804C4C9BF800C099F8CB
:1021A000002098F80080D4F800E096E74B4C00251A
:1021B00025700AB13A781ABB0022494C8842227035
:1021C0004849C4BF484AC2F800E00A68934213D0A5
:1021D000464A474C106805900598206012680692A0
:1021E000444C069A24880B60121AA24284BF424AC9
:1021F00013600BB0BDE8F08F3D483C4A0068EDE746
:10220000BCF1000FD8D1B8F1000FD5D10122D4E72D
:10221000042323702449F3E6304A00241470CBE7EA
:10222000294A9BF800C092F800E098F8008099F8DD
:10223000002094F800B09AF800902C780194AEEB4E
:102240004C0EC2EB0E0EA8EB88047444C9EBC9090E
:10225000D944A31EDFF878A0DFF8C8E0019C97F806
:1022600000B05EF829E0BAF800A096F8009003EB01
:1022700044045C4409FB0A4909F11809134CCE4493
:10228000C4F800E029E700BF849EFF1FB89CFF1F31
:10229000869EFF1F879EFF1F889EFF1F899EFF1F30
:1022A0008A9EFF1FCA9DFF1FD49DFF1FB59EFF1F63
:1022B000B69EFF1F649EFF1F9889FF1F109EFF1F81
:1022C0005E9EFF1F049CFF1FAA89FF1F189EFF1F11
:1022D0006C9CFF1F549EFF1F369EFF1F969EFF1F84
:1022E000979EFF1F789CFF1FA09EFF1FA09FFF1FB0
:1022F000689CFF1F6E9EFF1FA89EFF1FB19EFF1FC1
:10230000B39EFF1FB29EFF1FB49EFF1FCC9CFF1FFA
:10231000169CFF1F829CFF1F909EFF1F84210100BF
:10232000601C010070230100394A9BF800C092F83C
:1023300000B0247899F8002098F800800394ABEB63
:102340004C049AF80090334B95F800A0CDF804A007
:10235000A8EB880BA41A5C444FF0050B1BFB094B40
:10236000039C97F800A0CDF808A0C9EBC909B3F801
:1023700000A009EB0403BDF80490029C0BF1050BCF
:102380001EFB09BE96F800B0DFF8B090A6440BFB28
:102390000AEE59F82390204C0EF10C0ECE44C4F8EE
:1023A00000E09AE64FBB0B78012B2FD91B4A237014
:1023B00012882AB31A4A1288013A92B2062A1FD802
:1023C000184A1278E2B1184A1268012A7FF418AE4E
:1023D0001648174A0068174E82FB0025C217C2EB49
:1023E000650202EB4202A0EB82023280124A032015
:1023F000107005E60323237002E601232370FFE536
:10240000094A1268012A7FF4FBADEFE73B46F7E586
:10241000AA89FF1F6C9CFF1F189EFF1F409EFF1F75
:10242000DE9DFF1FC69CFF1F589EFF1FA89EFF1F1B
:10243000ABAAAA2A1C9EFF1F8C89FF1F082501003A
:102440002DE9F04F3A4B1B788BB0002B6BD10E204F
:102450000AF022FE0EF01EF901463648364E374D80
:10246000FEF768F83348FEF73BF80EF02DFB80F3DB
:102470000C003060FFF782FD2C68012C7AD0022C12
:1024800000F0B782032C00F0C9832D4E2D4C336829
:102490002D4A2E4E0993099B316812882360591AE0
:1024A000013A9142274F00F29F82294E32689A1AD0
:1024B0000D2A00F28882274E32689A1A132A00F2F7
:1024C0007D82254E32689A1A252A1AD9234B1B88F9
:1024D000002B40F06081224B1B78002B40F05B8189
:1024E000FEF7BCFE1F4B1B881B3B9BB2022B04D884
:1024F0001D4B1B78002B40F0518104F05BF82368E2
:1025000033601A4D2A689B1A502B00F21382184B25
:102510001B88012B00F02B8206F0EEFE06F01CFD5E
:102520000BB0BDE8F08F08F01FF80BB0BDE8F08FDE
:10253000329CFF1FF09DFF1F2C9EFF1F589EFF1F08
:10254000A09FFF1FEC9DFF1F9489FF1FC09CFF1FD2
:10255000AC9CFF1F8C9CFF1F909CFF1FD09DFF1FFA
:102560002C9CFF1F5E9EFF1F109EFF1FE09DFF1F04
:10257000309EFF1FDFF82C93A24AB9F800001378B1
:10258000834204D0C3B21846137006F0F1FDDFF8A1
:1025900010839D4AB8F800301178994204D09B4FBF
:1025A0003978002940F0F886994A33681288994EA4
:1025B0009A42C0F2FD80984A1278002A40F0F880D2
:1025C000DFF8E4A2BAF8003023B9944B1B88002B43
:1025D00000F00C85924A934B11881B88924A0B4459
:1025E00012685B109342914A126880F2AE84002117
:1025F0009342B4BF01230B4604910093ACBF4FF04C
:10260000010B8B4605910E200AF046FD884B894A46
:102610001B68176803930133A7F25232002B8446DC
:10262000029240F3E086802BA8BF8023824A834930
:1026300012780191002A00F0C5800978914200F0DB
:10264000C180B8F80010DFF858E2994201F0FD802F
:102650006E49AEF800307A4B4FF0010E81F800E081
:102660001978DFF848E2019B8EF800101A70009B81
:10267000002B00F01D81BAF80030002B00F018810B
:10268000704B1B685A1C002A40F3B186802A00F365
:10269000AD866D4C6D496E482488098800682144D8
:1026A000B0EB610FC1F24683A3F148020F2A02D8B2
:1026B000473BA9F800300E200AF0EEFC6FF454738B
:1026C0001F44874202DC634B00221A7000200BF08B
:1026D00027FC614A614B1168614C1B888842D4BF5A
:1026E000002201222270002B00F026845D4B1C7812
:1026F000944243D0884241DD5B490C78002C00F0C5
:102700003A875A4991F800C0BCF1000F40F0318778
:10271000574F0097574F58480297554F007887F802
:1027200000C0544F4FF0010E87F800C081F800E060
:10273000002841F0E18051490978002900F0FD8727
:102740004F4903910C460978002940F0F3874D4822
:10275000484F0078397001210297217070B14448C8
:1027600042490090484803270770002008700099EC
:10277000029F0870039901243C7008701A70434B43
:102780001B88A3F11B02012A40F2CA851D2B00F011
:1027900014863F4C7BE6FEF703FDA1E63D4B1B781C
:1027A000002B3FF4AAAE2B68012B7FF4A6AEA6E661
:1027B0003168394A069106983849106002220B6048
:1027C0002A60FDE61E49DFF8E4E0097800293FF4BD
:1027D0004AAF9EF8000081423FF445AF03984B2872
:1027E00040F3FA871833802BB8F80000A8BF802385
:1027F00098423FF438AF2A4803800448012303700D
:1028000031E700BFBE9DFF1F949CFF1F1C9CFF1F54
:10281000C49CFF1FA09FFF1F2C9CFF1FB29CFF1F8B
:10282000409CFF1F289EFF1F609CFF1F249CFF1FD2
:10283000A09EFF1F0C9CFF1F969EFF1F749CFF1FF6
:10284000979EFF1F189EFF1FD69DFF1FD29DFF1F43
:10285000509CFF1FC99DFF1F9889FF1FDE9DFF1F12
:10286000469CFF1FFC9BFF1FB49EFF1F209EFF1F67
:10287000729EFF1FC69CFF1FB59EFF1FB19EFF1FCC
:10288000FD9BFF1F109EFF1F8C89FF1F5E9EFF1F79
:10289000EC9DFF1F649EFF1F849CFF1FE89DFF1F90
:1028A000609EFF1FDC9DFF1F7C9CFF1F759CFF1F10
:1028B000029B9C45BFF6FFAE8B4B1B88002B3FF461
:1028C000FAAEBBF1000F7FF4DBAE884B1B881BB167
:1028D000059B002B7FF4D4AE049B002B3FF4EBAEA2
:1028E000834B1A78002A7FF4E6AEDFF8809299F8DD
:1028F000004001221A70002C40F045837D4B1B786C
:10290000002B02F0D8807C4B1B78002B02F09B83BD
:102910007A4B1B78002B7FF4CEAE794B1B78002BC3
:102920003FF4C9AEB8F8003076490A3BA8F8003049
:102930000A70C0E605F004FA734B1B7873B9734B49
:102940001B785BB9724B1B7843B9724B1B782BB960
:10295000714B1B7813B903F003FE01E003F00CFE8A
:1029600023682B606D4B1B88012B7FF4D5AD6C4A1F
:102970006C4B11686C481A78A1F118032A2101FBED
:1029800003F10160002A00F0C182684C236899427B
:1029900000F36A8310DA66480278002A40F09287D2
:1029A000644A1068D0F17F0048BF033080100130C6
:1029B0001B1A994242F3D0862160A9E2FEF742FF3A
:1029C000236833607DE5FDF7DBFFFEF773FC5A4BB0
:1029D0001B88032B00F02B85584B1B88032B00F022
:1029E00022852368336066E5FDF716FF3B68336098
:1029F0005BE5534A34681188A14204DB464B1B78DF
:102A0000002B00F061834F4E4F48336807934F4BC4
:102A1000079A00681B88121A9A4200F2AD80002BB8
:102A200000F0AA804A4B1A88002A3FF4B2AE494B04
:102A300049481B680088A342B8BF2346994241F326
:102A40007281464B1960DFF8288188F80020344FE6
:102A5000FDF7E2FE38687F2840F37D85404B7F38E4
:102A600083FB0032C317C3EB620303EB4303A0EB0A
:102A7000830073303B4B01931B883860002B40F080
:102A8000D686234B00931B78002B00F0CA83364C6C
:102A90002378002B00F0C583DFF8D890DFF8C0A0C2
:102AA0004FF0000B0CE003F17300C0B298F8001077
:102AB00006F0B6FB23780BF1010B5B4540F3B183C5
:102AC0003B6859F8040F1844A0F17F038AFB0321E7
:102AD000DA17C2EB610202EB42027F28A3EB82030A
:102AE000E1DCFDF7B9FDE0E7B29CFF1FE49DFF1FAD
:102AF000C99DFF1FB19EFF1FB29EFF1FB39EFF1F08
:102B0000B49EFF1F1C9CFF1FC69CFF1F209EFF1F23
:102B1000729EFF1FFD9BFF1F2C9CFF1F309EFF1FFF
:102B2000A89EFF1F809CFF1FA49CFF1FB49CFF1F3B
:102B3000789EFF1F749EFF1F329EFF1FC09DFF1FC8
:102B4000C49CFF1FA09FFF1F849CFF1FB09CFF1F02
:102B50001A9CFF1FE89DFF1F8C9EFF1F009CFF1FFC
:102B6000ABAAAA2A5C9CFF1F5489FF1FCA9DFF1FA6
:102B7000A09CFF1F2C89FF1F554B564A1B681088CD
:102B8000554AA342B8BF2346994200F38482534C6E
:102B900012888342A8BF03462360002A7FF453AF04
:102BA0009942C8BF134640F37D82401AB0F5804F6A
:102BB000AABF9B03C3EB8333013093FBF0F0FDF717
:102BC00011FEC0F3C6100DF065FD454B0446188894
:102BD0000DF060FD4349074620460DF0AFFD01466C
:102BE00038460DF0ABFD21460DF0A0FC4FF07E51B4
:102BF00004460DF041FF002841F079803A49204613
:102C00000DF058FF002840F0718620460DF082FF3D
:102C1000C0B2DFF8F48088F8000018E7334B34685E
:102C20001988A14274DD324B1B78002B70D1DFF87C
:102C3000DC9099F800007F2840F34086A3F15533DB
:102C40007F3803F1004383FB0032C317C3EB6203F9
:102C500003EB4303A0EB83007330264B01931B88E7
:102C6000C0B289F80000002B41F03380224B009362
:102C70001B78002B00F0AC84204C2378002B00F054
:102C8000A7841F4FDFF87C804FF0000A0AE003F1B1
:102C90007300C0B206F0ECFA23780AF1010A53453A
:102CA00040F3968457F8043F99F800001844A0F1C7
:102CB0007F0388FB0321DA17C2EB610202EB4202B9
:102CC0007F28A3EB8203E2DCFDF7C6FCE1E700BF4F
:102CD000E89DFF1F8C9EFF1F1A9CFF1F009CFF1F7B
:102CE000989EFF1FCDCCCC3D0000FE42C49CFF1F30
:102CF0002C9CFF1F5C9CFF1F729EFF1F5489FF1FAF
:102D00002C89FF1FABAAAA2AA09CFF1F149EFF1F9D
:102D1000B84F38687F2840F3CC81B74B7F3883FBAE
:102D20000032C317C3EB620303EB4303A0EB830042
:102D30007330DFF8249399F800A0824500F01782E1
:102D4000AE4B1B88002B43D1AD4AAE4812680088B9
:102D5000914205DC8242D4BFC1EB0203C1EB000308
:102D6000411AB1F5804FA6BF9B030131C3EB8333FA
:102D700093FBF1F0FDF736FDC0F3C6100DF08AFCB1
:102D8000A14B044618880DF085FCA04980462046DA
:102D90000DF0D4FC014640460DF0D0FC21460DF06C
:102DA000C5FB4FF07E5104460DF066FE002840F052
:102DB0000A87974920460DF07DFE002840F0938554
:102DC00020460DF0A7FEC0B2DFF8908288F8000020
:102DD000BAF17F0F40F3B8838748AAF17F0A80FBDE
:102DE0000A304FEAEA73C3EB600000EB4000AAEB45
:102DF00080007330874B00931B78C0B289F80000C5
:102E0000002B40F01883844B03931B78002B40F079
:102E10004985824B02931B78002B40F07C87804BC6
:102E20000193029B1B78FBB17E4B1B88012B00F0AA
:102E3000C185022B01F04D80032B01F08C81042B06
:102E400001F09783052B01F03884062B01F0FF85F4
:102E5000072B01F0BB87082B02F0BA80092B02F088
:102E6000BF810A2B02F09283009B1B78002B00F09D
:102E70007484019B6A4C1988002900F0FB8438682F
:102E80007F2840F365835C4B7F3883FB0032C31798
:102E9000C3EB620303EB4303A0EB830073303860A2
:102EA000002940F0AA84009B1B78002B00F06B8166
:102EB0005D4C2378002B00F06681DFF8A4A1DFF8D9
:102EC0009C814FF0000B0CE003F17300C0B298F846
:102ED000001006F0A5F923780BF1010B5B4540F3D8
:102EE00052813B685AF8040F434A1844A0F17F030B
:102EF00082FB0321DA17C2EB610202EB42027F2858
:102F0000A3EB8203E0DCFDF7A7FBDFE7474B19608B
:102F1000474B1B68A92202FB03F3002BBCBF03F540
:102F20007F533F339B13543B194481F30C012820FA
:102F30000AF038FCFFF7F0BA384C3E483549364ABB
:102F4000237003700B70137019E493424FF0000B61
:102F500080F2B2800123CDF800B0CDF814B0049314
:102F6000FFF751BB344B1B78002B7FF4A4AB039BC2
:102F7000324A243B83F34703D9B25B20136006F047
:102F800027F999F80040032C30D1DFF8D88098F861
:102F90000030002B42F05D82294F3B78002B42F03D
:102FA0004B82254C2378002B42F03982254B1B782D
:102FB000002B42F02782244A1380244B1B78002BDD
:102FC00042F013820D4B7F221A8098F800306BB9C3
:102FD0003B785BB923784BB91D4A7F2107201380CA
:102FE00006F0F6F87F210B2006F0F2F8194B1F6867
:102FF000FFF761BBA89EFF1FABAAAA2A1A9CFF1F5E
:10300000009CFF1F8C9EFF1F989EFF1FCDCCCC3DC8
:103010000000FE42729EFF1FFD9BFF1FC69CFF1F0C
:103020005C9CFF1FDE9DFF1F5489FF1FB49CFF1F88
:103030009089FF1F209EFF1FB49EFF1F3C9CFF1F17
:10304000B39EFF1FB29EFF1FBA9CFF1FB59EFF1FBE
:10305000129EFF1F0C9CFF1F149EFF1FA09CFF1FB2
:103060002C89FF1FB19EFF1FB64A1078002840F040
:103070005783B54A1268D2F17F0248BF033203EB8F
:10308000A202531CB14A23609942B8BF1160FFF6F7
:103090003FAF19463CE7AE4B12881960002A7FF417
:1030A000D2AC0B469842D4BFC1EB0003C1EB030383
:1030B0007BE5FDF7D1FA3CE60123CDF810B0CDF861
:1030C00000B00593FFF79FBA01232B60A14EA24CDD
:1030D000FFF7DDB9029B1B78FBB1A04B1B88012BCE
:1030E00000F0EA84022B00F07386032B01F0A98024
:1030F000042B01F06382052B01F05683062B01F0AF
:10310000AF84072B01F0AF85082B01F01987092B3D
:1031100002F02F800A2B02F0C381019B1B88002B39
:1031200000F07483009B1B783BB9039B1B7823B989
:10313000029B1B78002B01F00480894B1B78002B2D
:1031400000F0FE8087490B78082B00F2F980864852
:103150003A680068854C0133DBB25F1E101A44F8F0
:1031600027000B70824B3468198889F800208C4244
:10317000784E7FF70EAB32687E4B0892089A764CF9
:103180001A60FFF784B9039B1B78002BA2D03B6821
:10319000A3F10C007F2840F3828377488B3B80FBB0
:1031A0000320DA17C2EB600000EB4000A3EB8003C2
:1031B00003F17300DFF8D481C0B298F8001006F074
:1031C0002FF8009B1B78002B84D0664C2378002BB3
:1031D00080D0DFF8BCA14FF0000B0CE003F17300CE
:1031E000C0B298F8001006F01BF823780BF1010B21
:1031F0005B457FF76FAF3B685AF8040F5E4A18448F
:10320000A0F18B0382FB0321DA17C2EB61020C38B9
:1032100002EB42027F28A3EB8203DFDCFDF71CFAFE
:10322000DEE74F4B1B78002B40F0F6823B68534A99
:103230001278002A45D0A3F10C007F2840F33B838D
:103240004D4A8B3B82FB0321DA17C2EB610202EB92
:103250004202A3EB820303F17300C0B298F800109E
:1032600005F0DEFF009B1B7853B33E4C23783BB345
:10327000DFF81C91DFF800A14FF0000B0BE003F129
:103280007300C0B298F8001005F0CAFF23780BF164
:10329000010B5B4514DD3B6859F8040F1844A0F19D
:1032A0008B038AFB0321DA17C2EB61020C3802EBB5
:1032B00042027F28A3EB8203E1DCFDF7CDF9E0E7D2
:1032C0003B682F4A1278FAB1244A1288012A00F08A
:1032D0007D84022A00F07B86032A01F02F80042AD5
:1032E00001F09381052A01F0CC82062A01F0D083F7
:1032F000072A01F01384082A01F0D386092A01F075
:1033000090870A2A02F00A81019A1288002A00F0A6
:1033100095821C4A104C137003232B60FFF7B7B83B
:10332000DFF8708098F80030002B40F01881164FBD
:103330003B78002B40F01485074C3B70FFF7A7B893
:103340003A680FE7789EFF1F749EFF1FB49CFF1F13
:10335000009CFF1FA09FFF1FEC9DFF1FDE9DFF1F16
:10336000209EFF1F5489FF1F209CFF1F3089FF1FD5
:10337000C49CFF1F4C9FFF1FABAAAA2AFD9BFF1FE7
:10338000C69CFF1F149EFF1F189CFF1FA09CFF1FC1
:103390002C89FF1F109EFF1FDBB21846137005F02B
:1033A000F5FEB04BB0491A46B04B184600230B70DF
:1033B0003B7013700370FFF7F7B8DFF8CC8298F812
:1033C0000030002B40F0D781A94F3B78002BB3D0C1
:1033D000A84BA94C1988A22006F07EF898F8003076
:1033E0003B70FFF754B80123FFF720B98024A349AD
:1033F000A34BA44A09881B8812680B44B2EB630FE5
:10340000BFF659A9A04B1B78002B40F02482B8F8D6
:1034100000309E4AA3423FF44EA99D4B14800122E6
:103420001A70FFF748B9FDF77FF9FFF7DABAFDF731
:1034300025F9FFF7D1BA974B01931B88002B42F077
:1034400085818A4B0393944B0293944C23786BB3FE
:10345000DFF85C82DFF848A24FF0000B09E003F1CF
:103460007300C0B205F004FF23780BF1010B5B453C
:103470001CDD58F8043F99F800001844A0F17F03C0
:103480008AFB0321DA17C2EB610202EB42027F28BA
:10349000A3EB8203E3DCFDF7DFF8E2E77E4B029368
:1034A00005F0E6FE009B1B78002BCED1039B1B781A
:1034B000002B3FF4B6AC99F80030A3F10C007F2844
:1034C00040F3EA8176488B3B80FB0320DA17C2EB9E
:1034D000600000EB4000A3EB800303F17300C0B277
:1034E00005F0C6FE009B1B78002B00F0CA816B4CD8
:1034F0002378002B01F0C582DFF8B481DFF8A0A1AA
:103500004FF0000B0AE003F17300C0B205F0B0FE0B
:1035100023780BF1010B5B457FF783AC58F8043F30
:1035200099F800001844A0F18B038AFB0321DA17F5
:10353000C2EB61020C3802EB42027F28A3EB82034C
:10354000E1DCFDF789F8E0E75046FDF785F851E446
:10355000FDF782F8A3E4FDF77FF8FFF78BBA514A35
:103560001278002A40F0D581414F434C3B70FEF762
:103570008EBF002008704C49087840B1394900914D
:103580000978002900F0B581009F00213970474972
:10359000097800297FF4D4A8002C40F0CE800028C0
:1035A00040F0CB80384C2F4F94F800E02F4C039420
:1035B000394C02942D4C2C492070374C00970870E0
:1035C00038702070BEF1000F7FF4CCA8FFF7D6B89A
:1035D000264B1B78002B6DD099F80030A3F10C001E
:1035E0007F2840F3C8832E4A8B3B82FB0321DA17E6
:1035F000C2EB610202EB4202A3EB820303F1730010
:10360000C0B205F035FE009B1B78002B52D0234C36
:103610002378002B4ED0264FDFF884804FF0000A2D
:1036200009E003F17300C0B205F022FE23780AF12D
:10363000010A53453EDD57F8043F99F8000018444D
:10364000A0F18B0388FB0321DA17C2EB61020C386F
:1036500002EB42027F28A3EB8203E2DCFCF7FCFFD3
:10366000E1E700BF729EFF1F209EFF1FFD9BFF1F13
:10367000189CFF1F629EFF1FEC9DFF1FD69DFF1F22
:10368000D29DFF1F509CFF1F109EFF1F609EFF1FBB
:103690001C9CFF1F5C9CFF1FC69CFF1F5489FF1FC3
:1036A000ABAAAA2A649EFF1FB59EFF1FB19EFF1FF3
:1036B0002C89FF1FA84B1B78FBB1A84B1B88012B43
:1036C00000F0D086022B00F0CB87032B01F0428163
:1036D000042B01F0CD81052B01F01784062B01F09E
:1036E000D884072B01F0E785082B01F07087092BA0
:1036F00001F0D5870A2B01F0A287019B1B88002BC4
:1037000000F0F082964B1B78002B40F0E682954B40
:10371000954A198834680020012310602B6026E543
:103720000130C0B2022886BF002111701070194606
:10373000FFF7EEBB0398002101708C49097800293E
:103740003FF41CA8844902910978002900F0AE8753
:10375000029800210170FFF711B8039B1B78002B22
:103760007FF487AB029B1B78002B7FF482AB019B1D
:103770001988FFF784BB7E4A1278002A3FF4F4AE22
:103780007C4F387802F066FF7B4B1B78002B00F0F3
:10379000B78439887E2900F2B384784CDFF80C9224
:1037A0002368D9F800209B1A0F2B40F29680744BA7
:1037B00001311B8889B239802BB1052B03D0C9B2E6
:1037C000052005F005FD6F4F226898F80030C9F814
:1037D00000203B70FEF75BBE243B002BB8F80000D6
:1037E00040F3748498423EF43EAF9BB26648A8F81A
:1037F000003001230370FEF736BFDFF89081C0B2BE
:1038000098F8001005F00CFDFFF74DBB5F4B3878C2
:10381000197805F005FD85E47F21402005F0D8FCEE
:103820005B495C4A3B680B6000211170FFE4C0B249
:1038300098F8001005F0F4FCFFF723B9D8B298F817
:10384000001005F0EDFC3B6863E5534BDFF860E1E9
:103850001978FEF708BF4B2C40F34C821834802CAB
:10386000B8F800304D4AA8BF8024A3427FF4D5ADFC
:10387000FEF721BF99F8000005F0FAFC2188FFF758
:10388000FEBA029B1B78002B7FF4CEAA039B1B7809
:10389000002B7FF4EEAA6AE7FCF7DEFE1FE6FCF7DA
:1038A000DBFE87E43E4B01931B88002B7FF4F6ADD3
:1038B000294B0293FFE5FCF7CFFECEE4FCF7CCFEEC
:1038C000FFF7CBB90132D2B2022A40F25A8200226B
:1038D00002701946FFF71CBB284C2A4F98F800309D
:1038E0003B70FEF7D4BD7F20FFF76EBA7F20FFF755
:1038F00090B9194F1A4902974FF0000C81F800C097
:10390000009F02994FF0010E87F800E081F800C097
:103910003DE6244F387802F09DFE174B1B78002BB4
:1039200000F0368239887E2900F23282134CDFF8AB
:103930007C902368D9F800209B1A0F2BCDD91A4B05
:103940000131188889B23980002800F03D82C9B25F
:10395000C0B205F03DFC36E7C69CFF1FDE9DFF1F91
:10396000209EFF1FC49CFF1F009CFF1F109EFF1F77
:10397000649EFF1F629EFF1FB69EFF1FEC9DFF1FF0
:10398000CA9CFF1F189CFF1F1C9CFF1FA09CFF1FB1
:10399000209CFF1F5489FF1F979EFF1F609EFF1FE3
:1039A0005C9CFF1F4C9CFF1F9C9CFF1FA49EFF1F45
:1039B000759CFF1FDFF89CA399F80000BAF800304F
:1039C000DF4AE04CC31A82FB031ED917C1EB6E011C
:1039D00001EB4101A3EB810303EB430354F82330D4
:1039E00018447F2840F3A6847F3882FB0032C31737
:1039F000C3EB620303EB4303A0EB83007330DFF8F8
:103A000058B3C0B205F034FCBBF80030022B7FF68F
:103A10002BAA99F80010BAF80030C94ACB1A82FBD9
:103A2000030ED817C0EB6E0000EB4000A3EB800341
:103A300003EB430304EB8303586808447F2840F3F7
:103A400018877F3882FB0032C317C3EB620202EB98
:103A50004202A0EB82007330C0B205F009FCBBF853
:103A60000030032B7FF600AA99F80010BAF8003056
:103A7000B34ACB1A82FB030ED817C0EB6E0000EBE3
:103A80004000A3EB800303EB430304EB8304A06833
:103A900008447F2840F351817F3882FB0032C317EE
:103AA000C3EB620202EB4202A0EB82007330C0B2B1
:103AB00005F0DEFBFFF7D8B9DFF898A23868BAF84E
:103AC00000309F4A9F4CC31A82FB031ED917C1EBDB
:103AD0006E0101EB4101A3EB810303EB430354F8B7
:103AE000233018447F2840F3A0847F3882FB0032C3
:103AF000C317C3EB620303EB4303A0EB83007330F4
:103B0000DFF85882DFF850B298F80010C0B205F024
:103B100087FBBBF80030022B7FF6FFAA3968BAF8A2
:103B20000030874ACB1A82FB030ED817C0EB6E0019
:103B300000EB4000A3EB800303EB430304EB8303A0
:103B4000586808447F2840F398867F3882FB00320B
:103B5000C317C3EB620202EB4202A0EB8200733098
:103B6000C0B298F8001005F05BFBBBF80030032BE7
:103B70007FF6D3AA3968BAF80030714ACB1A82FBB3
:103B8000030ED817C0EB6E0000EB4000A3EB8003E0
:103B900003EB430304EB8304A06808447F2840F34D
:103BA000F4807F3882FB0032C317C3EB620202EB62
:103BB0004202A0EB8200733098F80010C0B205F00A
:103BC0002FFBFFF7AABA0120FFF7FEB8DFF884A1A8
:103BD0005B49BAF800205B4C9A1A81FB020ED017A1
:103BE000C0EB6E0000EB4000A2EB800202EB420251
:103BF00054F8220018447F2840F31B84A0F17F036F
:103C000081FB0321DA17C2EB610000EB4000A3EB5C
:103C100080007330DFF840B198F80010C0B205F0B2
:103C2000FFFABBF80030022B50D93968BAF80030DF
:103C3000434ACB1A82FB030ED817C0EB6E0000EB91
:103C40004000A3EB800303EB430304EB83035868BA
:103C500008447F2840F3E1867F3882FB0032C31797
:103C6000C3EB620202EB4202A0EB82007330C0B2EF
:103C700098F8001005F0D4FABBF80030032B25D9D2
:103C80003868BAF800302E4AC31A82FB031ED917CF
:103C9000C1EB6E0101EB4101A3EB810303EB430395
:103CA00004EB8304A36818447F2867DD7F3882FB18
:103CB0000032C317C3EB620202EB4202A0EB8200A8
:103CC0007330C0B298F8001005F0AAFA3B68FFF70D
:103CD0001BBB05F0CDFAFEF7C9BF0021402005F05F
:103CE00077FA14E599F8000005F0C2FA0AE5012018
:103CF000FEF78FBF243C002CB8F8003040F3248638
:103D0000A3423EF4D8ACA4B20F4BA8F80040012265
:103D10001A70FEF7D0BC0D4B01931B88002B7FF46B
:103D2000BFABFFF77EB80A498342A8BF03460B60CA
:103D3000FEF789BE1446FFF765BBFCF78DFCB6E6BF
:103D4000ABAAAA2A642001001C9CFF1F5C9CFF1FD9
:103D5000009CFF1F1C9EFF1F309CFF1FA09CFF1F8D
:103D6000DD4BDE4C19886A2005F0B6FB98F8003070
:103D70003B70FEF78CBBFCF76FFC41E4FCF76CFC7E
:103D80009FE702701946FFF7C3B8FCF765FC13E71D
:103D9000D34B1B78002B3FF49FAD3B88CE4F002BBD
:103DA0003FF49AADCD4CDFF848932268D9F8001063
:103DB000521A0F2A7FF691ADCA4A013B108899B278
:103DC000398000287FF4C3ADC8B205F075FAFAE473
:103DD000DFF820A33868BAF80030C34AC34CC31ACE
:103DE00082FB031ED917C1EB6E0101EB4101A3EB6E
:103DF000810303EB430354F8233018447F2840F336
:103E000028847F3882FB0032C317C3EB620303EBC5
:103E10004303A0EB83007330DFF8DC82DFF8DCB211
:103E200098F80010C0B205F0FBF9BBF80030022B87
:103E30007FF673A93968BAF80030AB4ACB1A82FB17
:103E4000030ED817C0EB6E0000EB4000A3EB80031D
:103E500003EB430304EB8303586808447F2840F3D3
:103E600026867F3882FB0032C317C3EB620303EB65
:103E70004303A0EB83007330C0B298F8001005F044
:103E8000CFF9BBF80030032B7FF647A93868BAF8A2
:103E90000030954AC31A82FB031ED917C1EB6E018D
:103EA00001EB4101A3EB810303EB430304EB830428
:103EB000A36818447F287FF768AF7F3882FB003201
:103EC000C317C3EB620303EB4303A0EB8300733020
:103ED00072E6DFF820A299F80000BAF80030824AB2
:103EE000824CC31A82FB031ED917C1EB6E0101EB92
:103EF0004101A3EB810303EB430354F8233018443F
:103F00007F2840F37F837F3882FB0032C317C3EBE7
:103F1000620303EB4303A0EB83007330DFF8DCB1F3
:103F2000C0B205F0A5F9BBF80030022B7EF69CAFBD
:103F300099F80010BAF800306B4ACB1A82FB030ED6
:103F4000D817C0EB6E0000EB4000A3EB800303EB3F
:103F5000430304EB8303586808447F2840F39F859C
:103F60007F3882FB0032C317C3EB620303EB4303CA
:103F7000A0EB83007330C0B205F07AF9BBF80030D3
:103F8000032B7EF671AF99F80010BAF80030564A4C
:103F9000CB1A82FB030ED817C0EB6E0000EB40007B
:103FA000A3EB800303EB430304EB8304A068084402
:103FB0007F287FF7C2AE7F3882FB0032C317C3EB86
:103FC000620303EB4303A0EB830073306FE5DFF87C
:103FD00024A14549BAF80020444C9A1A81FB020EEC
:103FE000D017C0EB6E0000EB4000A2EB800202EBAA
:103FF000420254F8220018447F2840F32E83A0F197
:104000007F0381FB0321DA17C2EB610000EB400064
:10401000A3EB80007330DFF8E4B098F80010C0B272
:1040200005F0FEF8BBF80030022B7FF64FAE396882
:10403000BAF800302C4ACB1A82FB030ED817C0EB1B
:104040006E0000EB4000A3EB800303EB430304EBA3
:104050008303586808447F2840F325857F3882FB16
:104060000032C317C3EB620303EB4303A0EB8300EF
:104070007330C0B298F8001005F0D2F8BBF80030E9
:10408000032B7FF623AE3868BAF80030164AC31AFD
:1040900082FB031ED917C1EB6E0101EB4101A3EBBB
:1040A000810303EB430304EB8304A36818447F28D4
:1040B0007FF764AE7F3882FB0032C317C3EB620325
:1040C00003EB4303A0EB83007330FAE501283EF4D1
:1040D000CAAA0123FFF78ABB4C9CFF1FEC9DFF1F60
:1040E000B59EFF1F9C9CFF1FABAAAA2A2C22010091
:1040F000A49EFF1F1C9EFF1FA09CFF1F309CFF1F44
:10410000CE4B1B78002B3FF4E7AB3B88CC48012B10
:104110007FF6E2ABCB4CDFF83C932268D9F8001075
:10412000521A0F2A7FF6D9ABC74A013B128899B2BF
:104130000180002A3FF447AB052A7FF440ABFFF72C
:1041400042BB4FF47A43013BFDD199F8000005F0E2
:104150008FF8FEF7F2BFDFF800A399F80000BAF875
:104160000030BA4ABA4CC31A82FB031ED917C1EBFE
:104170006E0101EB4101A3EB810303EB430354F810
:10418000233018447F2840F3E8817F3882FB0032D7
:10419000C317C3EB620202EB4202A0EB8200733052
:1041A000DFF8B8B2C0B205F063F8BBF80030022BFC
:1041B0007EF65AAE99F80000BAF80030A34AC31A46
:1041C00082FB0321DA17C2EB610202EB4202A3EB8E
:1041D000820303EB430304EB83035B6818447F28EB
:1041E00040F325847F380C2290FBF2F302FB13008E
:1041F0007330C0B205F03CF8BBF80030032B7EF6FC
:1042000033AE99F80000BAF80030904AC31A82FB26
:104210000321DA17C2EB610202EB4202A3EB820335
:1042200003EB430304EB8304A36818447F287FF760
:1042300084AD7F380C2290FBF2F302FB1300733045
:1042400035E4DFF814A23868BAF800307F4A804CB1
:10425000C31A82FB031ED917C1EB6E0101EB4101AA
:10426000A3EB810303EB430354F8233018447F2866
:1042700040F370817F3882FB0032C317C3EB6202C8
:1042800002EB4202A0EB82007330DFF8D481DFF84A
:10429000CCB198F80010C0B204F0C2FFBBF80030F7
:1042A000022B7EF63AAF3868BAF80030674AC31A74
:1042B00082FB0321DA17C2EB610202EB4202A3EB9D
:1042C000820303EB430304EB83035B6818447F28FA
:1042D00040F3B4837F380C2290FBF2F302FB13000F
:1042E0007330C0B298F8001004F09AFFBBF80030A9
:1042F000032B7EF612AF3868BAF80030534AC31A5F
:1043000082FB0321DA17C2EB610202EB4202A3EB4C
:10431000820303EB430304EB8304A36818447F2860
:104320007FF733AD7F380C2290FBF2F302FB1300D2
:10433000733041E4FCF790F9FFF761BBDFF818A197
:104340004249BAF80020424C9A1A81FB020ED0175B
:10435000C0EB6E0000EB4000A2EB800202EB4202D9
:1043600054F8220018447F2840F3FA80A0F17F031C
:1043700081FB0321DA17C2EB610101EB4101A3EBE1
:1043800081007330DFF8D4B098F80010C0B204F0A8
:1043900047FFBBF80030022B7FF698AC3868BAF8BC
:1043A00000302A4AC31A82FB0321DA17C2EB6102EA
:1043B00002EB4202A3EB820303EB430304EB830310
:1043C0005B6818447F2840F33C837F380C2290FBC5
:1043D000F2F302FB13007330C0B298F8001004F03F
:1043E0001FFFBBF80030032B7FF670AC3868BAF8BB
:1043F0000030164AC31A82FB0321DA17C2EB6102AE
:1044000002EB4202A3EB820303EB430304EB8304BE
:10441000A36818447F287FF7B1AC7F380C2290FB4B
:10442000F2F302FB130073304BE4FCF715F9FFF7CE
:1044300067BBFCF711F9FFF7EDBB00BFB59EFF1F8F
:10444000629EFF1FEC9DFF1FCA9CFF1FABAAAA2AFA
:10445000BC220100A49EFF1F1C9EFF1F309CFF1F5B
:10446000A09CFF1FDFF838A399F80000BAF80030CD
:10447000C34AC44CC31A82FB0317D917C1EB6701A7
:1044800001EB4101A3EB810303EB430354F8233019
:1044900018447F286ADD7F3882FB0032C317C3EBE4
:1044A000620202EB4202A0EB82007330DFF8F4B24A
:1044B000C0B204F0DDFEBBF80030022B7FF61DA970
:1044C00099F80000BAF80030AD4AC31A82FB032104
:1044D000DA17C2EB610202EB4202A3EB820303EBA9
:1044E000430304EB83035B6818447F2840F3AC82EA
:1044F0007F380C2290FBF2F302FB13007330C0B242
:1045000004F0B6FEBBF80030032B7FF6F6A899F84E
:104510000000BAF800309A4AC31A82FB0321DA1766
:10452000C2EB610202EB4202A3EB820303EB430303
:1045300004EB8304A36818447F2814DD7F380C2221
:1045400090FBF2F302FB13007330C0B204F090FE54
:10455000FFF7D3B8FCF780F897E6FCF77DF81FE685
:10456000FCF77AF80EE7FCF777F8EEE7FCF774F85B
:104570009CE7DFF82CA299F80000BAF80030804AD6
:10458000814CC31A82FB031ED917C1EB6E0101EBEC
:104590004101A3EB810303EB430354F82330184498
:1045A0007F28DADD7F3882FB0032C317C3EB62035A
:1045B00003EB4303A0EB83007330F1E5DFF8E0A1E8
:1045C0003868BAF800306E4A6F4CC31A82FB031E7B
:1045D000D917C1EB6E0101EB4101A3EB810303EBA2
:1045E000430354F8233018447F28B3DD7F3882FB1F
:1045F0000032C317C3EB620303EB4303A0EB83005A
:10460000733042E6FCF728F888E4DFF894A15C49AF
:10461000BAF800205C4C9A1A81FB020ED017C0EB4E
:104620006E0000EB4000A2EB800202EB420254F865
:10463000220018447F2893DDA0F17F0381FB032132
:10464000DA17C2EB610000EB4000A3EB800073308F
:1046500098E6FCF701F8FFF7DFBBFBF7FDFFDAE4B4
:10466000DFF83CA199F80000BAF80030444A474C02
:10467000C31A82FB0317D917C1EB670101EB410194
:10468000A3EB810303EB430354F8233018447F2842
:104690007FF76CAF7F3882FB0032C317C3EB620336
:1046A00003EB4303A0EB83007330FFE63848009030
:1046B000384839490390FEF755B8DFF8E4A099F877
:1046C0000000BAF800302E4A344CC31A82FB032192
:1046D000DA17C2EB610202EB4202A3EB820303EBA7
:1046E000430354F8233018447F2840F3A4817F38D3
:1046F0000C2290FBF2F302FB13007330DFF8A4B03E
:10470000C0B204F0B5FDBBF80030022B19D999F8FE
:104710000000BAF800300C22C11A91FBF2F302FB40
:10472000131302FB03435B6818447F2840F384841F
:104730007F3890FBF2F302FB13007330C0B204F039
:1047400097FDBBF80030032B7EF68EABBAF8003035
:1047500099F800000C22C11A91FBF2F302FB13132B
:1047600002FB0344A36818447F287FF7E6AA7F383A
:1047700090FBF2F302FB13007330FFF798B900BF10
:10478000ABAAAA2A64200100D01C01002C2201003F
:10479000729EFF1FFD9BFF1F209EFF1F40250100F3
:1047A0001C9EFF1F309CFF1FDFF864A33868BAF817
:1047B0000030CE4ACE4CC31A82FB0321DA17C2EB7B
:1047C000610202EB4202A3EB820303EB430354F8C2
:1047D000233018447F2840F324817F380C2290FB3B
:1047E000F2F302FB13007330DFF82883DFF828B3FD
:1047F00098F80010C0B204F013FDBBF80030022B93
:104800001AD93868BAF800300C22C11A91FBF2F3B9
:1048100002FB131302FB03435B6818447F2840F339
:10482000D4837F3890FBF2F302FB13007330C0B2E5
:1048300098F8001004F0F4FCBBF80030032B7EF66F
:104840006CACBAF8003038680C22C11A91FBF2F354
:1048500002FB131302FB0344A36818447F287FF76D
:1048600094AA7F3890FBF2F302FB13007330FFF73A
:10487000A3B9FBF7F1FEFFF7EFB8FBF7EDFEFFF78B
:104880006FB9DFF88CA29949BAF80020984C9A1AAF
:1048900081FB0210D117C1EB600101EB4101A2EBDA
:1048A000810202EB420254F8220018447F2840F3B0
:1048B000BB80A0F17F030C2093FBF0F200FB1230D1
:1048C0007330DFF854B298F80010C0B204F0A8FCBE
:1048D000BBF80030022B1AD93868BAF800300C2225
:1048E000C11A91FBF2F302FB131302FB03435B6853
:1048F00018447F2840F39D837F3890FBF2F302FB3E
:1049000013007330C0B298F8001004F089FCBBF8B3
:104910000030032B7FF6DAA9BAF8003038680C2291
:10492000C11A91FBF2F302FB131302FB0344A368C9
:1049300018447F287FF722AA7F3890FBF2F302FB0E
:1049400013007330FFF7BDB9012B3DF4B4AE012461
:10495000FFF7DAB9DFF8B8A199F80000BAF800302B
:10496000624A644CC31A82FB0321DA17C2EB61026C
:1049700002EB4202A3EB820303EB430354F8233020
:1049800018447F2846DD7F380C2290FBF2F302FBAF
:1049900013007330DFF880B1C0B204F069FCBBF8DB
:1049A0000030022B19D999F80000BAF800300C2217
:1049B000C11A91FBF2F302FB131302FB03435B6882
:1049C00018447F2840F38F807F3890FBF2F302FB7E
:1049D00013007330C0B204F04BFCBBF80030032B63
:1049E0007EF68BAEBAF8003099F800000C22C11A9E
:1049F00091FBF2F302FB131302FB0344A368184478
:104A00007F287FF7B0AD7F3890FBF2F302FB1300F5
:104A100073309AE5FBF720FEBCE7FBF71DFEFFF7BE
:104A200026B9FBF719FEDFE6FBF716FE49E7FBF7B1
:104A300013FEFFF7DEBBFBF70FFE5FE6FBF70CFE96
:104A40004FE4FBF709FEC7E4FBF706FE57E5DFF886
:104A5000C0A099F80000BAF80030244A264C34E689
:104A6000DFF8ACA03868BAF80030204A224CA2E641
:104A7000DFF89CA099F80000BAF800301B4A1F4CE0
:104A800070E7029B1B78002B7EF4CEA9FEF7F1B9EC
:104A9000DFF87CA01549BAF80020174CF7E6FBF7C1
:104AA000DBFDFFF768BAFBF7D7FDFFF7E2BAFBF7CC
:104AB000D3FDFFF7E1B9124B1B78002B00F0D68233
:104AC000104B1B78002B7DF4F6AD0F4B1B78002BA1
:104AD0003DF4F1ADB8F800300C490A33A8F80030C5
:104AE0000A70FDF7E8BDFBF7B7FD73E7ABAAAA2A8A
:104AF00040250100BC220100E8230100D01C010078
:104B0000B29EFF1FB39EFF1FB49EFF1F1C9CFF1F82
:104B10001C9EFF1FA09CFF1F309CFF1FA44C2288DF
:104B2000002A00F02383A349DFF89CB20988BBF870
:104B300000000331884227DD9F48A0490088B1F872
:104B400000E0DFF87CC2181A0C2190FBF1F901FBA0
:104B500019004FF0900909FB0EFE01FB00E06FF019
:104B60000B0E5CF8000003440EFB02307F2840F37C
:104B7000CE847F3890FBF1F301FB13007330C0B299
:104B800098F8001004F04CFBBBF800202388134475
:104B9000022B23DD884B894A38681B88B2F800C095
:104BA000DFF81CE2C31A0C2193FBF1F201FB123275
:104BB000902303FB0CF301FB023373445B6818443E
:104BC0007F2840F3A7857F3890FBF1F301FB1300AA
:104BD0007330C0B298F8001004F022FBBBF800203C
:104BE00023881344032B23DD734B744A38681B88D6
:104BF000B2F800C0DFF8C8E1C31A0C2193FBF1F250
:104C000001FB1232902303FB0CF301FB02337344CC
:104C10009B6818447F2840F30B857F3890FBF1F3A5
:104C200001FB13007330C0B298F8001004F0F8FADA
:104C3000BBF8002023881344042B7FF747A85D4B63
:104C40001B88012B7FF442A83A68A2F10C007F2850
:104C50007FF794A88B3A0C2092FBF0F300FB132013
:104C60007330FFF72EB8524C2388002B40F00D8391
:104C7000DFF854B15049514A0988D7F80080B2F89A
:104C800000E04F48C1EB080C0C229CFBF2F102FB48
:104C900011C14FF0900C0CFB0EFE02FB01E16FF016
:104CA0000B0E405880440EFB03807F2840F36A843B
:104CB000A0F17F0393FBF2F002FB10307330414B05
:104CC000C0B2197804F0ACFABBF800202388134472
:104CD000022B23DD384A394B11883868B3F800C0FD
:104CE000DFF8DCE0411A0C2291FBF2F302FB131116
:104CF000902303FB0CF302FB013373445B681844FD
:104D00007F2840F3F1847F3890FBF2F302FB13001D
:104D100073302C4BC0B2197804F082FABBF8002033
:104D200023881344032B23DD234A244B118838683E
:104D3000B3F800C0DFF888E0411A0C2291FBF2F3CF
:104D400002FB1311902303FB0CF302FB01337344AA
:104D50009B6818447F2840F3CF847F3890FBF2F3A0
:104D600002FB13007330174BC0B2197804F058FAE5
:104D7000BBF8002023881344042B7EF7CEA90D4BEB
:104D80001B88012B7EF4C9A93A68A2F10C007F2888
:104D900040F356818B3A0C2092FBF0F300FB13207A
:104DA0007330084BC0B2197804F03AFAFEF7B5B97F
:104DB000A89CFF1F4A9CFF1F1C9EFF1FCC9DFF1F2E
:104DC000601D0100A09CFF1F309CFF1FCF4C23885B
:104DD000002B40F06582DFF868B3CD49CD4A0988E1
:104DE00099F80000B2F800E0DFF85883C1EB000C3E
:104DF0000C229CFBF2F102FB11C14FF0900C0CFB5A
:104E00000EFE02FB01E16FF00B0E58F80110084492
:104E10000EFB03007F2840F37E83A0F17F0393FB0A
:104E2000F2F002FB10307330C0B204F021FABBF88C
:104E3000002023881344022B22DDB54AB54B11888C
:104E400099F80000B3F800C0DFF8F8E2411A0C222C
:104E500091FBF2F302FB1311902303FB0CF302FB13
:104E6000013373445B6818447F2840F341847F38E2
:104E700090FBF2F302FB13007330C0B204F0F8F9B8
:104E8000BBF8002023881344032B22DDA04AA14B4A
:104E9000118899F80000B3F800C0DFF8A8E2411AC1
:104EA0000C2291FBF2F302FB1311902303FB0CF392
:104EB00002FB013373449B6818447F2840F320842D
:104EC0007F3890FBF2F302FB13007330C0B204F0A2
:104ED000CFF9BBF8002023881344042B7DF7C4AF1F
:104EE0008D4B1B88012B7DF4BFAF99F80020A2F1F8
:104EF0000C007F287EF721AF8B3A0C2092FBF0F359
:104F000000FB13207330FEF7D2BDDFF804A299F83E
:104F10000000BAF80030814CC11A0C2291FBF2F368
:104F200002FB131302FB03F3E35818447F287FF7B7
:104F300071AD7F3890FBF2F302FB1300733029E56B
:104F4000774B1A88182A13D03B681344A3F1180032
:104F50007F2840F3C6830C20973B93FBF0F200FBC5
:104F6000123303F173006F4BC0B2197804F058F993
:104F70006D4B6E491A78022A94BF013200221A70D2
:104F80001A7831F81200182810D10424022A02F1EC
:104F90000100C2B288BF002231F81200182804D1E3
:104FA000013CF3D11A70FEF7B8B81A703B6803449D
:104FB000A3F118007F2843DD0C20973B93FBF0F210
:104FC00000FB123303F17300EBE6FBF745FB2EE425
:104FD000534B1B88182B12D099F800201344A3F1CF
:104FE00018007F2840F393830C20973B93FBF0F24B
:104FF00000FB123303F17300C0B204F039F94A4ADE
:105000004A4B127833F81230182B3DF42DAF99F833
:1050100000201344A3F118007F287EF78EAE0C20E9
:10502000973B93FBF0F200FB123303F17300FEF7A2
:105030003EBDFBF711FB65E4FBF70EFBFFF77EBB04
:10504000FBF70AFBADE63A4B1B78002B7DF433AB44
:10505000384B1B78002B3DF42EABB8F800303649A6
:10506000013BA8F800300A70FDF725BB304B1B78D8
:10507000002B7DF477AF2F4B1B78002B3DF41BAB3F
:10508000B8F800302C490133A8F800300A70FDF759
:1050900012BBDFF87CA099F80000BAF80030274C6A
:1050A0003AE71F4A1288182A12D01344A3F11800B5
:1050B0007F2840F3C1820C20973B93FBF0F200FB6A
:1050C000123303F17300C0B298F8001004F0A8F88E
:1050D000154B16491A78022A94BF013200221A7021
:1050E0001A7831F8120018282FD10424022A02F16C
:1050F0000100C2B288BF002231F81200182823D163
:10510000013CF3D11A703B68FEF7FEB8A89CFF1F64
:105110001C9EFF1FCC9DFF1F4A9CFF1F40250100C6
:10512000389CFF1FA09CFF1F8C89FF1F389EFF1F0C
:10513000B39EFF1FB49EFF1F1C9CFF1FE8230100AE
:10514000309CFF1F601D01001A703B680344A3F1EF
:1051500018007F287EF712AE0C20973B93FBF0F2ED
:1051600000FB123303F17300FEF7ABBDDFF82CB385
:10517000E2E4BE4B1A88182A13D03B681344A3F10B
:1051800018007F2840F37A820C20973B93FBF0F2C3
:1051900000FB123303F17300B54BC0B2197804F071
:1051A0003FF8B44BB4491A78022A94BF0132002266
:1051B0001A701A7831F8120018287FF4F7AE042418
:1051C000022A02F1010294BFD2B2002231F8120089
:1051D00018287FF4EAAE013CF2D11A70FDF79DBFAA
:1051E000A24B1B88182B12D099F800201344A3F16E
:1051F00018007F2840F372820C20973B93FBF0F25B
:1052000000FB123303F17300C0B204F031F8994A85
:10521000994B127833F81230182B7FF4F8AEFDF763
:1052200023BE924A1288182A12D01344A3F1180000
:105230007F2840F369820C20973B93FBF0F200FB40
:10524000123303F17300C0B298F8001003F0E8FFC6
:10525000884B89491A78022A94BF013200221A70B9
:105260001A7831F8120018287FF46FAF0424022A4C
:1052700002F1010294BFD2B2002231F812001828C4
:105280007FF462AF013CF2D13CE77C4ADFF80CB21C
:105290001288BBF80010033291427FF715ADE9E4A4
:1052A000764ADFF8F8B11288BBF800100332914259
:1052B0007FF7BDAD91E5724C2388002B40F0E4816F
:1052C000DFF8D8B16F4999F800006F4A098817884C
:1052D000DFF8B8E1411A0C2291FBF2FC02FB1C1131
:1052E0004FF0900C0CFB07F702FB01716FF00B07FE
:1052F0005EF80110014407FB03107F2840F3C181D1
:105300007F3890FBF2F302FB13007330C0B203F05E
:10531000AFFFBBF8002023881344022B21DD594B3B
:10532000594A99F800001B88B2F800E0574FC31A99
:105330000C2193FBF1F201FB1232902303FB0EF3DD
:1053400001FB02333B445B6818447F2840F3F8813B
:105350007F3890FBF1F301FB13007330C0B203F010
:1053600087FFBBF8002023881344032B21DD454B26
:10537000454A99F800001B88B2F800E0434FC31A71
:105380000C2193FBF1F201FB1232902303FB0EF38D
:1053900001FB02333B449B6818447F2840F3C181E2
:1053A0007F3890FBF1F301FB13007330C0B203F0C0
:1053B0005FFFBBF8002023881344042B7EF79DA9D0
:1053C0002E4B1B88012B7EF498A999F80020A2F19E
:1053D0000C007F287FF7C7A88B3A0C2092FBF0F3D4
:1053E00000FB13207330FFF7B0B8294B00227F2158
:1053F00007201A8003F0ECFE7F210B2003F0E8FE6B
:10540000FDF7E3BD234B01227F2107201A8003F023
:10541000DFFE7F210B2003F0DBFEFDF7CEBD1E4B30
:1054200004227F2107201A8003F0D2FE00210B20E6
:1054300003F0CEFEFDF7BABD174B02227F210720F5
:105440001A8003F0C5FE7F210B2003F0C1FEFDF79B
:10545000A8BD114B002107201C8003F0B9FE7F215D
:105460000B2003F0B5FEFDF797BD00BF429CFF1F68
:10547000A09CFF1F8C89FF1FAC9DFF1F4A9CFF1F34
:10548000A89CFF1F1C9EFF1FCC9DFF1F601D0100DD
:105490001A9CFF1FBA9CFF1F129EFF1F309CFF1F0C
:1054A000AF4B1A88182A13D03B681344A3F1180095
:1054B0007F2840F33F810C20973B93FBF0F200FBE9
:1054C000123303F17300A74BC0B2197803F0A8FEA2
:1054D000A54BA6491A78022A94BF013200221A70FD
:1054E0001A7831F8120018287FF460AD0424022ADB
:1054F00002F1010294BFD2B2002231F81200182842
:105500007FF453AD013CF2D11A70FDF706BEFBF7F4
:10551000A3F8FFF734BBFBF79FF885E4904A1288A5
:10552000182A12D01344A3F118007F2840F3F68004
:105530000C20973B93FBF0F200FB123303F1730056
:10554000C0B298F8001003F06BFE874B87491A78B9
:10555000022A94BF013200221A701A7831F8120020
:1055600018287FF4F2AD0424022A02F1010294BF4C
:10557000D2B2002231F8120018287FF4E5AD013CC8
:10558000F2D1BFE5FBF768F8FFF799BB744B1B88B6
:10559000182B12D099F800201344A3F118007F288B
:1055A00040F3C5800C20973B93FBF0F200FB1233D5
:1055B00003F17300C0B203F05BFE6B4A6B4B1278D1
:1055C00033F81230182B7FF422ADFDF74DBC684B39
:1055D0001B88182B12D099F800201344A3F118004F
:1055E0007F2840F3B0800C20973B93FBF0F200FB48
:1055F000123303F17300C0B203F03AFE5A4A5D4B16
:10560000127833F81230182B3EF477A899F800205E
:105610001344A3F118007F287EF7A5AF0C20973B19
:1056200093FBF0F200FB123303F17300FEF78DBF22
:10563000FBF712F8FFF7F7BAFBF70EF843E5484B14
:105640001B88182B11D099F800201344A3F11800DF
:105650007F2872DD0C20973B93FBF0F200FB1233A6
:1056600003F17300C0B203F003FE3F4A3F4B1278D0
:1056700033F81230182BC9D1FEF73FB8FAF7ECFF18
:105680008AE5FAF7E9FF41E63B4ADFF800B1128804
:10569000BBF80010033291427FF73BAE12E6374B66
:1056A0001B88182B11D099F800201344A3F118007F
:1056B0007F2839DD0C20973B93FBF0F200FB12337F
:1056C00003F17300C0B203F0D3FD274A2C4B1278CC
:1056D00033F81230182B99D1FEF70FB8FAF7BCFF48
:1056E00092E5FAF7B9FF3EE4FAF7B6FFFFF711BB10
:1056F000FAF7B2FFFFF7C1BBFAF7AEFFFFF733BB14
:10570000FAF7AAFFFFF7E2BBFAF7A6FF9BE5FAF765
:10571000A3FF71E4FAF7A0FFFFF75BBAFAF79CFF6B
:105720000EE7FAF799FF41E6FAF796FFCAE7FAF7AC
:1057300093FF3FE7FAF790FFC5E6FAF78DFF91E791
:10574000FAF78AFF0AE6FAF787FF54E70D4B03934F
:105750000D4B0293FDF7A4BE23601946FDF7D8BB9D
:10576000449CFF1FA09CFF1F8C89FF1FB49DFF1F3F
:10577000389CFF1F389EFF1F4A9CFF1F429CFF1F43
:10578000AC9DFF1FFD9BFF1FC69CFF1F309CFF1F92
:1057900038B507F01DFD0B4805F054FC00234FF011
:1057A0007E5201210848FAF761FE084B084A094970
:1057B000802400251C7118461D60BDE838400BF0A0
:1057C000C9B900BFB89CFF1FF09DFF1F7C9EFF1F43
:1057D0001C89FF1FFD05000010B50446A420636866
:1057E000198803F079FEE368A6201988BDE8104007
:1057F00003F072BE43682A20198803F06DBE00BF13
:1058000010B5044622206368198803F065FEE3683A
:1058100024201988BDE8104003F05EBE10B5044690
:105820000A206368198803F057FEE3680C20198882
:10583000BDE8104003F050BE10B504460620636872
:10584000198803F049FEE36808201988BDE8104074
:1058500003F042BE10B5044602206368198803F0C5
:105860003BFEE36804201988BDE8104003F034BE15
:1058700070B50E4C84B01225042201230646039015
:10588000029320468DE824001423102106F0DEFD4B
:1058900006220923029303960195204600921423C1
:1058A000102106F0D3FD04B070BD00BFE49EFF1FC1
:1058B00070B5AE4CB4F90030032B00F0E880002B3B
:1058C0004DD0022B6CD0052B00F09880012B00F0FE
:1058D000C080042B00D070BD00244FF4AF75E1B23E
:1058E000A34805F017FC01348542A8BF05460C2CDF
:1058F000F5D1012008F014FB0446002008F010FB4D
:10590000323CA0F132039B496FF4957000FB03F326
:1059100000FB04F081FB034281FB0041DB17C01751
:10592000C3EB6223C0EB612003F5AF7200F5AF73E8
:105930009342A8BF13469D42A8BF1D46A5F114017E
:10594000312900F3E28040F26C7332218A488B4A9D
:105950000180BDE870402A20136003F0BDBD0E2019
:1059600007F09AFB40F6FF71C8308842A8BF08468E
:1059700020EAE07000F5FA6283B28A42804D814EDF
:10598000A8BF0A460220194633802A8003F0A4FDEE
:105990002988042003F0A0FDB4F90030022B92D135
:1059A000172008F0BDFA0546162008F0B9FAA842FB
:1059B000B8BF284600F1C801B1F5FA7FC0F2BF8038
:1059C000B1F57A6FA8BF4FF47A6101F54873B3F56A
:1059D0007A6FA8BF4FF47A639BB289B26A4A6B4D63
:1059E00011800A202B8003F077FD29880C2003F01A
:1059F00073FDB4F90030052B7FF468AF0F2008F079
:105A00008FFAC0F53F630433B3F5AF6FC0F28F80F8
:105A1000B3F5FA6FA8BF4FF4FA6399B25C4BC0F5C7
:105A20004360B0F5AF6F19807EDBB0F5FA6FA8BFA9
:105A30004FF4FA6083B2574DA4202B8003F04CFD45
:105A40002988A62003F048FDB4F90030012B7FF42B
:105A500040AF0B2008F03CF800283CD0112008F0A3
:105A60005FFA00F1C801B1F52F7F3CDB41F25C2306
:105A7000994278DC484A00F5487089B2B0F52F7F2A
:105A800011806DDB8342A8BF03469BB231E010203A
:105A900008F046FAC830B0F5FA7F4BDBB0F57A6F04
:105AA0000146A8BF4FF47A6101F51673B3F57A6F1A
:105AB000A8BF4FF47A639BB289B2384A384D11803F
:105AC00022202B8003F008FD2988242003F004FD08
:105AD000B4F90030F3E6152007F0DEFA00F5967110
:105AE000B1F52F7F30DA40F214534FF42F712A4A68
:105AF00011802C4D06202B8003F0EEFC2988082015
:105B000003F0EAFCB4F90030E3E640F23A72A5F59E
:105B1000B975254B02FB05F583FB0523ED17A5EBB6
:105B2000631389B2323311E74FF4AF6383E74FF465
:105B3000AF6173E740F24C434FF4FA71BDE740F2B6
:105B400014534FF4FA7149E741F25C2399420ADC9D
:105B5000114A00F5617089B2B0F52F7F118091DA9A
:105B60004FF42F73C5E71946C1E700BFC09EFF1F62
:105B7000B89CFF1F67BBCF46849EFF1F9889FF1FFD
:105B80008C9EFF1FC49CFF1F289EFF1F409CFF1F71
:105B9000C89CFF1F489EFF1F7E9CFF1FD69DFF1FB6
:105BA000D29DFF1F5C9EFF1FB5814E1B2DE9F0416A
:105BB000224D82B0012602B284B20092284601969C
:105BC0007823192106F088FB04F10C0212B28DE84B
:105BD00044002846A7197823192104F1020806F089
:105BE0007BFB3FB20FFA88F819233A46284619463C
:105BF0000196CDF8008006F06FFB78233A462846E0
:105C00001946CDF80080019604F10A070B3406F01E
:105C100063FB3FB224B278233A46284619468DE802
:105C2000500006F059FB192300943A460196284685
:105C3000194606F051FB02B0BDE8F081E49EFF1F5B
:105C400030B583B000230C4605B2009326225B23B7
:105C50001C210C4806F090F8294601232622094809
:105C600005F09AFB002C24B205DB214601232622F5
:105C7000044805F091FB044A044B15801C8003B0D6
:105C800030BD00BFE49EFF1FAE89FF1FB089FF1F1C
:105C900070B5A54C237882B01BB1A44B4FF6FF72B0
:105CA0001A80A34BB3F90030C3B9A24A9F4B1068C6
:105CB000B3F9002080F30C005B2303FB00F000131A
:105CC0001C3082424AD04FF0FF31FFF7B9FF9A48AB
:105CD00006F0B6F80023237002B070BD012B1BD074
:105CE000022B5AD0032B3FD0042B00F09A80052BB7
:105CF000F0D10F2008F014F9C0F53B600830B0F582
:105D0000AF6F48DBB0F5FA6FA8BF4FF4FA60A0F5AB
:105D1000AF625B23894835E0894B1B78002B70D03C
:105D2000152007F0B9F9874B1860B0F52F7F32DBEB
:105D300041F25C239842A8BF1846A0F52F735B225E
:105D4000814802FB03F380FB0320DB17C3EBA02099
:105D50001C30764BB3F900308342B4D17B4BB3F99E
:105D600000300133AFD1B5E7794B1B68B3F5FA7F4B
:105D700011DBB3F57A6FA8BF4FF47A637548A3F5CA
:105D8000FA725B2303FB02F380FB0320DB17C3EBF8
:105D900020201C30DDE71C20DBE76F4B1B68B3F5D0
:105DA000FA7F36DBB3F57A6FA8BF4FF47A63A3F5B9
:105DB000FA7268485B2303FB02F380FB0320DB17C6
:105DC000C3EB20201C30654B1B68B3F5FA7F1EDB4C
:105DD000B3F57A6FA8BF4FF47A63A3F5FA725D4901
:105DE0005B2303FB02F381FB0321DB17C3EB2121C0
:105DF0001C314E4BB3F9003083420CD0FFF720FF2B
:105E000065E7112008F08CF84E4B18608DE71C21D7
:105E1000EFE71C20D7E74D4BB3F900308B42EDD1B3
:105E200058E7272200258DE8240076231C214248CC
:105E30004B4E06F051FA16E0B0F5AF7FA8BF4FF415
:105E4000AF70323803FB00F386FB0321DB17C3EB93
:105E500061111C3109B201231D442722364805F087
:105E60009BFA0C2D09D0E9B23E4805F053F93128D0
:105E70004FF05B03E0DC1C21EDE7012008F050F857
:105E80006FF495733238384A03FB00F082FB00232D
:105E9000C017C0EB632303F5AF73312B42DDB3F5BD
:105EA000AF7FA8BF4FF4AF735B22323B2C4D02FB98
:105EB00003F385FB0325DB17C3EB65151C350020B9
:105EC00008F02EF86FF495733238274A03FB00F080
:105ED00082FB0023C017C0EB632303F5AF73312BA4
:105EE0001EDDB3F5AF7FA8BF4FF4AF735B22323B2B
:105EF0001B4902FB03F381FB0321DB17C3EB611199
:105F00001C310A4BB3F90030AB4201D0284675E78B
:105F10000E4BB3F900308B423FF4D9AE28466DE703
:105F20001C21EEE71C25CAE7BA9EFF1FAE89FF1FA2
:105F3000C09EFF1F2C9EFF1FE49EFF1F37800B6D2E
:105F4000429EFF1F089CFF1FD3058541B089FF1F9C
:105F5000509CFF1F011FB812609CFF1F249CFF1F55
:105F60004B48371BB89CFF1F67BBCF462DE9F0415C
:105F7000044682B071482768E56805F055FE112097
:105F8000FFF714FE012619234FF028081946242292
:105F90006A480196CDF8008006F09EF978231946EC
:105FA000242266480196CDF8008006F095F9314626
:105FB000624806F027FD02221921604806F01EFD06
:105FC00038460BF09DFB394602465C4806F0B0FEB1
:105FD0005A4806F0C3FE14220021584806F00EFD70
:105FE00003225749554806F0A3FE544806F0B6FE72
:105FF00023220021514806F001FD032251494F4858
:1060000006F096FE4D4806F0A9FE7DB12F20FFF761
:10601000CDFD32220021494806F0F0FC03224A4916
:10602000464806F085FE454806F098FE0123474A9B
:1060300018461370FFF71CFC2189638962685B1A9C
:106040005C2B128854DD521A02EB4202C2EB421260
:10605000013392FBF3F31B333D4A3848138001268A
:106060001A221BB28DE844001946142206F034F9B6
:10607000002D4FD0218A638AE2685B1A5C2B12885C
:106080003EDC511A5C2202FB01F292FBF3F31B335C
:10609000304A2A48138001251BB2382219468DE860
:1060A0002400322206F018F94023002209218DE84D
:1060B00006002248194606F0DDF829461F4806F07A
:1060C000A1FC022244211D4806F098FC63681B488D
:1060D000198806F093FE2A461F49184806F028FE44
:1060E000E3681648198802B0BDE8F04106F086BEA4
:1060F000511A5C2202FB01F292FBF3F31B33ABE774
:10610000521A02EB4202C2EB4212334492FBF3F307
:106110001B33BDE7402309212A460091074801951A
:10612000194606F0A7F83146044806F06BFC022237
:106130006821024806F062FC6368D2E7E49EFF1F14
:10614000182601001C26010020260100619FFF1F68
:10615000BC9EFF1FBE9EFF1F242601002DE9F047B5
:106160001F4682B01446002A4ED0052A0646D0F8B3
:106170000C8000F0AB800B9B894A00EBC305012C1F
:10618000B5F80AE029896868C1EB0E0382FB03C2F7
:106190001A444FEAE373C3EBA213028851D0042CD4
:1061A00000F08D800022402309218DE806007D4803
:1061B000194606F05FF801217A4806F023FC022216
:1061C000B8F1000F00F0E1804421764806F016FC9B
:1061D00073687448198806F011FE734971480122EA
:1061E00006F0A6FDF3686F48198806F007FE6F4BAE
:1061F000022CB3F9001000F0A680082C00F0C28039
:10620000012002B0BDE8F087694E6A4A336812681F
:10621000CB1A93420D4655D9674A3B88117861489D
:10622000012918BF012414700A9A06321BB212B257
:106230008DE814001946BDF9282006F04DF83560A8
:10624000DEE79BB2D31A994203DC9E457146A8BF94
:1062500019460A9A0180B7F90030BDF928A05148C3
:1062600002F106094FF0000E0FFA89F9194652465D
:10627000CDF80090CDF804E006F02EF829896A895F
:106280006868521A03885C2AA3EB010373DD03EBF1
:1062900043030132C3EB431393FBF2F303F11B02FD
:1062A00013B201203A80194652460190CDF8009071
:1062B0003C4806F011F8404B00221A7072E712FABF
:1062C00083F3C0E7204602B0BDE8F08707254FF012
:1062D00000095A2323228DE820021A21314805F0B3
:1062E000C9FF01212F4806F08DFB01212D4806F042
:1062F0008FFB232235212B4806F080FB2A462F49AD
:10630000284806F015FD274806F028FD254805F029
:1063100097FD4FF4FA6007F011FCFFF7C9FA5A2312
:1063200023221A218DE820021E4805F0A3FF1D48F4
:1063300005F086FD3046FFF719FE214B01221A7049
:10634000FFF7A6FC2EE74A1C12B21A8091423FF4D6
:1063500057AF0A9AB7F9003012480632012412B238
:10636000009219460194BDF9282005F0B5FF20469A
:1063700002B0BDE8F0875C2101FB03F393FBF2F26E
:106380001B328DE700221A80E0E76821054806F0FD
:1063900035FB73680348198806F030FD27E700BF16
:1063A000C94216B2E49EFF1F24260100C49EFF1FAF
:1063B0004C9FFF1FB8350100619FFF1F2826010079
:1063C000BA9EFF1F2DE9F04F5A4E5B4DB6F9007093
:1063D0004C7855F8277085B08146984604B10C7802
:1063E000DFF874A11AB99AF80030002B39D0534D58
:1063F000002338462B808AF80030FFF7B7FD504A5B
:10640000504BB5F90000012111704FF6FF721A8050
:1064100060B301285ED00120322322460190009310
:106420004946494B3846FFF799FE00240346B5F923
:106430000020022A39DD00222A80B6F900203D49D9
:10644000002A3BDB052AC4BF00220A80B8F1000FF6
:1064500039D1002C0CBF18464FF0FF3005B0BDE815
:10646000F08F364DB5F900000028D2D1DFF8ECB03E
:10647000364ADBF800301268C3EB0903934227D990
:10648000334B1A78012A18BF01201870FFF7F0F972
:106490000123CBF80090012C2AD0042C35D0022CFB
:1064A0003AD0082C3ED00024C1E7C6D1FA68002AB1
:1064B000C1D0B6F900201F49002AC3DA05220A809C
:1064C000B8F1000FC5D00393FFF7E2FB039BC0E7D1
:1064D0000346E0E74FF0000E142322468DE8084003
:1064E00049461C4B38467446FFF738FE03469EE784
:1064F00032888AF80040013232807A6982B1002401
:10650000384603939047039B91E732880121013A73
:1065100032808AF80010F0E701222A8000248CE7FC
:10652000144684E77A69002129804FF0FF34002A5D
:10653000E6D182E7C09EFF1FB489FF1FC49EFF1FE4
:10654000BA9EFF1FAE89FF1FBE9EFF1FB835010018
:10655000619FFF1FBC9EFF1FC29EFF1F4C9FFF1F1E
:1065600001210D2007F0AEBA00210D2007F0AABAD4
:1065700001460D2007F0A6BA08B50D2007F0A8FACD
:10658000B0FA80F149090D20BDE8084007F09ABA39
:1065900010B5002144080D2007F094FA204607F0BA
:1065A000CDFA0D20012107F08DFA2046BDE81040FC
:1065B00007F0C4BA214A224B10881B68984210B5D4
:1065C00035DA204A1288141A9A42A8BF1A46B4F53E
:1065D000157F22DA121A40F2532303FB02F393FBD6
:1065E000F4F105310A2007F0DDF8174B197801B3F3
:1065F000164B17491B6840F2271283F3070302FB6F
:1066000003F381FB03211944DB17C3EBA11105310F
:106610000920BDE8104007F0C5B8131A4FF41572F1
:10662000611C02FB03F393FBF1F10531DAE7002172
:10663000D8E70920BDE8104007F0B4B8C49CFF1F9C
:10664000009CFF1F8C9EFF1F809CFF1F749EFF1FDE
:10665000090402817F2838B5A8BF7F200F4C4FF472
:10666000167202FB00F284FB02311144D217054678
:10667000C2EBA1110A2007F095F87F3D4FF4967305
:1066800003FB05F384FB03211944DB17A3EBA111E2
:106690000920BDE8384007F085B800BF0904028131
:1066A000C368B3F9003030B583EAE374A4EBE37454
:1066B000002BA0B218DB012300E0134603EB83029A
:1066C00052009442F9DA0A4D90FBF3F285FB03E4A1
:1066D00003FB1200DB173032D3EBA40380B201F8C6
:1066E000012BF1D10B7030BD2D230B700131E2E78E
:1066F0006766666638B5094D8224204602F006FFBB
:1067000035F8021B00B28842204601D002F0E4FEB8
:106710000234A4B28A2CF0D138BD00BFB49DFF1F53
:10672000024B8020198802F0D7BE00BF449CFF1F97
:1067300038B5094D7824204602F0E8FE35F8021BF2
:1067400000B28842204601D002F0C6FE0234A4B254
:10675000802CF0D138BD00BFAC9DFF1F024B7620CE
:10676000198802F0B9BE00BF429CFF1F38B5094D21
:106770004624204602F0CAFE35F8021B00B28842C9
:10678000204601D002F0A8FE0234A4B24E2CF0D173
:1067900038BD00BF389EFF1F024B4420198802F00D
:1067A0009BBE00BF389CFF1F024B4E20198802F091
:1067B00093BE00BF5C9CFF1F024B9A20198802F019
:1067C0008BBE00BFA89CFF1F024B9820198802F0C7
:1067D00083BE00BF4A9CFF1F024B8C20198802F029
:1067E0007BBE00BFCC9DFF1F024B9C20198802F08E
:1067F00073BE00BF309CFF1F024BA020198802F01F
:106800006BBE00BF409EFF1F024B9620198802F00E
:1068100063BE00BF1C9EFF1F024B8A20198802F036
:106820005BBE00BFDE9DFF1F08B5034B102019881B
:1068300002F052FE012008BDDC9DFF1F024B10201C
:10684000198802F049BE00BFDC9DFF1F024B2C20BF
:10685000198802F041BE00BF2E9CFF1F024B1E2074
:10686000198802F039BE00BF489CFF1FC3680E2084
:10687000198802F031BE00BF024B2820198802F0AF
:106880002BBE00BF369EFF1F024B6220198802F00C
:1068900023BE00BF6C9CFF1F024B6420198802F0CE
:1068A0001BBE00BF309EFF1F024B5A20198802F00A
:1068B00013BE00BF109CFF1F024B1620198802F068
:1068C0000BBE00BF1A9CFF1F024B2E20198802F03E
:1068D00003BE00BFB09CFF1F024B3020198802F09E
:1068E000FBBD00BF989EFF1F024B9E20198802F03F
:1068F000F3BD00BF9489FF1F024BAC20198802F042
:10690000EBBD00BF329EFF1F024BAE20198802F084
:10691000E3BD00BF549CFF1F024BB020198802F05A
:10692000DBBD00BFC09DFF1F024BB220198802F0E3
:10693000D3BD00BF769CFF1F024B1820198802F0C0
:10694000CBBD00BFCA9CFF1F024BA220198802F0DA
:10695000C3BD00BF629EFF1F024B1A20198802F0C0
:10696000BBBD00BF649CFF1F024B1C20198802F0B6
:10697000B3BD00BF5E9CFF1F024B6620198802F06A
:10698000ABBD00BF709EFF1F024B7220198802F042
:10699000A3BD00BF949EFF1F024B2020198802F068
:1069A0009BBD00BF6E9EFF1F024B3220198802F074
:1069B00093BD00BF5E9EFF1F024B6820198802F046
:1069C0008BBD00BF9C9CFF1F024B6C20198802F0FE
:1069D00083BD00BF049CFF1F024B5220198802F0A8
:1069E0007BBD00BF2E89FF1F024B5020198802F08B
:1069F00073BD00BF2089FF1F024B5420198802F08D
:106A00006BBD00BFA889FF1F024B5C20198802F0F4
:106A100063BD00BFAC89FF1F024B5E20198802F0E6
:106A20005BBD00BF2C89FF1F024B5620198802F066
:106A300053BD00BF9E9CFF1F244B1B880B2B43D8CC
:106A4000DFE803F00B10151A1F24292E33383D06FA
:106A5000084604221E490AF011BF084604221D49B7
:106A60000AF00CBF084604221B490AF007BF08467B
:106A700004221A490AF002BF0846042218490AF003
:106A8000FDBE0846042217490AF0F8BE0846042253
:106A900015490AF0F3BE0846042214490AF0EEBE76
:106AA0000846042212490AF0E9BE084604221149A8
:106AB0000AF0E4BE084604220F490AF0DFBE084689
:106AC00004220E490AF0DABE704700BF1C9EFF1F69
:106AD000542E0100C42B0100302A0100082F0100B0
:106AE000342A0100F02E0100382A01003C2A01005E
:106AF000E82C0100402A0100602E0100442A010018
:106B0000064B074A10B41C88064B0846002C14BFDD
:106B100011461946042210BC0AF0B0BE7C9CFF1F2F
:106B2000482A01004C2A0100064B074A10B41C8871
:106B3000064B0846002C14BF11461946042210BC0F
:106B40000AF09CBEB29CFF1F482A01004C2A01009B
:106B5000064B074A10B41C88064B0846002C14BF8D
:106B600011461946042210BC0AF088BED09DFF1FB2
:106B7000482A01004C2A0100064B074A10B41C8821
:106B8000064B0846002C14BF11461946042210BCBF
:106B90000AF074BEE49DFF1F482A01004C2A010040
:106BA000064B074A10B41C88064B0846002C14BF3D
:106BB00011461946042210BC0AF060BE1E9EFF1F3B
:106BC000482A01004C2A0100064B074A10B41C88D1
:106BD000064B0846002C14BF11461946042210BC6F
:106BE0000AF04CBEBA9CFF1F482A01004C2A010043
:106BF0001B4B1B880A2B0AD8DFE803F00A0E12167B
:106C00001A1E22262A2E0600164B186808607047A6
:106C1000154B186808607047144B18680860704777
:106C2000134B186808607047124B1868086070476B
:106C3000114B186808607047104B1868086070475F
:106C40000F4B1868086070470E4B18680860704753
:106C50000D4B1868086070470C4B18680860704747
:106C6000DE9DFF1F742A01004C2A0100502A0100FA
:106C7000542A0100582A01005C2A0100602A010000
:106C8000642A0100682A01006C2A0100702A0100B0
:106C9000F0B52B4E2B4FDFF8C4E005460FCE87B082
:106CA0006C460FC496E803003B68274A274F44F818
:106CB000040B40F6CC308342C8BF3A46BEF80060B1
:106CC0002180012E11889278ADF80D108DF80F20DB
:106CD0002AD032D340F6CA02022E18BF00229A42AE
:106CE00026DAA3F698031A491A4AC3EB031381FB69
:106CF00003011944DB17C3EB6123243382FB032117
:106D0000DA17C2EBA10202EB8201A3EB410330339D
:106D100030328DF813308DF811206946284616223E
:106D20000AF0ACFD07B0F0BD40F698029A42D8DBFD
:106D3000094B1868CDF81100EFE740F6FC02CEE7EA
:106D4000882A0100249EFF1F7C2A0100782A010066
:106D50003B773B9867666666802A0100BC9DFF1FF3
:106D6000F8B5174C174E2278174D33782F888E467A
:106D7000003218BF012201467046FFF723FB0023B3
:106D800098423370237015DB14BF012000202B883C
:106D90009F420ED040F23A72A3F5AF730B490C4CF0
:106DA00002FB03F381FB0312DB17A3EB6213323305
:106DB0002360F8BD0749012218460A702270E6E7F1
:106DC000A48AFF1FD59EFF1F849EFF1FB5814E1B07
:106DD0009889FF1F609FFF1F014B187802F014BBBA
:106DE000489FFF1F014B187802F028BB9890FF1FA7
:106DF000134BB3F9003030B583EAE374A4EBE374CA
:106E0000002BA0B218DB012300E0134603EB830242
:106E100052009442F9DA0B4D90FBF3F285FB03E448
:106E200003FB1200DB173032D3EBA40380B201F86E
:106E3000012BF1D10B7030BD2D230B700131E2E736
:106E40009890FF1F67666666144BB3F9003070B503
:106E500083EAE375A5EBE375002BACB21ADB0123E3
:106E600000E0034603EB830040008542F9DA0C4E54
:106E700094FBF3F086FB03E503FB1044DB17303093
:106E8000D3EBA503A4B201F8010BF1D105480B70B7
:106E9000106070BD2D230B700131E0E7109CFF1FC7
:106EA00067666666A02A0100134BB3F9003030B55F
:106EB00083EAE374A4EBE374002BA0B218DB012394
:106EC00000E0134603EB830252009442F9DA0B4DC3
:106ED00090FBF3F285FB03E403FB1200DB17303277
:106EE000D3EBA40380B201F8012BF1D10B7030BDBC
:106EF0002D230B700131E2E79489FF1F67666666F8
:106F0000134BB3F9003030B583EAE374A4EBE374B8
:106F1000002BA0B218DB012300E0134603EB830231
:106F200052009442F9DA0B4D90FBF3F285FB03E437
:106F300003FB1200DB173032D3EBA40380B201F85D
:106F4000012BF1D10B7030BD2D230B700131E2E725
:106F5000549CFF1F67666666134BB3F9003030B56B
:106F600083EAE374A4EBE374002BA0B218DB0123E3
:106F700000E0134603EB830252009442F9DA0B4D12
:106F800090FBF3F285FB03E403FB1200DB173032C6
:106F9000D3EBA40380B201F8012BF1D10B7030BD0B
:106FA0002D230B700131E2E7769CFF1F6766666652
:106FB000134BB3F9003030B583EAE374A4EBE37408
:106FC000002BA0B218DB012300E0134603EB830281
:106FD00052009442F9DA0B4D90FBF3F285FB03E487
:106FE00003FB1200DB173032D3EBA40380B201F8AD
:106FF000012BF1D10B7030BD2D230B700131E2E775
:10700000629EFF1F67666666134BB3F9003030B5AA
:1070100083EAE374A4EBE374002BA0B218DB012332
:1070200000E0134603EB830252009442F9DA0B4D61
:1070300090FBF3F285FB03E403FB1200DB17303215
:10704000D3EBA40380B201F8012BF1D10B7030BD5A
:107050002D230B700131E2E72E89FF1F67666666FC
:10706000134BB3F9003030B583EAE374A4EBE37457
:10707000002BA0B218DB012300E0134603EB8302D0
:1070800052009442F9DA0B4D90FBF3F285FB03E4D6
:1070900003FB1200DB173032D3EBA40380B201F8FC
:1070A000012BF1D10B7030BD2D230B700131E2E7C4
:1070B0002089FF1F67666666134BB3F9003030B551
:1070C00083EAE374A4EBE374002BA0B218DB012382
:1070D00000E0134603EB830252009442F9DA0B4DB1
:1070E00090FBF3F285FB03E403FB1200DB17303265
:1070F000D3EBA40380B201F8012BF1D10B7030BDAA
:107100002D230B700131E2E7A889FF1F67666666D1
:10711000134BB3F9003030B583EAE374A4EBE374A6
:10712000002BA0B218DB012300E0134603EB83021F
:1071300052009442F9DA0B4D90FBF3F285FB03E425
:1071400003FB1200DB173032D3EBA40380B201F84B
:10715000012BF1D10B7030BD2D230B700131E2E713
:10716000AC89FF1F67666666134BB3F9003030B514
:1071700083EAE374A4EBE374002BA0B218DB0123D1
:1071800000E0134603EB830252009442F9DA0B4D00
:1071900090FBF3F285FB03E403FB1200DB173032B4
:1071A000D3EBA40380B201F8012BF1D10B7030BDF9
:1071B0002D230B700131E2E72C89FF1F676666669D
:1071C00008B5702002F0A2F9044B1988884204D057
:1071D0007020BDE8084002F07FB908BDBC9DFF1FCC
:1071E00008B5742002F092F9044B1988884204D043
:1071F0007420BDE8084002F06FB908BD549EFF1F1F
:10720000054B1B880846042213B904490AF036BB13
:1072100003490AF033BB00BF5C9CFF1FA82A010092
:10722000A42A01000E4B1B88032B17D8DFE803F0BC
:10723000110C0702084604220A490AF01FBB08463F
:10724000042209490AF01ABB0846042207490AF039
:1072500015BB0846042206490AF010BB704700BF60
:10726000CC9DFF1FB82A0100B42A0100B02A0100FA
:10727000AC2A010010B40A4B0A4C0A4693E80300FA
:1072800083B0238802AC04E9030004EB83031046B7
:1072900053F8081C052203B010BC0AF0EFBA00BF77
:1072A000A8260100309EFF1F30B40A4B0A4D0C4641
:1072B00093E8070084B02B8804AD05E9070005EBCF
:1072C0008303204653F80C1C042204B030BC0AF09F
:1072D000D5BA00BFB0260100BC9DFF1FF0B40C4D15
:1072E0000C4F0E460FCD8CB001AC0FC40FCD0FC4A8
:1072F00095E807003B8884E807000CAA02EB8303AB
:10730000304653F82C1C04220CB0F0BC0AF0B6BA7C
:10731000BC260100129EFF1F30B50A4B0A4D0C46D9
:107320000FCB85B00DF1100E0EE90F002B880EEB80
:107330008303204653F8101C042205B0BDE83040FA
:107340000AF09CBAF8260100329EFF1F30B50A4BA6
:107350000A4D0C460FCB85B00DF1100E0EE90F0053
:107360002B880EEB8303204653F8101C042205B033
:10737000BDE830400AF082BAF8260100C09DFF1F28
:10738000F0B40B4D0B4F0E460FCD86B06C460FC4BC
:1073900095E803003B8884E8030006AA02EB830318
:1073A000304653F8181C042206B0F0BC0AF066BA46
:1073B00008270100CA9CFF1FF0B40A4D0A4F0E4671
:1073C0000FCD86B001AC0FC42A683B88226006AAA4
:1073D00002EB8303304653F8141C0C2206B0F0BCB9
:1073E0000AF04CBA202701005E9CFF1FF0B40B4D41
:1073F0000B4F0E460FCD86B06C460FC495E80300C8
:107400003B8884E8030006AA02EB8303304653F866
:10741000181C042206B0F0BC0AF030BA3427010070
:10742000549EFF1F164B1B880BB31BB283EAE370FD
:10743000A0EBE370002B30B584B21DDB012300E02C
:10744000134603EB830252009042F9DA0D4894FB95
:10745000F3F280FB03E503FB1244DB173032D3EB7E
:10746000A503A4B201F8012BF1D10B7030BD084681
:10747000042205490AF002BA2D230B700131DDE721
:107480009C9CFF1F67666666BC2A010030B40A4BED
:107490000A4D0C4693E8070084B02B8804AD05E93B
:1074A000070005EB8303204653F80C1C042204B0AC
:1074B00030BC0AF0E3B900BF4C270100049CFF1F59
:1074C000054B1B881BB9054B1868086070470846B8
:1074D000042203490AF0D2B9A89CFF1F4C2A0100DC
:1074E000482A0100164B1B880BB31BB230B583EA48
:1074F000E374A4EBE374002BA0B21CDB012300E0D7
:10750000134603EB830252009442F9DA0D4D90FBCF
:10751000F3F285FB03E403FB1200DB173032D3EBFD
:10752000A40380B201F8012BF1D10B7030BD064BE2
:107530001868086070472D230B700131DEE700BF2B
:10754000489CFF1F676666664C2A0100164B1B8825
:107550000BB31BB230B583EAE374A4EBE374002BE6
:10756000A0B21CDB012300E0134603EB83025200B0
:107570009442F9DA0D4D90FBF3F285FB03E403FB33
:107580001200DB173032D3EBA40380B201F8012BD9
:10759000F1D10B7030BD064B1868086070472D2381
:1075A0000B700131DEE700BF229EFF1F6766666633
:1075B0004C2A0100164B1B880BB31BB230B583EA73
:1075C000E374A4EBE374002BA0B21CDB012300E006
:1075D000134603EB830252009442F9DA0D4D90FBFF
:1075E000F3F285FB03E403FB1200DB173032D3EB2D
:1075F000A40380B201F8012BF1D10B7030BD064B12
:107600001868086070472D230B700131DEE700BF5A
:107610001A9CFF1F67666666C02A0100174B1B880D
:107620001BB31BB270B583EAE375A5EBE375002BC2
:10763000ACB21EDB012300E0034603EB83004000F5
:107640008542F9DA0E4E94FBF3F086FB03E503FB6B
:107650001044DB173030D3EBA503A4B201F8010BC3
:10766000F1D108480B70106070BD074B18680860B6
:1076700070472D230B700131DCE700BFB09CFF1F6A
:1076800067666666C42A01004C2A0100164B1B88F7
:107690000BB31BB230B583EAE374A4EBE374002BA5
:1076A000A0B21CDB012300E0134603EB830252006F
:1076B0009442F9DA0D4D90FBF3F285FB03E403FBF2
:1076C0001200DB173032D3EBA40380B201F8012B98
:1076D000F1D10B7030BD064B1868086070472D2340
:1076E0000B700131DEE700BF989EFF1F676666667C
:1076F0004C2A0100164B1B880BB31BB230B583EA32
:10770000E374A4EBE374002BA0B21CDB012300E0C4
:10771000134603EB830252009442F9DA0D4D90FBBD
:10772000F3F285FB03E403FB1200DB173032D3EBEB
:10773000A40380B201F8012BF1D10B7030BD064BD0
:107740001868086070472D230B700131DEE700BF19
:10775000709EFF1F676666664C2A0100164B1B88E9
:107760000BB31BB230B583EAE374A4EBE374002BD4
:10777000A0B21CDB012300E0134603EB830252009E
:107780009442F9DA0D4D90FBF3F285FB03E403FB21
:107790001200DB173032D3EBA40380B201F8012BC7
:1077A000F1D10B7030BD064B1868086070472D236F
:1077B0000B700131DEE700BF949EFF1F67666666AF
:1077C0004C2A0100174B1B881BB31BB270B583EA10
:1077D000E375A5EBE375002BACB21EDB012300E0E3
:1077E000034603EB830040008542F9DA0E4E94FB1A
:1077F000F3F086FB03E503FB1044DB173030D3EBDB
:10780000A503A4B201F8010BF1D108480B70106078
:1078100070BD074B1868086070472D230B7001314D
:10782000DCE700BF6E9EFF1F67666666C42A010024
:107830004C2A0100054B1B881BB1054B18680860DA
:107840007047044B18680860704700BF9E9CFF1F7C
:10785000D82A0100D42A0100184B1A8852B3184ABA
:10786000128830B50A80B3F90030002B83EAE37444
:10787000A4EBE374BCBF2D238B70A0B2ACBF02316C
:107880000331012300E0134603EB830252009442CC
:10789000F9DA0C4D90FBF3F285FB03E403FB1200D5
:1078A000DB173032D3EBA40380B201F8012BF1D106
:1078B0000B7030BD044B186808607047649CFF1F54
:1078C000DC2A0100676666664C2A010070B53C4DF3
:1078D0002B780646002B35D11C4673780BB9204611
:1078E00070BDFAF74BFB374A374B3848127831787E
:1078F0001B78007802EB43034A1E03EB80030E2A39
:10790000EDD801A050F822F07179000093790000C1
:10791000DF78000071790000DF780000DF78000078
:10792000DF7800005F790000DF780000DF7800007A
:10793000DF780000DF780000DF780000DF780000EB
:107940005B790000AE21224803F01EFF204804F0BE
:107950006BF900232B700124BFE706F001FCAF2177
:107960001B4803F011FF1B4A012313702B70B6E76D
:1079700083B91948038804294FF6FF7103F1FF32D8
:107980000CBF01230B46134403F07F030133038034
:107990000FE073B1013B114A32F813304BB10E4E78
:1079A0000F481049104A33800123002606700B70DF
:1079B0001370084A0221012311702B70204670BDFC
:1079C000A48AFF1FB59EFF1FB69EFF1F649EFF1F68
:1079D000E49EFF1F609FFF1F609EFF1F9C9DFF1F77
:1079E000949CFF1F1C9CFF1F639FFF1F10B5064B3D
:1079F000064C1A882046012101F05CFD21884220B6
:107A0000BDE8104001F068BD7C9CFF1F8E9EFF1FEB
:107A100010B5064B064C1A882046022101F04AFD9B
:107A200021884220BDE8104001F056BDB29CFF1FE6
:107A30008E9EFF1F10B5064B064C1A882046042167
:107A400001F038FD21884220BDE8104001F044BD1E
:107A5000D09DFF1F8E9EFF1F10B5064B064C1A8847
:107A60002046062101F026FD21884220BDE8104075
:107A700001F032BDE49DFF1F8E9EFF1F10B5064B27
:107A8000064C1A882046002101F014FD218842206E
:107A9000BDE8104001F020BD1E9EFF1F8E9EFF1FFF
:107AA00008B5122001F032FD054B1988884206D036
:107AB000122001F011FDBDE8084001F025BC08BD11
:107AC000129EFF1F08B5582001F020FD054B1988B4
:107AD000884206D0582001F0FFFCBDE8084001F0C4
:107AE00013BC08BD229EFF1F08B5142001F00EFD37
:107AF000054B1988884206D0142001F0EDFCBDE842
:107B0000084001F001BC08BDBA9CFF1FF0B480EA38
:107B1000E075A5EBE0750028ACB21FDB1DBF2B2381
:107B20000B704E1C0E46012300E0134603EB83024C
:107B300052009542F9DA0B4F94FBF3F287FB0305F1
:107B400003FB1244DB173032D3EBA503A4B206F8D3
:107B5000012BF1D133700846F0BC70472D230B7018
:107B60004E1CE0E767666666174B18880C2813D032
:107B7000192815D01A2817D01B2819D01C281BD05B
:107B80001D281DD01E2803D00C3800B2FFF7BEBF41
:107B90000E4A1068086070470D4A10680860704708
:107BA0000C4A1068086070470B4A106808607047FC
:107BB0000A4A106808607047094A106808607047F0
:107BC000084A1068086070475E9EFF1FFC2A01008B
:107BD000E42A0100E82A0100EC2A0100F02A010051
:107BE000F42A0100F82A0100034B1888A0EB80005A
:107BF000400000B2FFF78ABF489FFF1F024BB3F956
:107C00000000FFF783BF00BF6C9CFF1F024B18886A
:107C1000033800B2FFF77ABF369EFF1F024B188869
:107C20000C3800B2FFF772BF169CFF1F024B18887A
:107C3000183800B2FFF76ABF449CFF1F024B188838
:107C4000183800B2FFF762BF429CFF1F024B188832
:107C5000183800B2FFF75ABF389CFF1FC368188856
:107C6000183800B2FFF752BF054B1B881BB9054BF4
:107C700018680860704708460422034909F0FEBDF1
:107C8000409EFF1F4C2A0100482A0100054B1B881B
:107C90001BB9054B18680860704708460422034961
:107CA00009F0ECBD4A9CFF1F4C2A0100482A010044
:107CB00030B5134C85B001252B463C2202212046CD
:107CC000009503F0D7FD204603F0AEFF00224021CF
:107CD000802320460191009311460A4B029504F03F
:107CE00051FC204604F0ACF807480849084A002334
:107CF000036083800B608B801360938005B030BD80
:107D0000E49EFF1F70310100C89EFF1FDC9EFF1F15
:107D1000509FFF1F10B500EBC00000F10F02D2B260
:107D200093B284B09C1E981C3D2303918DE81900EA
:107D30003921024804F08AFB04B010BDE49EFF1F05
:107D4000014B01221A707047D59EFF1FF0B5734B8F
:107D5000734C744D744F754E85B004228DE80C0041
:107D600002932046724B4022802103F08BFB204679
:107D7000704A7149714C08F0EDFEAF61704FEF61D0
:107D8000704FA7617048714FE761714F876171490A
:107D9000714FC761714F8F61714A724FCF61724FDE
:107DA0009761724B724FD761724F9F61724FDF6163
:107DB000724FB761724D734FF761734FAF61734C80
:107DC000734FEF61734FA7617348744FE761744F4E
:107DD00074498761744FC761744F754A8F61754FDD
:107DE000CF61754F754B9761754FD761754F764E63
:107DF0009F61764FDF61764F764DB761764FF761C1
:107E0000764F774CAF61774FEF61774F7748A76137
:107E1000774FE761774F87617749784FC761784F30
:107E20008F61784A784FCF61784F9761784B794F5F
:107E3000D761794F9F61794E794FDF61794FB76193
:107E4000794D7A4FF7617A4FAF617A4C7A4FEF6193
:107E50007A4FA7617A487B4FE7617B4F87617B4907
:107E60007B4FC7617B4F8F617B4A7C4FCF617C4FDB
:107E700097617C4B7C4FD7617C4F7D4E9F617D4FDE
:107E8000DF617D4F7D4DB7617D4FF7617D4F7E4C4A
:107E9000AF617E4FEF617E4F7E48A7617E4FE76105
:107EA0007E4F7F4987617F4FC7617F4F7F4A8F61D8
:107EB0007F4FCF617F4F804B9761804FD761804F5D
:107EC0009F61804E804FDF61804F814DB761814F50
:107ED000F761814F814CAF61814F82488249EF61E8
:107EE000824F834DA761E561824F834D834CDFF85C
:107EF00030E2834A834B8761C5618C61824E834F38
:107F0000834D844CC1F81CE0834884499761D56156
:107F10009C61D861B16005B0F0BD00BF40420F0068
:107F2000E49EFF1F148AFF1F1D7C0000BC8CFF1FF6
:107F3000E490FF1F1C89FF1FDDB40000F08EFF1FBF
:107F40006D6800000D7C00003C8EFF1F796800000A
:107F5000016B00002C8CFF1FED790000296B0000E5
:107F6000148FFF1F117A0000516B0000388AFF1F29
:107F7000357A0000FD7B000089680000796B000005
:107F80004C8DFF1F597A000075720000988CFF1FFE
:107F900099680000A16B0000288DFF1F7D7A00000A
:107FA000E97B0000048DFF1FD96D0000F16D00001A
:107FB000CC8EFF1FE56D0000A9720000C08BFF1F73
:107FC000C1710000DD720000808FFF1FA17A0000E8
:107FD0004D750000748CFF1FC57A0000496E0000CB
:107FE000808BFF1FA9680000C96B00001090FF1F65
:107FF000E97A0000B5750000508CFF1FB9680000D9
:108000001D760000708DFF1FC96800008D7600008E
:10801000088CFF1FD9680000A96E0000388BFF1F75
:10802000E968000019730000C88FFF1FF96800009D
:10803000016F0000848EFF1F096900004D7300006E
:10804000148BFF1F19690000596F0000CC89FF1FB6
:1080500029690000817300005C8AFF1F39690000F4
:10806000B16F0000E08CFF1F4969000059780000E3
:10807000A88EFF1F59690000B9730000A890FF1F68
:1080800069690000F5760000188EFF1F796900000D
:108090005D770000F08AFF1F89690000ED73000022
:1080A000A48FFF1FE1710000C5770000608EFF1FE5
:1080B00099690000697B0000CC8AFF1FA969000054
:1080C00025740000A88AFF1FB96900008D740000A4
:1080D0007490FF1FC969000009700000E48BFF1F46
:1080E000D9690000808AFF1F5C8BFF1F6170000050
:1080F000E9690000B9700000F96900001171000021
:10810000388FFF1FF089FF1F9C90FF1F69710000CF
:10811000196A000035780000296A0000A98600006D
:10812000096A0000F0B5461C83B00D460127032301
:1081300036B22AB2044631468DE888002348ADB2F3
:1081400004F01AF90C23AA1C12B20093019705231C
:1081500021B21E4804F010F91D4A1E4B12881B68FC
:10816000BA422AD023D3022A10D11B4CA3F6CA0349
:1081700084FB03241C44DB17C3EB24140A2CA8BF84
:108180000A2424EAE474A2B223B202E000231A46CD
:108190001C460D35AA1A01200093019012B23146F7
:1081A00003230A4804F066F8204603B0F0BD0B4CE8
:1081B000A3F6FC0384FB0324DDE7094CA3F6980334
:1081C00084FB0324DB17C3EBA404D7E7E49EFF1F63
:1081D000BC9DFF1F249EFF1F898888881F85EB5147
:1081E000398EE3382DE9F0438FB283B0DFF84C804D
:1081F000BD1D461D2DB204B236B24FF001090AB2C0
:108200002346314640460095CDF8049004F064F8CA
:108210002A463346214640468DE8200204F05CF8A9
:1082200007F10C020095334612B22146CDF80490B6
:10823000404604F051F803B0BDE8F083E49EFF1F10
:108240002DE9F043804685B0002956D10121304800
:1082500004F0D8FB2F4998F8062098F8083011F858
:108260000290994522DA4FEA89064D460C24D8F847
:108270000C3027489B595F6822B2002104F0BEFBF6
:10828000384609F03DFA39460246214804F050FDCF
:108290001F4804F063FD98F8083001350934AB42FB
:1082A000A4B206F1040601DD422CE0D1B9F1000FC1
:1082B00013D109F1060999450CDA3C2301213B222F
:1082C000039102930093019239233F223A211048EF
:1082D00004F0BCF805B0BDE8F0830F2301213B2278
:1082E000039102930093019239230C223A2108480A
:1082F00004F0ACF898F80830DBE700213423009351
:1083000001913F230C22024803F0B4FF9EE700BF17
:10831000E49EFF1FDC9EFF1F10B5104C012120467C
:1083200004F076FB2046012104F06CFB2046342249
:10833000552104F063FB20460222094904F0F8FCB1
:1083400020460522074904F0F3FC204604F006FD10
:108350002046BDE8104003F073BD00BFE49EFF1F40
:10836000482B01004C2B010070B50D46064609F064
:10837000C7F900EB40008400002D36D0284609F0F4
:10838000BFF900EB4000400023185B1003F16001CF
:10839000091A282209B21748C3F1600404F02EFB21
:1083A0000121144804F02EFB284609F0A9F92946BA
:1083B0000246104804F0BCFC0E4804F0CFFC022139
:1083C0000C4804F01FFB21B221220A4804F016FBDE
:1083D000304609F095F931460246064804F0A8FCFB
:1083E0000448BDE8704004F0B9BC6410C4F16004F6
:1083F000E5E700BFE49EFF1F184B70B5B3F90030EE
:1084000083EAE374A4EBE374002B82B0A1B21EDB19
:1084100068466D46012300E0134603EB83025200D9
:108420009442F9DA0E4E91FBF3F286FB03E403FB70
:108430001211DB173032D3EBA40389B205F8012BFC
:10844000F1D119462B70FFF78FFF02B070BD2D23BD
:108450008DF800300DF101056846DBE7DC9DFF1F5C
:108460006766666610B50D4B1B5C51F82340237898
:1084700084B013B1012004B010BD04AA01A942F8D0
:10848000103D2046A3699847A38A9B07F2D401A810
:108490000099FFF769FF012004B010BDC89EFF1FBF
:1084A0002DE9F04F2F4DDFF8CCB0DFF8C4A0DFF896
:1084B000C8900FCD91B003AC0FC40FCD0FC40FCD3A
:1084C0000FC42B6823600025A8462F462E4600E0E7
:1084D0009846BAF8003024495BF823202846112337
:1084E000F8F76AF900EBC00400EB840089FB003464
:1084F0000444C017C0EB6434C4F13C00C6F13C0234
:1085000007F14101012600B208F1410300901BB2BE
:10851000019612B209B2154803F0DEFE08EB06031D
:1085200005F211153C2B2646ADB24746D0D1342278
:108530006B210E4804F062FA00210C4804F062FA44
:108540000B4B1B8810AA02EB830353F8344C2046D4
:1085500009F0D6F802460548214611B0BDE8F04FB3
:1085600004F0E6BB582701003C210100E49EFF1FF8
:108570002E9CFF1FA01F01000900028010B5424C75
:10858000424882B003F050FB2378C3B906213F482C
:1085900004F038FA2378012B37D90A22022B11462E
:1085A0003A486BD004F02AFA39490322374804F0DC
:1085B000BFFB364802B0BDE8104004F0CFBB354BDE
:1085C0001A7801210523002A35D101910093114623
:1085D0002E4803F0D1FE304B1A78002A36D00523FE
:1085E00001220192009300220A21284803F042FE52
:1085F0002A4B1A78002A35D10121052301910093D5
:108600001421224803F0B8FEC0E7254C2388092B2B
:1086100032D9632B8CBF0A211F210A221B4804F088
:10862000EDF92188194804F0E9FB184802B0BDE8CB
:10863000104004F093BB00220191009311461348AF
:1086400003F018FE144B1A78002AC8D10523012123
:10865000019100930A210D4803F08EFE0F4B1A780A
:10866000002AC9D00122052301920093002214217F
:10867000064803F0FFFD89E73021CEE704F0BEF99C
:108680000322084992E700BF639FFF1FE49EFF1F7C
:10869000582B0100B59EFF1FB69EFF1F649EFF1F53
:1086A000609EFF1F542B0100F8B56D4D287840B92E
:1086B0006C4B1B6899425CD36B4A012313702B707F
:1086C000F8BD0C4600266948664F03F0ADFA04F683
:1086D000AC53324665483B6031212E7004F08EF970
:1086E00001216248624D04F093F931465F4804F07D
:1086F00089F905225F495D4804F01AFB5B4804F0E4
:108700002DFB0C221021594804F078F90B225A490C
:10871000564804F00DFB05225849544804F008FB64
:10872000524804F01BFB564B50481C68A4F69803B3
:10873000C3EB031385FB03251D441021DB17202207
:10874000C3EB652504F05AF940F6CC339C4205F1A1
:1087500024054FF022014FF004000BDCFFF7E2FC90
:10876000484B1C88064674B3012C46D0022C41D0DD
:108770000120F8BDFFF736FD092243493B4804F0CC
:10878000D7FA2A221021394804F038F93F4C3748EB
:1087900084FB0534EB17C3EBA404214604F02EFB45
:1087A00001223B49314804F0C3FA04EB8401A5EBF4
:1087B00041012E4804F022FB012236492B4804F0E7
:1087C000B7FA0120F8BD34491022284804F0B0FA65
:1087D000264804F0C3FA2A221021244804F00EF996
:1087E0003146224804F00AFB07222C491F4804F0B6
:1087F0009FFACBE70C222A49E7E70C2229491B48BC
:1088000004F096FA194804F0A9FA2A221021174810
:1088100004F0F4F8314615481C4E04F0EFFA072234
:108820001E49124804F084FA86FB0536EB17C3EBA9
:10883000A60631460D4804F0E1FA224614490B48D9
:1088400004F076FA06EB8601A5EB4101074804F037
:10885000D5FA22460F49054804F06AFA2046F8BDC9
:10886000A48AFF1F449FFF1F609FFF1FE49EFF1FFE
:108870003B773B985C2B0100642B01004C2B0100E3
:10888000249EFF1FBC9DFF1F702B0100676666665C
:1088900058370100D03601007C2B0100902B0100DD
:1088A000A82B0100982B01002DE9F041754C22788E
:1088B000002A05460F4614BF4FF001084FF000088C
:1088C0004ED1714E3368CB1AB3F5FA6F04D86B787A
:1088D000A3B94046BDE8F0816C4B6D486D49DFF8A7
:1088E000D0E11A70012303700988237026208EF8C6
:1088F000002000F0F1FD6B78002BEAD03760F9F72B
:108900003DFB654A654B6649127828781B780978E3
:1089100002EB4303421E03EB81030E2AD9D801A1C7
:1089200051F822F0158A0000E1890000D388000088
:10893000158A0000D3880000D3880000D388000087
:10894000C9890000D38800007B890000D38800001B
:10895000D3880000D3880000D38800007789000006
:10896000AF215048484E02F00FFFFFF707FE0023EB
:1089700037602370ABE705F0F3FB4A4803F054F986
:108980000221484804F03EF80F222321454804F014
:1089900035F805224449434804F0CAF9414804F037
:1089A000DDF91E2223213F4804F028F805223F4923
:1089B0003C4804F0BDF93B4804F0D0F9394803F0D5
:1089C0003FFA00F0ADFC84E7394D2B78012B50D9EC
:1089D000304B2620198800F07FFD00232B7078E7AC
:1089E000002B3FF476AF013B324A32F81330002BB4
:1089F0003FF46FAF274C304825492D4A23804FF074
:108A000001080023037081F8008082F80080FFF7DE
:108A1000B5FD5EE793B1013B264A32F8131019B356
:108A20001C4B254D1A4C224A198000260123262072
:108A30002E702370137000F04FFD15E0154C1E4989
:108A400022880B7004284FF6FF7002F1FF310CBF33
:108A5000012202460A440E4E154D02F07F020132F9
:108A60000121228031702B70FFF788FD4FF0010843
:108A70002FE70649064A012300200870137023706F
:108A8000A6E700BFA48AFF1F5C9FFF1F609FFF1F18
:108A90001C9CFF1F609EFF1FB59EFF1FB69EFF1F01
:108AA000649EFF1FE49EFF1FB82B0100C02B010036
:108AB000639FFF1F9C9DFF1F949CFF1F2DE9F04F9C
:108AC00005468BB00F46AD480121164603F0A0FFC6
:108AD000AA8812F0010440F0B080DFF8CC8298F848
:108AE0000030002B7DD1AB79A54AD15CA1B9DFF86C
:108AF000BCA279781AF8039041B339780139072973
:108B000000F2B780DFE811F0F1005401B5006C010C
:108B1000B500B500B500E9007C78002C00F0CA80F3
:108B20000139EC68387854F82170FC68411EB4F8BB
:108B30000080072900F2A780DFE811F074015901D5
:108B4000A5006C01A500A500A5009F00DFF854A2B8
:108B5000DAF80020B21AB2F5967F75D9894A1078F2
:108B600001281ABF012010701170874A18BF0146F2
:108B7000D05CC0EB0900C0B2FFF7CCF80124CAF802
:108B80000060AB889B0770D57B78002B6DD0F9F720
:108B9000F5F97E4B7E4A7F481B7812783978007849
:108BA000022515FB02330A2903EB800300F04E81F6
:108BB0000C295AD1002B58D003F11900764E774A70
:108BC000013B0021400080B226F8131001231570EC
:108BD00088F8003000F080FC714B032220461A70A8
:108BE0002FE0664803F020F80121644803F00AFFF3
:108BF00062482246214603F001FFAB88580725D47E
:108C00002C68204608F07CFD214602465B4804F0B3
:108C10008FF85A4804F0A2F8092201238DE80C00CD
:108C200000217F23554803F057FB00212846FFF71A
:108C300007FB002388F8003055E7AB68314638461B
:108C400098470BB0BDE8F08F0846FAE72B6804A8F8
:108C5000984704A808F054FD04A90246474804F0C8
:108C600067F8464804F07AF8D6E720460BB0BDE82E
:108C7000F08F00240AF8039083E70021D15438468E
:108C8000FB699847FC68A4F80080002725223C2354
:108C90008DE8840041211822384803F0EBFAE96896
:108CA000A879FFF7DFFB374A3E4B17701E600BB009
:108CB000BDE8F08F3B490A68B21AB2F5967FD4D965
:108CC000304F0E603E78012E00F0B480E9681846FF
:108CD00001233B70FFF7C6FBB3E7304AE979117017
:108CE000012288F800200024C4E72A7A013A4A4584
:108CF000BFDD09F10104E4B2A145BAD0224E16F855
:108D000003B0CBEB0900C0B20021FFF703F82B7AC8
:108D1000052BD9461BD9CBEB0402042A40F3AE80C5
:108D2000A4F1040BBBF1000FC0F2B080063B5B4521
:108D3000A8BF5B465FFA83F9AA791348B15C9942F0
:108D400005D000F8029001212846FFF779FAC9EB17
:108D50000400C0B201210B4EFEF7DCFF00213423DA
:108D6000019100930548317040230B223F21A14619
:108D700003F080FA0124AB797CE700BFE49EFF1F7B
:108D8000509FFF1F619FFF1FDC9EFF1FB59EFF1FAF
:108D9000B69EFF1F649EFF1F9C9DFF1F609FFF1FCD
:108DA000639FFF1F4C9FFF1FA48AFF1FC89EFF1FCA
:108DB0000FFA89F1E868604C50F82160216804914D
:108DC00034785E4904980860002C71D0012C7FF43F
:108DD00050AF5B4A317A88F800401170002449E7AF
:108DE000B9F1000F50D009F1FF34E4B284E7B98A39
:108DF00001F0040189B200293FF440AF3B6A0392BD
:108E00009847039A00283FF43DAFAB79FC680021F6
:108E1000D15438E77B8A43453CD908F101081FFA51
:108E200088F830E73B8A43453BD208F1FF381FFA08
:108E300088F828E725238DE8180042483C703C2339
:108E40001822412103F016FA3046FAE6002B3FF4CF
:108E50000CAF3D4A3D4E1188394A03F11900013BE0
:108E6000400080B226F81310012388F800301570F6
:108E700000F032FB364B20461D70E2E6002A3FF739
:108E800055AF04F1FF3B4DE74C46F3E64FF00009C8
:108E90004B4651E7BB8ADA077FF5F5AEB7F810808D
:108EA000F1E6BB8AD9077FF5EEAEB7F81280EAE6A5
:108EB0002849C85CC0EB090009F1010EC0B20121CC
:108EC0004FF0340B02F803E0FEF724FFB6681D48AC
:108ED000019440230B223F210124CDF800B003F080
:108EE000C9F940230B223F211648CDF800B0019468
:108EF00003F042FA2146134803F084FD304608F09F
:108F0000FFFBA0EB800000F15F0109B20F220D48CA
:108F100003F074FD304608F0F3FB31460246094881
:108F200003F006FF074803F019FFE968A879FFF787
:108F300099FAAB799EE600BFA09FFF1F4C9FFF1FD1
:108F4000609FFF1FE49EFF1F609EFF1F9C9DFF1FF1
:108F5000639FFF1FDC9EFF1F2DE9F047DFF808929B
:108F60006D4B99F800601B68DFF800A282B00036F4
:108F700001934FF0030018BF0126019F9AF800806B
:108F800004F0A6FD0546042004F0A2FD04460520D9
:108F900004F09EFD800040EA4404062004F098FDA1
:108FA0002C4364B25D4944EAC0000A7880F00F03A4
:108FB000DBB29A425A4A3CD01760002259480B70E3
:108FC00003788DF800808DF8012053B3564A12685B
:108FD0004EF66021BA1A8A4219D8022B59D0012BB9
:108FE0005FD0062B48D0032B63D0042B69D0052B10
:108FF00077D0072B7DD0082B00F08380092B68D019
:1090000016B14A4802F01CFF02B0BDE8F087484A9A
:10901000484C00230121237003701360938089F86A
:1090200000103A4669464448FFF748FD3043C6B24F
:10903000E6E71268BA1A1E2A6BD99AF80020934202
:1090400022D0394C3D488AF80030012B276082EA53
:10905000030207609846B1D0042BAFD137480068AF
:10906000381AB0F5C87FA9D9354C2068381A32288B
:10907000A4D927601A46A1E73A4669463148FFF766
:109080001DFD3043C6B2BBE7012B4FF00002E3D118
:10909000E4E73A4669462C48FFF710FD3043C6B274
:1090A000AEE73A4669462948FFF708FD3043C6B2A5
:1090B000A6E73A4669462648FFF700FD3043C6B2A8
:1090C0009EE73A4669462348FFF7F8FC3043C6B2AC
:1090D00096E73A4669462048FFF7F0FC3043C6B2AF
:1090E0008EE73A4669461D48FFF7E8FC3043C6B2B2
:1090F00086E73A4669461A48FFF7E0FC3043C6B2B5
:109100007EE73A4669461748FFF7D8FC3043C6B2B7
:1091100076E7002252E700BFA09FFF1F649FFF1F5A
:10912000D09EFF1F609FFF1F589FFF1FE49EFF1FE1
:10913000509FFF1F629FFF1F84290100689FFF1F30
:10914000D89EFF1FB4290100002901001428010046
:109150001436010004360100042801006C280100C7
:10916000503601009C90FF1FA48AFF1FD49EFF1F52
:1091700028B11028044BA8BF102018607047024B7C
:1091800001201860704700BF6C9FFF1F38B50F4D5E
:109190002B78013B01381B02C4B203F47063200436
:1091A00043F4404343F00C0300F4FE00184305F081
:1091B000F7FD2868013860F03F00C0B204F01EFEE1
:1091C0002046BDE8384004F019BE00BF6C9FFF1F69
:1091D00070B5124D2B78013B1B0203F470630646F9
:1091E00043F430430806320400F0FE4043F00B0322
:1091F000034302F4FE0018430C4605F0D1FD286835
:10920000013860F04F00C0B204F0F8FD304604F0C1
:10921000F5FD2046BDE8704004F0F0BD6C9FFF1FD7
:1092200070B5124D2B78013B1B0203F470630646A8
:1092300043F410430806320400F0FE4043F00903F3
:10924000034302F4FE0018430C4605F0A9FD28680C
:10925000013860F06F00C0B204F0D0FD304604F079
:10926000CDFD2046BDE8704004F0C8BD6C9FFF1FD7
:1092700038B5104D2B78013B1B0203F47063044694
:1092800043F41043000443F0090300F4FE001843C4
:1092900005F086FD2868013860F06F00C0B204F068
:1092A000ADFD204604F0AAFD0020BDE8384004F0E2
:1092B000A5BD00BF6C9FFF1F38B50E4D2B78013B3D
:1092C0001B0203F47063044643F45043000443F06C
:1092D0000D0300F4FE00184305F062FD2868013814
:1092E00060F02F00C0B204F089FD2046BDE8384090
:1092F00004F084BD6C9FFF1F08B5002005F01AFE26
:109300000028FAD108BD00BF08B564210720FFF787
:109310005FFF7F210B20BDE80840FFF759BF00BF6A
:1093200010B500217B20FFF753FF0024E0B2FFF7C8
:109330009FFF0134022004F001FC802CF6D110BD07
:1093400010B504464FF4406004F008FD04F060FDE1
:109350002CB1102C044BA8BF10241C6010BD024B74
:1093600001241C6010BD00BF6C9FFF1F10B5044698
:1093700041F0E00004F042FD04F07F0004F03EFD07
:10938000C4F3C610BDE8104004F038BD38B5134D25
:109390002B78044641F6FF72A0F50050824203F19B
:1093A000FF33A8BF02461B0202F5005203F47063AC
:1093B000100443F4604343F00E0300F4FE00520433
:1093C000184302F0FE42104305F0EAFC2968013917
:1093D0002046C9B2BDE83840FFF7C8BF6C9FFF1FE9
:1093E00038B504460D46F02004F008FD35B125449B
:1093F00014F8010B04F002FDAC42F9D1F720BDE8EE
:10940000384004F0FBBC00BF00B50B4B83B00246F4
:10941000998818680090032AADF8041002D903B0A7
:109420005DF804FB684606218DF80520FFF7D8FF9C
:1094300003B05DF804FB00BF9036010000B50B4B94
:10944000024683B0186899880090131F4C2BADF822
:10945000041002D903B05DF804FB684606218DF8BC
:109460000520FFF7BDFF03B05DF804FB983601004F
:10947000030203F4FE43C0F3C6101843704700BF55
:1094800003784078DB0103F47E5300F07F0018433B
:10949000704700BF82B002AA114642F8040D0020B6
:1094A00012F8013B03F07F03914243EA0020F7D119
:1094B00002B07047003210B403884FF0010404FA80
:1094C00001F418BF012202FA01F123EA04020A435F
:1094D000028010BC704700BF70B5CEB20C46054686
:1094E00003F0BEFE864203D03146284603F0D2FE8A
:1094F0000135284603F0B4FE240A844205D02146F3
:109500002846BDE8704003F0C5BE70BD38B50546BD
:1095100003F0A6FE4FF0000460F30704681C03F09C
:109520009FFE60F30F24A0B238BD00BFF8B504461B
:109530000020FFF7EBFF002C00F077814FF4AF61C4
:109540000220FFF7C9FF04204FF47A61FFF7C4FF40
:109550000B2004F0BDFA002840F02E874FF49661EE
:109560000620FFF7B9FF4FF4FA610820FFF7B4FFB8
:109570004FF4FA610A20FFF7AFFF40F6B8310C2034
:10958000FFF7AAFF4FF42F612220FFF7A5FF40F657
:10959000AC512420FFF7A0FF7D212A20FFF79CFF7C
:1095A0000C210E20FFF798FF01211020FFF794FFF8
:1095B00002211220FFF790FF00211420FFF78CFFFB
:1095C00000211620FFF788FF02211820FFF784FFF3
:1095D00001211A20FFF780FF01211C20FFF77CFFEB
:1095E00004211E20FFF778FF14212020FFF774FFCD
:1095F00001212620FFF770FF03212820FFF76CFFD1
:1096000004212C20FFF768FF14212E20FFF764FFB0
:1096100000213020FFF760FF0C213220FFF75CFFB4
:1096200000213420FFF758FF00213620FFF754FFB8
:1096300000213820FFF750FF00213A20FFF74CFFB0
:1096400000213C20FFF748FF00213E20FFF744FFA8
:1096500000214020FFF740FF00214220FFF73CFFA0
:109660001F214420FFF738FF13214620FFF734FF66
:109670000E214820FFF730FF11214A20FFF72CFF71
:109680000A214C20FFF728FF00214E20FFF724FF7E
:1096900006215020FFF720FF02215220FFF71CFF78
:1096A0000C215420FFF718FF00215620FFF714FF6C
:1096B00000215820FFF710FF01215A20FFF70CFF6F
:1096C00008215C20FFF708FF0A215E20FFF704FF56
:1096D00000216020FFF700FF04216220FFF7FCFE5D
:1096E00001216420FFF7F8FE00216620FFF7F4FE59
:1096F0000B216820FFF7F0FE7F216A20FFF7ECFEC8
:1097000000216C20FFF7E8FE00216E20FFF7E4FE49
:1097100000217020FFF7E0FE00217220FFF7DCFE41
:1097200000217420FFF7D8FE1F217620FFF7D4FE1A
:1097300013217820FFF7D0FE0E217A20FFF7CCFE10
:1097400011217C20FFF7C8FE0A217E20FFF7C4FE0E
:109750001F218020FFF7C0FE13218220FFF7BCFEEF
:109760000E218420FFF7B8FE11218620FFF7B4FEFA
:109770000A218820FFF7B0FE00218A20FFF7ACFE07
:1097800000218C20FFF7A8FE00219620FFF7A4FE01
:1097900000219820FFF7A0FE00219A20FFF79CFEF1
:1097A00005219C20FFF798FE06219E20FFF794FEDE
:1097B0000021A020FFF790FE7F21A220FFF78CFE62
:1097C00040F2A461A420FFF787FE4FF4E161A620D8
:1097D000FFF782FE0021A820FFF77EFE0021AA20CD
:1097E000FFF77AFE0221AC20FFF776FE0121AE20C2
:1097F000FFF772FE0121B020FFF76EFE0B21B220B1
:10980000FFF76AFE2A210020FFF766FE0220FFF71D
:109810007DFEB0F5805F034616D34FF4AF610220A2
:10982000FFF75AFE4FF4AF630EE04FF6FF73984216
:109830003FF484AE2A2840F0CB850220FFF766FE75
:10984000B0F5805F0346E8D2D24A04201380FFF7C8
:109850005DFEB0F5805F034680F06285CE4A06204B
:109860001380FFF753FEA0F52F739BB2B3F57A6F09
:10987000024606D940F628210620FFF72DFE40F6C5
:109880002822C64B08201A80FFF740FEA0F52F7350
:109890009BB2B3F57A6F024606D940F6E441082040
:1098A000FFF71AFE40F6E442BD4B0A201A80FFF78C
:1098B0002DFEA0F5FA739BB240F6AC518B420246E6
:1098C00006D94FF4FA610A20FFF706FE4FF4FA6258
:1098D000B44B0C201A80FFF719FEA0F5FA739BB267
:1098E00040F6AC518B42024606D940F6B8310C2006
:1098F000FFF7F2FD40F6B832AB4B0E201A80FFF7AF
:1099000005FE1828034600F20A84A84A1020138096
:10991000FFF7FCFD431E9BB20F2B024604D9012129
:109920001020FFF7D9FD0122A14B12201A80FFF76A
:10993000EDFD0A28034600F2EC839E4A14201380B2
:10994000FFF7E4FD0128034604D900211420FFF7A6
:10995000C3FD0023984A16201380FFF7D7FD7F2808
:10996000034600F2D083954A18201380FFF7CEFDFE
:109970000528034600F2C183914A1A201380FFF79D
:10998000C5FD0C28034600F2C4848E4A1C201380B7
:10999000FFF7BCFD0428034600F2B4848A4A1E2067
:1099A0001380FFF7B3FD0928034600F2A484874A19
:1099B00020201380FFF7AAFD4628034600F2948476
:1099C000834A22201380FFF7A1FDA0F5FA739BB212
:1099D00040F6AC518B42024606D94FF42F6122204B
:1099E000FFF77AFD4FF42F627A4B24201A80FFF79D
:1099F0008DFDA0F5FA739BB240F6AC54A34202462B
:109A000004D921462420FFF767FD2246724B262009
:109A10001A80FFF77BFD7F28034600F25E846F4AC1
:109A200028201380FFF772FD0628034600F24E84BB
:109A30006B4A2A201380FFF769FDA0F132039BB225
:109A4000B3F5967F024604D97D212A20FFF744FD15
:109A50007D22644B2C201A80FFF758FD0C2803460A
:109A600000F22D84604A2E201380FFF74FFD1E2840
:109A7000034600F21D845D4A30201380FFF746FD47
:109A80000928034600F20D84594A32201380FFF75B
:109A90003DFD1E28034600F2FD83564A3420138004
:109AA000FFF734FD7F28034600F2EE83524C362048
:109AB0002380FFF72BFD7F28034600F2DF83382049
:109AC0006380FFF723FD7F28034600F2D1833A200D
:109AD000A380FFF71BFD7F28034600F2C3833C20D1
:109AE000E380FFF713FD7F28034600F2B5833E2095
:109AF0002381FFF70BFD7F28034600F2A783402058
:109B00006381FFF703FD7F28034600F2998342201B
:109B1000A381FFF7FBFC394D28804420FFF7F6FCBA
:109B20003028034600F28683354A46201380FFF72B
:109B3000EDFC3028034600F27783324C4820238026
:109B4000FFF7E4FC3028034600F268834A20638074
:109B5000FFF7DCFC3028034600F25A834C20A38038
:109B6000FFF7D4FC3028034600F24C834E20E380FC
:109B7000FFF7CCFC0128034604D900214E20FFF753
:109B8000ABFC0023204A50201380FFF7BFFC431E8C
:109B90003CE000BFC49CFF1F8C9EFF1F7E9CFF1FEC
:109BA0005C9EFF1F289EFF1F409CFF1F169CFF1FEF
:109BB000DC9DFF1F129EFF1FBA9CFF1F1A9CFF1FF8
:109BC000CA9CFF1F649CFF1F5E9CFF1F489CFF1FD9
:109BD0006E9EFF1FD69DFF1FD29DFF1F609EFF1F21
:109BE000369EFF1F849EFF1F2E9CFF1FB09CFF1FF1
:109BF000989EFF1F5E9EFF1F9C9DFF1F8E9EFF1F56
:109C0000389CFF1F389EFF1F5C9CFF1F9BB20B2BD5
:109C1000024604D906215020FFF75EFC0622CF4BF6
:109C200052201A80FFF772FC0428034600F2E482F7
:109C3000CB4A54201380FFF769FC431E9BB21D2BB7
:109C4000024604D90C215420FFF746FC0C22C54BD8
:109C500056201A80FFF75AFC0128034604D9002138
:109C60005620FFF739FC0023BF4A58201380FFF726
:109C70004DFC7F28034600F2B982BC4A5A2013806B
:109C8000FFF744FC431E9BB2092B024604D9012175
:109C90005A20FFF721FC0122B54B5C201A80FFF708
:109CA00035FC431E9BB2102B024604D908215C20D0
:109CB000FFF712FC0822AF4B5E201A80FFF726FC4C
:109CC000431E9BB21D2B024604D90A215E20FFF7DA
:109CD00003FC0A22A84B60201A80FFF717FC022819
:109CE000034600F27D82A54A64201380FFF70EFC34
:109CF0000128034604D901216420FFF7EDFB01236D
:109D00009F4A62201380FFF701FCC31E9BB2012B08
:109D1000024604D904216220FFF7DEFB0422994B9E
:109D200066201A80FFF7F2FB7F28034600F252827A
:109D3000954A68201380FFF7E9FB7F28034600F26D
:109D40004382924A6A201380FFF7E0FB7F28034694
:109D500000F234828E4A6C201380FFF7D7FB022872
:109D6000034600F225828B4A6E201380FFF7CEFB5C
:109D70001928034600F21682874A70201380FFF7E5
:109D8000C5FB0228034600F20782844A7220138032
:109D9000FFF7BCFB0628034600F2F881804A7420D6
:109DA0001380FFF7B3FB0528034600F2E9817D4AE3
:109DB0008A201380FFF7AAFB0A28034600F2DA8103
:109DC000794A8C201380FFF7A1FB0428034600F298
:109DD000CB81764A98201380FFF798FB0128034631
:109DE00004D900219820FFF777FB0023704A9A20BE
:109DF0001380FFF78BFB0128034604D900219A202A
:109E0000FFF76AFB00236B4A96201380FFF77EFB67
:109E10000B28034600F2A281674A9C201380FFF7BB
:109E200075FB831E9BB2032B024604D905219C209F
:109E3000FFF752FB0522614B76201A80FFF766FB85
:109E40003028034600F284815D4A78201380FFF7B2
:109E50005DFB3028034600F275815A4C7A2023803E
:109E6000FFF754FB3028034600F266817C206380B4
:109E7000FFF74CFB3028034600F258817E20A38078
:109E8000FFF744FB3028034600F231818020E38055
:109E9000FFF73CFB3028034600F223814A4A822028
:109EA0001380FFF733FB3028034600F21481474C40
:109EB00084202380FFF72AFB3028034600F2058127
:109EC00086206380FFF722FB3028034600F2F780EC
:109ED0008820A380FFF71AFB3028034600F2E980B0
:109EE000A020E380FFF712FB0128034604D90021DC
:109EF000A020FFF7F1FA0023354A9E201380FFF7D8
:109F000005FBC31E9BB20C2B024604D906219E20E2
:109F1000FFF7E2FA06222F4BA2201A80FFF7F6FA8B
:109F2000431E9BB27E2B024604D97F21A220FFF75D
:109F3000D3FA7F22284BA4201A80FFF7E7FAA0F576
:109F4000AF639BB2B3F5167F024647D940F2A461D6
:109F5000A420FFF7C1FA40F2A4623FE02089FF1F6E
:109F60002E89FF1FA889FF1F9E9CFF1F229EFF1F97
:109F7000109CFF1FAC89FF1F2C89FF1FCE9DFF1F68
:109F8000309EFF1F6C9CFF1F709EFF1F9C9CFF1F3D
:109F90004C9CFF1F049CFF1FB89EFF1FBC9DFF1F12
:109FA000949EFF1F549EFF1FDE9DFF1FCC9DFF1F31
:109FB0004A9CFF1FA89CFF1F1C9EFF1F309CFF1F79
:109FC000429CFF1FAC9DFF1F449CFF1FB49DFF1FC1
:109FD000409EFF1F9489FF1F629EFF1FD84BA62043
:109FE0001A80FFF793FAA0F5AF639BB2B3F5167F23
:109FF000024606D94FF4E161A620FFF76DFA4FF44F
:10A00000E162D04BA8201A80FFF780FA06280346A9
:10A0100000F2CC81CC4AAA201380FFF777FA0328FC
:10A02000034600F2BD81C94AAC201380FFF76EFAE7
:10A030000328034600F2AE81C54AB0201380FFF723
:10A0400065FA0328034600F29F81C24AAE201380BE
:10A05000FFF75CFA7F28034600F29081BE4AB220E7
:10A060001380FFF753FA7F2800F263812B88DFF813
:10A0700008E3BA4FBA4ABB4DBB4EBC4CBC4903F0D7
:10A08000010CAEF800C0C3F3400EA7F800E0C3F324
:10A0900080071780C3F3C007B64A2F70C3F30017B9
:10A0A000C3F34015C3F38013378025800B801080E5
:10A0B000F8BD0A218820FFF70FFA0A2310E71121C3
:10A0C0008620FFF709FA112302E70E218420FFF70B
:10A0D00003FA0E23F4E613218220FFF7FDF9132380
:10A0E000E5E61F218020FFF7F7F91F23D6E60A21B6
:10A0F0007E20FFF7F1F90A23C8E602211820FFF7B6
:10A10000EBF9022338E400211620FFF7E5F90023DC
:10A1100029E402211220FFF7DFF902230DE40C21CC
:10A120000E20FFF7D9F90C23FFF7EFBB11217C209C
:10A13000FFF7D2F91123A1E60E217A20FFF7CCF91F
:10A140000E2393E613217820FFF7C6F9132384E644
:10A150001F217620FFF7C0F91F2375E60021962006
:10A16000FFF7BAF9002357E600218C20FFF7B4F976
:10A1700000232EE600218A20FFF7AEF900231FE618
:10A1800000217420FFF7A8F9002310E600217220B7
:10A19000FFF7A2F9002301E600217020FFF79CF9E8
:10A1A0000023F2E500216E20FFF796F90023E3E596
:10A1B00000216C20FFF790F90023D4E57F216A206D
:10A1C000FFF78AF97F23C5E50B216820FFF784F9A3
:10A1D0000B23B6E500216620FFF77EF90023A7E5F3
:10A1E00000216020FFF778F900237CE5002158204A
:10A1F000FFF772F9002340E502215220FFF76CF9C6
:10A20000022315E50A214C20FFF766F90A23ADE485
:10A2100011214A20FFF760F911239FE40E21482005
:10A22000FFF75AF90E2391E413214620FFF754F962
:10A23000132382E41F214420FFF74EF91F2373E408
:10A2400000214020FFF748F9002360E400213E2070
:10A25000FFF742F9002352E400213C20FFF73CF9CC
:10A26000002344E400213A20FFF736F9002336E4C6
:10A2700000213820FFF730F9002328E400213620A0
:10A28000FFF72AF900231AE400213420FFF724F90C
:10A2900000230BE40C213220FFF71EF90C23FFF7FB
:10A2A000FCBB00213020FFF717F90023FFF7ECBBC0
:10A2B00014212E20FFF710F91423FFF7DCBB042133
:10A2C0002C20FFF709F90423FFF7CCBB032128203A
:10A2D000FFF702F90323FFF7ABBB01212620FFF7AD
:10A2E000FBF80123FFF79BBB14212020FFF7F4F8B4
:10A2F0001423FFF765BB04211E20FFF7EDF80423AC
:10A30000FFF755BB01211C20FFF7E6F80123FFF7FB
:10A3100045BB01211A20FFF7DFF80123FFF735BB0A
:10A320004FF47A610420FFF7D7F84FF47A63FFF710
:10A3300095BAB2200B21FFF7CFF80B2096E600BFAD
:10A34000C89CFF1F489EFF1F129CFF1F829CFF1F7F
:10A35000329EFF1FC09DFF1F549CFF1F7C9CFF1F50
:10A36000B29CFF1FC29DFF1FD09DFF1F349EFF1F89
:10A37000E49DFF1F769CFF1F1E9EFF1F0121AE2044
:10A38000FFF7AAF8012369E60121B020FFF7A4F83E
:10A3900001235AE60221AC20FFF79EF802234BE688
:10A3A0000021AA20FFF798F800233CE60021A8200E
:10A3B000FFF792F800232DE640F628210620FFF74C
:10A3C0008BF840F6E4410820FFF786F8FFF7D0B895
:10A3D00017287FF6B3A819287FF622A91B287FF635
:10A3E0003FA91C283FF454A91E287FF659A91F280D
:10A3F0003FF45EA920283FF477A921283FF480A9E3
:10A4000022283FF485A923283FF48EA924283FF46D
:10A41000BFA925283FF4C4A926283FF4C5A92728A9
:10A420003FF4CAA928283FF4D5A929287FF4EAA92E
:10A43000FFF7D8B9F8B5C52006F0C6FB204B214A76
:10A44000054603CB1368C5F803001A0CB420C5F801
:10A4500007102B80AA70FFF70BF82E46002426F871
:10A460000B0FA0B2FFF752F8FFF702F80234B42C3A
:10A4700026F8020FF5D16C1E05F1C0064FF0FF3033
:10A4800014F8013F082758400F4B40F300017A1E93
:10A490000B4012F0FF0783EA5000F5D1B442EFD130
:10A4A000C043FEF7F7FF3A46C5F8C100C52128466C
:10A4B00004F0C4FC2846BDE8F84006F08DBB00BFA0
:10A4C000A4360100A03601002083B8EDF0B50E4B94
:10A4D0000E4C054693E8070085B024682E88AD78B9
:10A4E00001AB83E80700270C184600220B21ADF8CA
:10A4F00004408DF80670ADF80C608DF80E5004F035
:10A500009DFC05B0F0BD00BFB0360100A0360100D3
:10A51000F0B5124B124D1E68124F0FCD87B06C462E
:10A520000FC495E8030044F8040B38683B79CDF874
:10A530000D00320C2A2021808DF802208DF8113078
:10A54000ADF80060FEF794FF0022ADF80B00122179
:10A55000684604F073FC07B0F0BD00BFA0360100F0
:10A56000BC3601004C2B0100002004F0E3BC00BF0E
:10A5700002F02EBE70B5124C82B000254023064674
:10A5800029462046009301958023202201F072FE87
:10A5900020222946204602F031FA2046012102F00D
:10A5A00037FA304607F0ACF831460246204602F052
:10A5B000BFFB204602B0BDE8704001F041BC00BFC7
:10A5C000E49EFF1FF0B5C42983B075D90546441E2B
:10A5D00000F1C0064FF0FF3014F8012F082750405B
:10A5E000404A40F300017B1E0A4013F0FF0782EA55
:10A5F0005000F5D1B442EFD1C043FEF74BFF014606
:10A60000D5F8C1000190019A914202D0B2F17F2F9A
:10A610000BD105F10B00FEF733FFB4280BD0324805
:10A62000FFF7A8FF002003B0F0BD3048FFF7A2FFFE
:10A63000384603B0F0BD05F10D00FEF721FF2A28D2
:10A6400040D1002440F6AC5613E004281AD0062866
:10A6500021D008281FD00A2828D00C2822D1A1F503
:10A66000FA7292B2B24201D8FEF736FF0234B42C2D
:10A670000ED004F10D002844FEF702FF022C014623
:10A68000A0B2E2D1B1F5805FEED30234B42CF0D1A8
:10A69000012003B0F0BDA1F52F7292B2B2F57A6F2E
:10A6A000E4D8E1E7222801D0242811D1A1F5FA72DB
:10A6B00092B2B242DAD8D7E70D48FFF75BFF00202D
:10A6C00003B0F0BD0B48FFF755FF002003B0F0BD0D
:10A6D0002A28C9D1A1F1320292B2B2F5967FC5D82B
:10A6E000C2E700BF2083B8ED00370100EC3601005F
:10A6F000D43601001437010003290CD970B5461C6B
:10A7000082B005460C46304603222A4907F066F817
:10A7100010B102B070BD70470B2C05D90522264937
:10A72000281D07F05BF840B12448FFF723FF2448B9
:10A7300002B0BDE87040FFF7C9BE05F10901032270
:10A7400001A807F09BF801A803221E4907F046F86C
:10A75000D8B103221C4901A807F040F808B301A8AA
:10A7600003221A4907F03AF8B0B91948FFF702FF77
:10A77000A11E89B23046FFF725FF0028C9D0154831
:10A7800002B0BDE87040FFF7F5BE1348FFF7F2FED8
:10A79000FFF750FE1148F3E71148FFF7EBFE1148B1
:10A7A000C6E71148FFF7E6FE02B0BDE87040FFF7CC
:10A7B000AFBE00BFA03601005C2B01002C370100AA
:10A7C00040370100443701006C3701008437010035
:10A7D000883701009C370100483701005C370100D1
:10A7E000B0370100C4370100703701002DE9F04394
:10A7F000174D2B6883B081460F469046F3B1154E36
:10A8000034880A1992B218461146328006F05AFD71
:10A8100028603A464946204402F06CFDB8F1000F2A
:10A8200009D031882868FFF767FF286806F0D4F957
:10A8300000232B60338003B0BDE8F083054E019305
:10A840000846318006F0C0F9019B28601C46E0E70D
:10A85000749FFF1F709FFF1F10B51F4C4FF4FA70BD
:10A86000FBF796FE204601F0DFF900221146204654
:10A8700002F0C4F82046012102F0CAF82046002167
:10A8800002F0C0F80B221549204602F051FA20468A
:10A8900002F064FA0F221249204602F049FA2046DB
:10A8A00002F05CFA0F490722204602F041FA2046E6
:10A8B00002F054FA204601F0C3FA0B4B0B4A1A601F
:10A8C0004FF4FA70FBF764FEFFF722FE0848BDE87C
:10A8D0001040FFF74FBE00BFE49EFF1FC8370100C6
:10A8E000D4370100E43701002CA1FF1FEDA70000C1
:10A8F000EC3701000020704790F8392090F83800BC
:10A90000101A704790F8383090F839209A4205D9DB
:10A910005A1C034480F83820187E70474FF0FF30EF
:10A92000704700BF90F8383090F839209A4286BFBF
:10A930001B18187E4FF0FF30704700BF704700BFF4
:10A9400038B50546B0F85E0090B195F85D30144614
:10A95000C3F1210294420CD805F13B001844224671
:10A9600002F0C8FC95F85D30234485F85D30204640
:10A9700038BD012014462871EEE700BFB0F85E3004
:10A980006BB190F85D30202B07D8C218013380F8E6
:10A990005D30012082F83B107047012303710020D5
:10A9A000704700BF0023426980F8383080F83930A2
:10A9B00080F85C3080F85D3080F85E3080F85F3081
:10A9C00006CA30B40D68046943662A4383660A6088
:10A9D000A370426990F861301649146813441D7AD7
:10A9E0005B7B01EBC5051B026D6803F4E06343F07C
:10A9F00064032B6090F8623013449D7CDB7D01EB97
:10AA0000C5011B02496803F4E06343F064030B6073
:10AA100021685368194205D0036927225A700369D7
:10AA200004229A71036920225A71036980229A7064
:10AA300030BC70472043010043690CCB12681A42B6
:10AA40000CD0094B99420AD9084B9942036994BF2B
:10AA50001A220D225A70036904229A717047036901
:10AA600027225A70F7E700BF7F1A06003F420F0007
:10AA700010B50269D378DBB2D90604463DD5102162
:10AA80005806D17038D503F0040303F0FF02002B01
:10AA900051D03D49626E00230B7084F85D30002A6E
:10AAA0005BD0904794F85D30002B56D02369D022BC
:10AAB0009A70236994F83B201A712369012284F863
:10AAC0005C200222DA7010BD304B84F860009C429A
:10AAD0004AD02F4B9C4252D094F8391013791F2939
:10AAE000DBB207D82848007820B16018013184F81B
:10AAF000391003760223D37010BD5906C3D4917860
:10AB000001F0100101F0FF000029DDD013F0010376
:10AB10001ED194F85C1094F85D00884281BF4B1CF4
:10AB2000091984F85C3091F83B3013712369D02205
:10AB30009A702269DEE7236984F83920C0229A706E
:10AB40002369114A1979012111700222DA7010BDAE
:10AB5000C023937022691379CCE70122002384F883
:10AB60005D2084F83B30A1E7626994F861300949BF
:10AB700013440322187A02F043FD2269ACE76269AC
:10AB800094F861300449F3E7789FFF1FE490FF1FBA
:10AB90005091FF1FF9AB000005AC00000369DB78A2
:10ABA00003F0200373B190F860300133DBB2012B66
:10ABB00080F860301AD9426990F861301344187AED
:10ABC00002F09ABD70B5426903F0FF0590F861305C
:10ABD00013440446187A02F08FFDA36E5BB184F82B
:10ABE000385094F83900BDE87040184790F85F304D
:10ABF000002BE0D0704770BD0148FFF7CFBF00BF0A
:10AC0000E490FF1F0148FFF7C9BF00BF5091FF1F2D
:10AC10002DE9F047374FDFF8E0903B68026982B0DA
:10AC200006460093DDF800800021A025D3789B061E
:10AC30005BD53B680193019BC8EB03030F2BF5D950
:10AC400049B1102BF2D000209070336980229A70A5
:10AC500002B0BDE8F087726996F8613013440521AF
:10AC6000187A02F043FF726996F8613013440121AB
:10AC700093F812A0504602F039FF092400215046F3
:10AC800002F020FF2B46013BFDD10121504602F08E
:10AC900019FF2B46013BFDD1013CEFD1706996F8BD
:10ACA000611001444FF4A0720C7A4B7B09EBC40194
:10ACB0001B02496803F4E06343F064030B6096F8F9
:10ACC00062300344997CDB7D09EBC1011B024968BA
:10ACD00003F4E06343F064030B60013AFDD1326991
:10ACE000D3789B064FF00101A3D4012002B0BDE848
:10ACF000F08700BFA09FFF1F20430100F0B503694C
:10AD00001222DA700269937803F0200385B00446BA
:10AD10000D46002B5ED0B42393703C4922690B682A
:10AD20000093009E05E00B680193019B9B1B042B85
:10AD300042D8D37803F0200303F0FF00002BF2D0B9
:10AD400094F85D30002B31D04FF0000E4FF0020C24
:10AD500004EB0E0393F83B3013710B680393039FCE
:10AD6000206907E09B060DD50B680293029BDB1B55
:10AD7000052B28D8C378DBB203F0020202F0FF06ED
:10AD8000002AEFD080F803C02669F378DBB2DF0633
:10AD900032462DD49F062BD5DB0731D40EF1010EA0
:10ADA00094F85D305FFA8EFE7345D1D800201DBB4C
:10ADB000002384F85E3004E09070236980229A704A
:10ADC000042005B0F0BD86702369802204209A70AB
:10ADD00005B0F0BD03F0FF06FFF71AFF10B904201D
:10ADE00005B0F0BD236984F85F60B0229A7094E7E3
:10ADF0008023B3700420DAE726698023B370D7E795
:10AE0000BEF1000F0CBF02200320F6E7A09FFF1F3A
:10AE10002DE9F04106690025122780F8385080F8A6
:10AE20003950F770D0F810C09CF802E00EF0200EF8
:10AE300088B00446884615461E46BEF1000F49D02C
:10AE4000B4238CF80230784B21691A680092DDF83F
:10AE500000E006E01A6801920198CEEB0000042899
:10AE600030D8C87800F0200000F0FF070028F1D0AB
:10AE70004FEA480242F00102D2B20A711A68029205
:10AE8000DDF808E0206906E01A6803920399CEEB2A
:10AE9000010105292AD8C17801F0020101F0FF075C
:10AEA0000029F1D04FF0020C80F803C02269D1785C
:10AEB00011F0110722D12DBB002E0CBFA02380233F
:10AEC000937003E08F70236980229A70384608B02F
:10AED000BDE8F0810EF0FF07FFF79AFE0028F5D0DD
:10AEE000236984F85F70B0229A70ACE78770236999
:10AEF000802238469A7008B0BDE8F08180239370B4
:10AF00000027E3E7012D75D0A021917021690A790E
:10AF1000BE4667464FF0A80C1A680492049805E0F4
:10AF20001A680592059A121A052A4AD8CA7802F0B8
:10AF3000020202F0FF08002AF2D0CF702169CA781D
:10AF4000D2B212F0100F08465AD1920658D5013DE0
:10AF5000EDB2012D49D0BEF11F0F3BD90A79012D69
:10AF6000DAD11A680692069D05E01A680792079AD8
:10AF7000521B052A46D8C27802F0020202F0FF01F5
:10AF8000002AF2D00223C3702269D378DBB2D9063B
:10AF90003AD49B0634D5B023BEF11F0F93703FD82F
:10AFA000226904EB0E0312791A760EF1010E5FFA94
:10AFB0008EFE16B1236980229A7084F839E07746B4
:10AFC00084E781F80280236980229A70774684F8AA
:10AFD00039E07BE704EB0E0291F8048082F81880D8
:10AFE0000EF1010E5FFA8EFEB9E781F802C0216909
:10AFF0000846B0E7A82191702069BE460279B0E703
:10B00000774663E78170DEE71021A023D170013B12
:10B01000FDD12269937803F0F7037746937055E7E3
:10B0200023691B79C5E700BFA09FFF1F0148FFF7F9
:10B030001FBD00BFE490FF1F0148FFF719BD00BF0F
:10B040005091FF1F704700BF38B5144C03780122A0
:10B050005B000546204684F83B3084F85E2084F887
:10B060005D20FFF78BFC20460021FFF747FE0B4CCD
:10B070002978012320461A46FFF7CAFE0128F6D197
:10B0800094F8383094F839209A4205D9E2180133FF
:10B0900084F83830107E38BDFF2038BDE490FF1FA3
:10B0A00038B51B4C037801225B000546204684F826
:10B0B0003B3084F85E2084F85D20FFF75FFC20467B
:10B0C0000021FFF71BFE124C2978204601230222A3
:10B0D000FFF79EFE0228F6D194F8382094F8391034
:10B0E0008A420FD2531CDBB2A018994284F8383040
:10B0F000007E0AD9234402321B7E84F8382040EABD
:10B10000032038BD4FF6FF7038BD40F47F4038BD96
:10B11000E490FF1F0C2901D900207047023149003B
:10B1200001F0FE01FFF7BCBF70B50C4C037816466A
:10B1300001255B00204684F83B3084F85E5084F89B
:10B140005D50FFF71BFC31462046FFF717FC2946F0
:10B150002046BDE87040FFF7D1BD00BFE490FF1F5F
:10B16000F8B505460F461646412421463A4628467C
:10B17000FFF7DAFF611C0234C9B232462846E4B256
:10B18000FFF7D2FF592CF0D1F8BD00BF38B5044607
:10B190000D463548FFF706FC6322802120462570C6
:10B1A000FFF7C2FF012002F0C9FC204600225E2109
:10B1B000FFF7BAFF20465D21FFF746FF242801D0A4
:10B1C000002038BD204606220C21FFF7C9FF20468B
:10B1D00001222B21FFF7A8FF204601222C21FFF797
:10B1E000A3FF20460E222D21FFF79EFF20460022BE
:10B1F0002E21FFF799FF204601222F21FFF794FF10
:10B20000204605223021FFF78FFF20460122312101
:10B21000FFF78AFF204600223221FFF785FF2046F4
:10B2200000223321FFF780FF204600223421FFF760
:10B230007BFF204600223521FFF776FF20460022C3
:10B240005B21FFF771FF204610225C21FFF76CFFA6
:10B25000204620225D21FFF767FF20468F225E21D6
:10B26000FFF762FF012038BDE490FF1F10B4047F98
:10B270004160022CC26002D010BC01F0D7BB8368D1
:10B2800010BC184790E80C00F0B41C685968256899
:10B29000164F174E29432160164D17491760D66087
:10B2A00015611160417A154A5C180A3194F82440FE
:10B2B00053F8215002EBC40149680D60017A5C1813
:10B2C00003EB8101247ECD6902EBC40149680D6066
:10B2D000817A581803EB810390F83000596B02EB28
:10B2E000C002F0BC53681960704700BF01401F00E6
:10B2F000011000380110007800001F802043010079
:10B30000704700BFF0B50C1EBDF8146034DBB0F917
:10B3100006701919B942C4BF3B1B1BB2002BA646CD
:10B320001CDD002A1146B8BFD11D02F00705CC1064
:10B33000826A012007FB04E1A840012E0A44C0B242
:10B340001ED00CD3022E09D1013B12FA83F3013A2D
:10B3500012F8011F41409A421170F9D1F0BDC0436B
:10B36000013B12FA83F3C0B2013A12F8011F014007
:10B3700093421170F9D1F0BD23441BB20024C6E7FB
:10B38000013B12FA83F3013A12F8011F01439A427A
:10B390001170F9D1F0BD00BFF8B50D1E0EDB1446DB
:10B3A0001F46064601F03AFBA84207DD002C05DBEC
:10B3B000304601F037FBA04201DCF8BDF8BD304655
:10B3C00001F02AFB022853D003284BD0012806D1D4
:10B3D0006540F3886C406540013B5D1B2DB2012F39
:10B3E00003D02AD3022F14D0F8BD002C2246B6F980
:10B3F0000630B06AB8BFE21D42F3CF0202FB03552C
:10B4000004F00704435D012101FA04F41C43445590
:10B41000F8BD002C2246B6F90630B06AB8BFE21D6E
:10B4200042F3CF0202FB035504F00704435D012100
:10B4300001FA04F45C404455F8BD002C2246B6F9EC
:10B440000630B06AB8BFE21D42F3CF0202FB0355DB
:10B4500004F00704435D012101FA04F423EA040423
:10B460004455F8BD3389013B591B25460CB2B6E75C
:10B47000F18832890139013A4D1B141B2DB224B2D7
:10B48000ADE700BF2DE9F041079E9DF91880089DAA
:10B4900004461F4600F0C0FF0D4B0E480E4984F8CD
:10B4A0003380FF22002F08BF1F4684F82F2000237F
:10B4B00084F8302084F8312084F832202060A6659A
:10B4C000E565676261652362A3622046BDE8F0819D
:10B4D000E490FF1F783801000110013810B50446D0
:10B4E000806A034B236008B105F076FB204610BD4F
:10B4F00078380100F8B5436ADBB190F82C200125BB
:10B50000AA4083F83B2083F85E5083F85D500446E0
:10B51000406A03680E461B6800219847606A03680A
:10B5200031461B6898472946606ABDE8F840FFF736
:10B53000E5BBC26BC56C1368046A23EA050313609C
:10B540004CB122684FF00043D3625163D36A002BA1
:10B55000FCDA936BF8BD836B466B0825802410E002
:10B560003768426C3A4332601F68826C3A431A6013
:10B570001A68876C013D22EA07024FEA54041A60F8
:10B5800007D02142ECD13268476C22EA07023260D0
:10B59000EAE7F8BD70B50446406A0D4600282BD096
:10B5A000A16DFFF749FA002D20460CBFA621A72167
:10B5B000FFF7A0FF606A20B1E16DBDE87040FFF7C2
:10B5C0003BBA216C226D0868236A02430A6093B17A
:10B5D000DA7A82B1D00703D5224A99691160DA7A02
:10B5E000910703D5204AD9691160DA7A520702D54A
:10B5F0001E4A1B6A136070BD236A002B2BD0D97AB8
:10B60000626DE1B172B6D97ACE0706D51848D9680D
:10B610000668314099610160D97A880706D51548D6
:10B62000196906683140D9610160D97A4E0705D59C
:10B6300011485969066831401962016062B61B6899
:10B64000D968914207D00D4818600D49DA6042F080
:10B65000804018611960226C216D136823EA010390
:10B660001360A0E700E100E004E100E008E100E091
:10B6700080E100E084E100E088E100E001403F007B
:10B6800000003F80436A2DE9F04105460E46904692
:10B69000002B3ED090F82C100124A14083F83B10E1
:10B6A00083F85E4083F85D40406A036800211B68B0
:10B6B00008F1FF379847FFB2B8F1000F23D03744A5
:10B6C000A046013E686A16F8011F03681B68984788
:10B6D0000134B742E4B216D0202CF3D10121686ABC
:10B6E000FFF70CFB95F82C206B6A520083F83B2087
:10B6F00083F85E8083F85D80686A036800211B68B8
:10B7000098470124DEE7686A0121BDE8F041FFF7B0
:10B71000F5BAC26BC16C136823EA010306EB080497
:10B7200013604FF00048A6420ED02B6A16F801EBCA
:10B7300063B11A68C2F82C80C2F834E0D36A002BD7
:10B74000FCDAA642936BF0D1BDE8F081AB6BD5F883
:10B7500034C008208021DCF800206F6C1EEA010F45
:10B7600014BF3A43BA43CCF800201A68AF6C3A438E
:10B770001A601A68AF6C013822EA07024FEA5101D9
:10B780001A60E8D1CFE700BF70B50446406A0D46A5
:10B79000002828D0A16DFFF74FF920462946FFF772
:10B7A000A9FE606A20B1E16DBDE87040FFF744B9C1
:10B7B000216C226D0868236A02430A6093B1DA7A29
:10B7C00082B1D00703D5234A99691160DA7A9107CB
:10B7D00003D5214AD9691160DA7A520702D51F4A86
:10B7E0001B6A136070BD236A002B2BD0D97A626D5F
:10B7F000E1B172B6D97ACE0706D51948D96806687C
:10B80000314099610160D97A880706D515481969D0
:10B8100006683140D9610160D97A4E0705D51248D2
:10B820005969066831401962016062B61B68D968BF
:10B83000914207D00D4818600D49DA6042F080400F
:10B8400018611960226C216D136823EA01031360EB
:10B85000A3E700BF00E100E004E100E008E100E050
:10B8600080E100E084E100E088E100E001403F0089
:10B8700000003F802DE9F041044686B0806A9DF8C3
:10B8800030801E460F461546B4F90830002800F0F7
:10B890004281DA1D48BF03F10E02B4F90630D2101E
:10B8A00003FB02F2002105F0BBFCB4F90820202ABA
:10B8B00000F39280B4F90610A34B0120203A7339AB
:10B8C00002EBD27201EBD1714FF0200E0290732087
:10B8D0008DE8014042F34F0241F34F01204600F052
:10B8E00051FE606A84F82D70002800F04D81002D13
:10B8F00040F08A80B4F90830202B14BF3D253C2548
:10B9000084F82C50B8F1000F40F0858006B394F90C
:10B910003300002818DBC0B2012102F0E7F8012152
:10B9200094F8330002F0CEF8012002F007F900216C
:10B9300094F8330002F0C6F80A2002F0FFF8012163
:10B9400094F8330002F0BEF8606A002800F08280AC
:10B95000A16DFFF771F804227C492046FFF792FEA3
:10B96000217A0139C9B22046FFF7C4FD7849042283
:10B970002046FFF787FE94F92D30012B14BF1421C8
:10B9800010212046FFF7B6FD042272492046FFF73A
:10B9900079FEB4F90630802B00F09280602B00F025
:10B9A000A680D9212046FFF7A5FD94F92D30012B63
:10B9B00014BFF12122212046FFF79CFD20460622DC
:10B9C0006549FFF75FFE606A50B3E16DFFF734F839
:10B9D000012006B0BDE8F081B4F906105F4B0120EC
:10B9E000403A52394FF0400E029002EBD272522090
:10B9F00001EBD1718DE8014042F34F0241F34F0159
:10BA0000204600F0BFFD6CE76DB284F82C50B8F111
:10BA1000000F3FF47BAFFEF7C5FF002E94D076E712
:10BA2000216C226D0868236A02430A6073B1DA7AD6
:10BA300062B1D00703D54A4A99691160DA7A910751
:10BA40007CD4520702D5474A1B6A1360012006B016
:10BA5000BDE8F081236A002B2BD0D97A626DE1B169
:10BA600072B6D97ACF0706D53F48D968056829400C
:10BA700099610160D97A8E0706D53C481969056835
:10BA80002940D9610160D97A4D0705D538485969EF
:10BA9000056829401962016062B61B68D968914245
:10BAA00007D0344818603449DA6042F080401861A9
:10BAB0001960226C216D136823EA010313604AE7C1
:10BAC000B4F90830202B00F08680402B7FF469AF5A
:10BAD0002A4920460322FFF7D5FD94F92D30012B8A
:10BAE00014BFCF219F212046FFF704FD59E7B4F989
:10BAF0000830102B7FF455AF214920460322FFF771
:10BB0000C1FD94F92D30012B14BFAF211021204627
:10BB1000FFF7F0FC45E7DA1D48BF03F10E02B4F968
:10BB20000630D21003FB02F21046059205F04CF8E5
:10BB3000A06200283FF44DAF059AB3E6114AD969D7
:10BB40001160DA7A7DE700BFD0380100B03A010019
:10BB5000B43A0100B83A0100BC3A0100C43A01000D
:10BB600000E100E008E100E080E100E084E100E0C5
:10BB700088E100E001403F0000003F80CC38010038
:10BB8000843D010004E100E0012194F83100244FDC
:10BB900001F0ACFF94F83200012101F0A7FF94F905
:10BBA000312094F9323057F83220E26357F83330BD
:10BBB000206A23640125E56425651A682A431A6012
:10BBC00078B1B8F1000F3FF428AFFFF75BFB002E10
:10BBD0003FF4BAAE9BE6042212492046FFF752FD1D
:10BBE000DFE6294694F82F0001F080FF294694F8FB
:10BBF000300001F07BFF94F92F2094F9303057F892
:10BC00003220626357F833306564A5641A68A36311
:10BC100022F001021A60002E3FF496AE77E600BFD4
:10BC200020430100C8380100B0F90820D31D48BFE7
:10BC300002F10E03B0F90620806ADB1002FB03F26A
:10BC4000002105F0EDBA00BFF0B50029BDF8145091
:10BC50002EDBB0F90660B1422ADA002A59DBB0F9CE
:10BC6000087014461C44BC42C4BFBB1A1BB2002B54
:10BC70001EDDD2B2D408D0F828E016FB041112F071
:10BC80000702DBB20EEB010421D0C2F10807FAB2C1
:10BC9000374F9342BF5C0CD2C3EB020CFF2646FA2F
:10BCA0000CF6012D07EA06073FD005D3022D36D04A
:10BCB000F0BD012D39D030D21EF8016026EA070709
:10BCC0000EF801709342F3D3B0F906100C449A1A9F
:10BCD000D2B2072A10D9022D36D0002D14BFFF266C
:10BCE000002613462670083BB0F90610DBB2072B7E
:10BCF0000C44F7D802F00702002AD9D01D4B012DC1
:10BD00009B5C1DD017D3022DD2D1227853402370D3
:10BD1000F0BD13441BB20022A1E7022D25D11EF86D
:10BD2000016077400EF80170CCE71EF801603743E0
:10BD30000EF80170C6E7227822EA03032370F0BDF3
:10BD4000227813432370F0BD11462378DB43237020
:10BD50000839B0F90630C9B207291C44F5D812F0E9
:10BD60000702A5D0034B9B5CCFE73444AFE700BF8D
:10BD7000683801005838010070B4C47DBDF80C501B
:10BD8000022C18D0032C1FD0012C0BD0002A03DB6F
:10BD9000B0F90840944201DC70BC7047039570BC58
:10BDA000FFF7B0BAC4880395013CA41A0A4621B231
:10BDB00070BCFFF749BF0689C488013E641AB21AF5
:10BDC000E41A12B221B2E1E704890395E41A641A75
:10BDD000114622B270BCFFF737BF00BF70B4C57DFB
:10BDE000BDF80C60022D1AD0032D12D0012D03D006
:10BDF000039670BCFFF728BFC488E41AA41A0A4649
:10BE000021B2002A03DBB0F90840944213DC70BC75
:10BE100070470489013C641A114622B2F1E7C488D4
:10BE200005890396013CAD1AED1A621A11B22AB2C5
:10BE300070BCFFF709BF039670BCFFF763BA00BF81
:10BE40002DE9F8430446406A002863D0A16DFEF74F
:10BE5000F3FD052274492046FFF714FCA17901394E
:10BE6000C9B22046FFF746FBB4F90820E588A66A68
:10BE7000D31D48BF02F10E03DB10626A15FB03F508
:10BE80001FFA85F8002A7BD094F82C300125AB40AE
:10BE900082F83B3082F85E5082F85D50606A036839
:10BEA00040211B6808F1FF379847BFB2B8F1000F77
:10BEB00023D03744A846013E606A16F8011F036884
:10BEC0001B6898470135B742EDB216D0202DF3D14B
:10BED0000121606AFEF712FF94F82C20636A520079
:10BEE00083F83B2083F85E8083F85D80606A036896
:10BEF00040211B6898470125DEE70121606AFEF7B3
:10BF0000FDFE606A002800F08D80E16DBDE8F84319
:10BF1000FEF792BD236A002B2BD0D97A626DE1B176
:10BF200072B6D97ACE0706D54048D9680568294047
:10BF300099610160D97A8D0706D53D481969056870
:10BF40002940D9610160D97A480705D5394859692E
:10BF5000056829401962016062B61B68D968914280
:10BF600007D0354818603549DA6042F080401861E2
:10BF70001960226C216D136823EA0103136068E7DE
:10BF8000E26BE36C1168276A0B4306EB0809136048
:10BF90004FF0004E4E450DD016F801CB2FB33A6846
:10BFA000C2F82CE0C2F834C0D36A002BFCDA4E454C
:10BFB000936BF1D1226C236D11680B43136097B121
:10BFC000FB7A83B1D90703D51D4BBA691A60FB7A96
:10BFD0009A0703D51B4BFA691A60FB7A5B0702D5F7
:10BFE000194B3A6A1A60BDE8F883A36BD4F8348021
:10BFF00008208021D8F80020656C1CEA010F14BFCE
:10C000002A43AA43C8F800201A68A56C2A431A607C
:10C010001A68A56C013822EA05024FEA51011A603C
:10C02000E8D1B7E7276AC5E76038010080E100E0A2
:10C0300084E100E088E100E001403F0000003F8033
:10C0400000E100E004E100E008E100E02DE9F04F4C
:10C0500085B09946BDF93870BDF83CA0BB1AC1EB5C
:10C06000090B002BB8BF5B42BBF1000FB8BFCBF18F
:10C07000000B5B450D4616460093804648DC4D4557
:10C080003A4633464CDC194613460A46C5EB0901CD
:10C090009B1A89B2002B0CB2B8BF5B4204EBD4747C
:10C0A000BE42ACBF4FF0FF3201224D4503910292D8
:10C0B0004FEA640429DC9BB201930DE0D8F80070CC
:10C0C000BF69B847019BE41AA3B21CB20135002C2A
:10C0D0002DB211DBA94518DB009B5B452A46534670
:10C0E00031464046EADCD8F8002053469769294695
:10C0F00032464046B847E5E7029A1644039AA945F6
:10C1000002EB030436B224B2E6DA05B0BDE8F08FE4
:10C110004A462B46B94635464D4517461E46B2DDC2
:10C12000304629463E464D4607468946AEE700BFA3
:10C1300010B404682469A44610BC604730B4046895
:10C14000BDF808500295A46BA44630BC604700BF00
:10C1500030B40468BDF808500295E46BA44630BCC6
:10C16000604700BF70B40468BDF90C60BDF81050A2
:10C1700003960495246CA44670BC6047704700BFCA
:10C1800010B582B0B0F90C20019101680092002234
:10C190000C6CB0F90A301146A04702B010BD00BFC8
:10C1A000704700BF01F003010129C17506D00329C2
:10C1B00004D0C28803894281838170470289C38881
:10C1C00042818381704700BF2DE9F0410568134E1D
:10C1D0006F6986B0B7420446BDF8308010D1013B8C
:10C1E00013441BB20093CDF804800B46AD6A204681
:10C1F000A8472368DB6AB3420AD106B0BDE8F081E4
:10C20000059304920391B84703A925680EC9E6E790
:10C21000204606B0BDE8F041184700BF7DC10000D0
:10C220002DE9F0410568124E6F6986B0B7420446A9
:10C23000BDF830800FD1013BCDF804800B44009253
:10C240001BB2AD6A2046A8472368DB6AB3420AD115
:10C2500006B0BDE8F081059304920391B84703A9A5
:10C2600025680EC9E7E7204606B0BDE8F04118474B
:10C270007DC100002DE9F04F0568DFF858B06F6907
:10C2800085B05F450646BDF93890BDF83CA00C4628
:10C29000904615D11F19BC420CDACDF800A02146FA
:10C2A00001342D6A4B464246304624B2A847BC4270
:10C2B0003568F2DBEB6A5B4507D105B0BDE8F08F6E
:10C2C0000393B8473568039BE4E7304605B0BDE803
:10C2D000F04F18477DC100002DE9F04387B0994227
:10C2E0000546BDF93840BDF83C6025D0A24212D0C9
:10C2F0000768DFF88080D7F81490C14532D18DE807
:10C3000050002846BC6AA0472B68DB6A434524D10D
:10C3100007B0BDE8F083994202DD0846194603469E
:10C3200028680E96C46B01335B1A1BB22846A446DC
:10C3300007B0BDE8F0436047A24202DD1346224643
:10C340001C4628680E96631C846B9B1A1BB22846F9
:10C35000A44607B0BDE8F0436047284607B0BDE8F3
:10C36000F0431847059304920391C84703A92F6827
:10C370000EC9C4E77DC100002DE9F04FD0F800E000
:10C38000DFF89090DEF814B083B0CB450446BDF9D9
:10C390003080BDF834A00D4617461E4631D1CDF889
:10C3A00000A0DEF824B0294633463A462046D84756
:10C3B0002368CDF800A008F1FF323A44D3F824B046
:10C3C000294612B233462046D8472368CDF800A04C
:10C3D0002946D3F820B03A4643462046D84720683D
:10C3E000CDF800A0711E29444346056A09B23A46B9
:10C3F0002046A8472368DB6A4B4506D103B0BDE859
:10C40000F08FD847D4F800E0C9E7204603B0BDE874
:10C41000F04F18477DC10000F0B4002401264FF60C
:10C42000FF75094F07600471C475C48104824476A6
:10C43000C4618675067685824582C180028141810C
:10C440008281F0BC704700BF903D01002DE9F04FA4
:10C4500085B00668BDF84450BDF93880CDF800803D
:10C4600004460195D6F848B00392BDF93C60BDF989
:10C47000407089469A46D8472368019500974246FE
:10C480005146D3F8488020463346C0472068039B76
:10C490000E930F95856C4B463A4631462046AC4686
:10C4A00005B0BDE8F04F60472DE9F04F87B0174663
:10C4B000BDF9404000912546E91D059344BF2B4638
:10C4C00003F10E010268BDF8486053690294C91077
:10C4D00003912B49BDF9444001968B42824645D1D8
:10C4E000002C3CDD029B3C445E1EB6B24FF00009BE
:10C4F00023B2049301364D46029B002B28DD059B99
:10C50000002403EB090806E0EDB22B0604F1010458
:10C5100011D4A6421CD0A1B211F0070F23B24FEAEA
:10C520004505F1D1002BB8BF0733DB10013418F8F3
:10C5300003502B06EDD5009BD2F818B019443A46AB
:10C5400009B2019B5046D847A642DAF80020E2D152
:10C55000039B01379944049B3FB2BB42CCD1D36AC1
:10C56000074A934206D107B0BDE8F08F9847DAF842
:10C570000020B5E7504607B0BDE8F04F184700BFB0
:10C580007DC1000070B4BDF90C60BDF91050BDF85C
:10C59000144003960495059470BCFFF785BF00BF57
:10C5A0002DE9F04F93B090460591C1691090BDF808
:10C5B00070000790BDF874909DF878A0049300294E
:10C5C00000F0CD800A7A0AC9894604998A1AD2B243
:10C5D00003EBC203BAF1010FDA780B9293F905204D
:10C5E0001E8893F802B00F9293F9064079D913B2DE
:10C5F000099323B20C93109B1A68A94B1193194607
:10C6000053698B4240F0A6800B9B002B55D01FFA3C
:10C6100088F300210D93C8462344DDF8409006912D
:10C620000E930F460C46BBF1000F3FD0BDF818101B
:10C630000C9B03971FFA8AF0CB1813FB00F30490AE
:10C640000E9801440D98034409B21BB20A91089355
:10C65000002505E00135EBB264009B45E4B222D928
:10C66000039B2B44590703D1731C18F806409EB254
:10C670002306EFD5099BBDF81000E91811FB00F166
:10C680000598BAF1010F0FFA8AF301441CD00798FC
:10C6900001900093D26909B217464846089AB847F4
:10C6A000D9F80020D6E7039F5F44FFB2069B0B99A1
:10C6B00001330693DBB29942B5D8D36A119A9342FB
:10C6C00043D113B0BDE8F08F0F9B191893690A9AF4
:10C6D00029441F4609B2079B4846B847D9F80020AD
:10C6E000B8E700230C93099385E70A9A0D9B013262
:10C6F000013B52B213F0FF030A920D936FD1DDF8A4
:10C700001890079BDDF83C80DDF820A04B4517D042
:10C71000BAF1010F00F0C8800B9A109DCDF804907B
:10C720000BEB8B014FEACB030A4400931146DEF872
:10C730001C405346424609B22846A047D5F800E0BF
:10C74000DEF82C30119A9342BBD0109813B0BDE89C
:10C75000F04F1847109D284698472A6854E7109ACA
:10C760000598B2F90A308342ABDDB2F90C3043458B
:10C77000A7DD062313FB0A03002BA2DD08EBCA0387
:10C78000002B9EDD537E2BB9049BAF2B02D90133C6
:10C79000DBB20493109BD3F800E0414B11931A468F
:10C7A000DEF81430934240F08E801FFA88F30E9327
:10C7B00008339BB2BDF81420059305230D93002385
:10C7C0000A93CDF83C800FFA8AF3DDF84080CDF86B
:10C7D00018900B921FFA8AFBCDF820A099460A9A6E
:10C7E000BDF810000B9C0E9D0523194611FB00237C
:10C7F0002C481146C75C039702FB0B4214FA81F3E5
:10C8000012B21BB209920C932C462E461CE0089BD8
:10C810000999012B2AB24B4640462DD0079F01971C
:10C82000CDF80090DEF81CA0D047D8F800E0039BBC
:10C830005B0801340393059BA4B25D445E44A342AC
:10C84000ADB2B6B23FF451AF039BD807DFD4079B1C
:10C85000069A9342EBD0089B012B16D0069B0193BE
:10C86000CDF80090DEF81CA009994B4632B2404644
:10C87000D047D8F800E0DAE7DEF818A0079B0C995B
:10C8800022B2D047D8F800E0D1E7DEF818A00C9922
:10C890001346404622B2D047D8F800E0C7E700BFB1
:10C8A0007DC10000E03D01000B99109DCDF8009086
:10C8B0000531DEF8204009B2424608232846A04749
:10C8C000D5F800E03CE7109C20469847D4F800E0FB
:10C8D0006BE700BFF0B5C36985B004462BB30A29E6
:10C8E00068D00D294AD01A7A914247D3587A8842A3
:10C8F00044D35D688A1A05EBC205AA78002A50D095
:10C90000E87800284DD0207E00283AD095F905E03F
:10C91000B4F90E00A67DB4F90A70724406FB020257
:10C92000BA4262DCB4F9102030E00A2956D00D2951
:10C9300024D0027E002A4BD0B0F90E00A57DB4F9B8
:10C940000A60062212FB0502B2423EDD228AE38122
:10C9500002EBC50212B218462282A78A668A0295A5
:10C960000B468DE8C00001462046FFF719FEA37D67
:10C97000E28903EB430302EB4303E381012005B0AB
:10C98000F0BDA67DB4F90E00B4F91020B4F814E09F
:10C99000678A02960B468DE8804001462046FFF7E5
:10C9A000FFFD2979E389A27D012001FB0233E381A8
:10C9B00005B0F0BD0022C2819A7A817D038A01FB15
:10C9C00002330382012005B0F0BDB4F91020C4E7A2
:10C9D000857DB4F91020B0F90E00BEE7028A817D92
:10C9E000C38102EBC1030382C8E70020E0819B7A88
:10C9F000228A03FB062212B22282C7E7C181028289
:10CA0000704700BF002908BF01218175704700BF32
:10CA100081824182704700BFC07D7047B0F90A0033
:10CA2000704700BFB0F90C00704700BF10B4EFF3BF
:10CA3000108272B6437F33B9017F012907D00329E1
:10CA40000FD00123437702B962B610BC7047124C75
:10CA50002168A1B1114943610B6883610860586185
:10CA6000EFE70F4C216881B10E4943610B68836188
:10CA7000086058610C4B4FF080511960E1E7074B9B
:10CA80004161816120601860DBE7064B4161816193
:10CA900020601860EEE700BF8C9FFF1F889FFF1F7C
:10CAA0007C9FFF1F809FFF1F04ED00E070B5EFF338
:10CAB000108272B60C4C206880B10C4E0025436980
:10CAC000236073B19D6102B962B645778368984768
:10CAD000EFF3108272B620680028F0D102B962B676
:10CAE00070BD3360EFE700BF7C9FFF1F809FFF1F7B
:10CAF000FFF7DCBF184A30B41468002C27D0036855
:10CB000021688B420ED2CB1A00218460C160236061
:10CB1000E06010600223037530BC704711688B42DF
:10CB2000144608D3A2685B1A0360002AF6D182601B
:10CB3000C460A060EEE7D268C2608460E060C5684F
:10CB4000CB1A0222A8602360027530BC7047846053
:10CB5000C4601060DEE700BF849FFF1FF8B5224E5F
:10CB600034682CB32368002B3AD1204F1D4604E0D3
:10CB70003468ECB12368002B32D1A36803B1DD60C7
:10CB800020693360036825751B68BB4221D1037F90
:10CB90004560022BC46020D0FFF748FF6368002B7C
:10CBA000E6D023602046FFF7A5FF3468002CE1D1D2
:10CBB000EFF3108372B60E4A00211068116003B9BA
:10CBC00062B628B18468FFF795FF20460028F9D1A6
:10CBD000F8BD224600219847E0E783689847DDE7E3
:10CBE000013B2360E4E700BF849FFF1F6DB200009C
:10CBF000949FFF1F024A136801331360FFF7AEBF13
:10CC0000A09FFF1F704700BF0368F0B4FBB1002571
:10CC100001249D60DC601B4C1A601C44241104F14B
:10CC200044056A11032692009E60174F0679174B40
:10CC300047F8241002F1604202F5614205F01F0539
:10CC4000012000FA05F5E6541560F0BC7047104C61
:10CC5000236843F40003236000BF0E4B0E4DA4F580
:10CC60008734A4F59E7401261E60234604609C68E8
:10CC7000002CD0D01033AB420360F8D10023036006
:10CC80001846E2E7008FFCBFBC91FF1F44E400E0C0
:10CC90003C80044000700340407103400168A9B12A
:10CCA0000B4BF0B40B441B110A4E0B4F0B4D46F8C7
:10CCB000237003F1440202F01F0401235211A34028
:10CCC000002445F822308C600460F0BC704700BF3F
:10CCD000008FFCBFBC91FF1F05CC000080E100E08D
:10CCE000024A034B012111601B6818470C71034075
:10CCF000BC91FF1F024A034B012111605B6818477A
:10CD00001C710340BC91FF1F024A034B01211160BB
:10CD10009B6818472C710340BC91FF1F024A034BCC
:10CD200001211160DB6818473C710340BC91FF1F73
:10CD3000F8B50E4671B17AB10746144600253B6836
:10CD400016F8011B1B6838469847013C0544F6D18C
:10CD50002846F8BD0846F8BD1046F8BD00B5064A9D
:10CD6000036812885B6883B001A9ADF80420022231
:10CD7000984703B05DF804FBE0420100F0B50746B8
:10CD80008BB0002A33D0012A08BF0A2251B32124D4
:10CD900000E0F4B2B1FBF2F502FB1511C8B20929AB
:10CDA00000F1300198BFC8B20AA988BF37302144CA
:10CDB00088BFC0B201F8240C661E2946002DE8D1B8
:10CDC00033B1013CE4B20AAB23442D2203F8242CF6
:10CDD0003B6801AA11195B683846C4F122029847E2
:10CDE0000BB0F0BD30228DF825202124E8E7036840
:10CDF000C9B21B6898470BB0F0BD00BF0029BABF8D
:10CE000049422D2300230A22FFF7B8BF374A384989
:10CE100013681B06FCD40B6813F08003F8D172B6BC
:10CE200034490A78002A5FD0334A3448F0B4344C8D
:10CE3000176806682568D4680C303E4414320068D0
:10CE40001268304F35442C4420440244C2F34E0251
:10CE50002D4E2E482E4D2F4C42F400423A6037683A
:10CE600006682D682C4A24680C303E44006812681D
:10CE70002A4F35442C4420440244C2F34E02284E2B
:10CE80002848294D294C42F400423A603768066828
:10CE90002D68274A24680C303E4400681268254FEC
:10CEA00035442C4420440244C2F34E02224E23480F
:10CEB000234D244C42F400423A60376806682D68DE
:10CEC000214A24680C303E440068126835442C44E2
:10CED00020440244C2F34E021C4842F40042026065
:10CEE0000B7062B6F0BC704762B6704724B0034066
:10CEF00024B00B40999FFF1F38B003403CB0034063
:10CF000040B003402CB0034058B003405CB0034035
:10CF100060B0034064B003406CB0034030B00340E5
:10CF200038B00B403CB00B4040B00B4044B00B401D
:10CF30004CB00B402CB00B4058B00B405CB00B40D9
:10CF400060B00B4064B00B406CB00B4030B00B4095
:10CF500030B42948294A2A4B2A4D6024E121047023
:10CF600011701B78284C082B30D00A2B27482849F1
:10CF700037D00C2B0CBF35223D2212232A602360B0
:10CF800002600B60234B24491B78244ABBB1012368
:10CF90000B601360224B23491B78234A012B26D9AF
:10CFA000042B0FD9082B1ED9102B94BF862387235F
:10CFB0000B6013601D4B01221A7030BC70470B6070
:10CFC0001360E7E784230B601360F3E700F58E201E
:10CFD0000F490830012213232A60236002600B608E
:10CFE000D0E73922F7E785230B601360E2E780235F
:10CFF0000B601360DEE700BF0040074001400740C0
:10D00000CC91FF1F08B003400CB0034008B00B40A8
:10D010000CB00B409C9FFF1F20B0034020B00B4082
:10D02000CD91FF1F24B0034024B00B40999FFF1FF8
:10D030000C2830B417D91023984228BF18461C4634
:10D04000104A114D1178181A8C42287018D00F49C7
:10D0500013700B7823B10E490E4A00230B60136046
:10D0600030BCFFF775BF0A2802D90C231C46E7E73E
:10D07000082802D90A231C46E2E708231C46DFE7FA
:10D0800030BC7047CC91FF1F989FFF1F999FFF1FD7
:10D0900024B0034024B00B4028282FD8334B2DE96F
:10D0A000F0411E5CFF2E2BD0314B1B78002B2AD178
:10D0B00032062CD472B62F4D2F4C2F4601232660FA
:10D0C0002B7062B672B623681B060CD43B781BB972
:10D0D000F4E72B78002BF1D062B602F09BF972B620
:10D0E00023681806F5D5254B1B6800222A7062B606
:10D0F000234A107843FA00F0BDE8F0810020704721
:10D100000020BDE8F081FFF781FE3206D2D572B66D
:10D110001C4DDFF87C801C4C06F04007FFB206F087
:10D120003F06D8F80030DFB123F01003C8F8003014
:10D1300001232660134A2B7062B672B62368190663
:10D140000CD413781BB9ECE72B78002BE9D062B62E
:10D1500002F060F972B623681B06F5D50B4BC3E7E6
:10D1600043F01003C8F80030E2E700BFE4420100DA
:10D17000999FFF1F9B9FFF1F00B0034010B003400B
:10D18000989FFF1F9A9FFF1F00B00B4010B00B40ED
:10D190000CB00B400A4A0B49136843F480531360E8
:10D1A0000B7843B9084BC0221A70084B80F30C006F
:10D1B00000B218807047044B80221A70F5E700BF58
:10D1C0002C8004409C9FFF1F21C00C4000C00C40DD
:10D1D000F0B51B4B1B4E596818689A68DB6885B020
:10D1E0006C460FC4337899071DD5174A174C13782E
:10D1F000174913F0700318BF1370164A164B802797
:10D20000177000263320032226706D4608701A70AE
:10D2100072B6043C45F001052046A84762B6237863
:10D2200013F0700309D10D4B064901E0013B02D018
:10D230000A78D207FAD505B0F0BD237005B0F0BD6D
:10D2400010430100010002400000024004000240BF
:10D250000B000240070002400A000240410D03009B
:10D26000B0F5006F0AD210B5094B1B78DB070446F6
:10D2700006D504F1A0500078C0B210BD0020704760
:10D28000FFF7A6FF04F1A0500078C0B210BD00BFA8
:10D2900001000240B0F5006F17D238B50F4B1B7874
:10D2A000DA070D46044611D504F1A0500378AB42CD
:10D2B0000AD00B4A137813F0700318BF1370074A93
:10D2C00005701378DB07FCD538BD7047FFF780FF8A
:10D2D00004F1A0500378AB42EBD1F5E70100024026
:10D2E0000000024008B5F4F7ABFCF5F7A9F802F02E
:10D2F00091F8FAE7844641EA000313F003036DD185
:10D30000403A41D351F8043B40F8043B51F8043B08
:10D3100040F8043B51F8043B40F8043B51F8043B0F
:10D3200040F8043B51F8043B40F8043B51F8043BFF
:10D3300040F8043B51F8043B40F8043B51F8043BEF
:10D3400040F8043B51F8043B40F8043B51F8043BDF
:10D3500040F8043B51F8043B40F8043B51F8043BCF
:10D3600040F8043B51F8043B40F8043B51F8043BBF
:10D3700040F8043B51F8043B40F8043B51F8043BAF
:10D3800040F8043B403ABDD2303211D351F8043B4F
:10D3900040F8043B51F8043B40F8043B51F8043B8F
:10D3A00040F8043B51F8043B40F8043B103AEDD2FE
:10D3B0000C3205D351F8043B40F8043B043AF9D24F
:10D3C000043208D0D2071CBF11F8013B00F8013B22
:10D3D00001D30B8803806046704700BF082A13D32F
:10D3E0008B078DD010F003038AD0C3F10403D21A47
:10D3F000DB071CBF11F8013B00F8013B80D331F87B
:10D40000023B20F8023B7BE7043AD9D3013A11F8FA
:10D41000013B00F8013BF9D20B7803704B78437065
:10D420008B7883706046704708B5104C08E023681D
:10D4300059050DD423681A050FD42368DB0411D4D1
:10D4400023685803F3D500F08DFE23685905F1D504
:10D4500002F044F823681A05EFD502F0D5F82368E6
:10D46000DB04EDD500F0F0FCEAE700BF34800440B7
:10D4700008B5FFF7D9FF00BF014B10221A80704793
:10D4800000200540704700BF094908B50B6830B15E
:10D490006A461844A2F58052904202D208601846AB
:10D4A00008BD03F063FB0C2303604FF0FF3008BDA1
:10D4B000D091FF1FFEE700BFEFF3138070B9EFF3C9
:10D4C00010836BB9EFF305825AB94FF48070EFF314
:10D4D00011832BB1984228BF184670474FF0FF3098
:10D4E00070470F2A01D81846F1E7014BD05CEEE7F0
:10D4F000F0E300E0F0B44D1E2E46002400E00134BD
:10D50000B0FBF2F302FB1300092800F130078ABFD9
:10D510003730F8B2C0B206F8010F1846002BEED132
:10D520000A1953704CB1107815F8016F2870013347
:10D53000E01A834202F80169F5DB0846F0BC704747
:10D54000704700BF10B40F4B53F8302092F8804260
:10D550002CB1012369B182F8803010BC704703EB15
:10D56000C0035B681A6841B922F002021A6010BC5D
:10D57000704782F8003110BC704742F003021A6015
:10D5800010BC7047204301001C4A02EBC003012974
:10D590005B6811D004291BD052F83000002280F8BB
:10D5A000802229B1022920D0032922D01A60704795
:10D5B0004FF480721A60704752F830004FF4A27234
:10D5C00080F880121A601A6822F020021A607047F0
:10D5D00052F830104FF4A272012081F880021A60D4
:10D5E0001A6842F020021A60704740F203121A6073
:10D5F00070474FF481721A60704700BF20430100EA
:10D60000212848D8F8B5042A44D8DFE802F0484B6E
:10D610004E0345004FF410262B4B03EBC0030D4681
:10D620005C68216811F4E06148D0284B284A2949F8
:10D63000C3F89C2104F140422748C3F8A411A2F585
:10D640009221264FC3F8A0017C292548C3F8A87170
:10D65000C3F8AC012CD9A2F594237C2B2AD9A2F5CE
:10D6600096237C2B28D9A2F598237C2B29D9A2F5C7
:10D670009A227C2A27D81B4872B6236823F4702389
:10D6800043F08072C4F384011643236040F82150B4
:10D69000266062B6F8BD70474FF43026BCE74FF401
:10D6A0000026B9E74FF44026B6E74FF42026B3E74B
:10D6B0000D48E1E70D48DFE70D48DDE7FFF764FFC0
:10D6C000B3E70C48D8E7F8BD204301000082FF1FF4
:10D6D000F188FF1F9988FF1FC588FF1F6D88FF1FF6
:10D6E0004188FF1FAC92FF1FD491FF1F0C92FF1FB8
:10D6F0005C92FF1F8C92FF1F1A4B03EBC00010B40B
:10D70000426802F14043A3F592217C2923D9A3F575
:10D7100094217C290DD9A3F596217C291FD9A3F545
:10D7200098217C2919D9A3F59A237C2B11D80E4C6A
:10D7300000E00E4C72B613680D4823F08773C2F3F5
:10D74000840123F4803343F08073136044F8210094
:10D7500062B610BC7047074CECE7074CEAE7074C91
:10D76000E8E700BF20430100AC92FF1F0C92FF1FAF
:10D7700041D50000D491FF1F8C92FF1F5C92FF1FC8
:10D7800030B4054B054D064C002210211A602A606A
:10D790002060196030BC704714D0034004D00340AF
:10D7A00000D00340282838B52ED0002904464FDD8C
:10D7B0005F4B1B78012505FA03F28A4202D8212823
:10D7C00037D938BD0338C2B2012A3AD9202C4AD001
:10D7D000192C48D0574A126802FB011222FA03F3AF
:10D7E0001D2800F29B80DFE800F0928B847D9999E0
:10D7F000766F99999999999999999968615A5399D4
:10D800004C99999999999945494B1B780B2B08D9B3
:10D810000C2B1CBF0C3B19410846BDE83840FFF7F4
:10D82000B9BCC3F10C0399400846BDE83840FFF786
:10D83000B1BC2946FFF786FE2946BDE83840FFF710
:10D84000A3BE3D4A126802FB011222FA03F3C7E7A6
:10D850002128B6D80021FFF775FE20460121BDE83A
:10D860003840FFF791BE354A126802FB011222FAD6
:10D8700003F3B5E73249334A0B604FF45173136039
:10D8800038BD3149314A0B604FF45173136038BDD4
:10D890002F49304A0B6040F24443136038BD2E4993
:10D8A0002E4A0B6040F24443136038BD2C492D4A88
:10D8B0000B6040F24443136038BD2B492B4A0B6088
:10D8C00040F24443136038BD29492A4A0B6040F2B4
:10D8D0004443136038BD2849284A0B6040F2444352
:10D8E000136038BD2649274A0B6040F24443136059
:10D8F00038BD2549254A0B6040F24443136038BDCA
:10D900002349244A0B604FF45173136038BD2249F8
:10D91000224A0B604FF45173136038BD212C3FF63F
:10D9200050AF7F29D4BF00210121204693E700BFDB
:10D93000B492FF1F088003400890034008800B400A
:10D9400010800B4048A0044018800B404CA00440BD
:10D950001880034008B004401080034004B0044025
:10D960004080034018C004403880034014C0044085
:10D970002880034010B00440208003400CB00440D5
:10D980003080034010C00440488003401CC0044065
:10D9900018900340349004401090034030900440AD
:10D9A00038B1102828BF1020044AC3B21078137071
:10D9B0007047024A0123107813707047B492FF1F1A
:10D9C0002DE9F8430E4680463249334D304603F088
:10D9D00053F847F6122300281ABF1D464FF00209DC
:10D9E0004FF00109002425FA04F002F04FFE4FF039
:10D9F0005E51074602F0A2FE0146304603F050F8A1
:10DA000030B90134072CEED1E80902F03FFE074699
:10DA10003146384602F046FF4FF07C5102F084FD5B
:10DA200003F078F84FF6FF729042A8F1030328BF85
:10DA30001046012B29D9B8F1170F17D8174B23FA25
:10DA400008F303F0010383F0010223B9B8F1190FC1
:10DA50000FD0BDE8F883124B124D13491A6044EA07
:10DA6000C9042A6008601C60BDE8F883B8F1200F83
:10DA7000ECD10E4B0E4D0F49002244EAC9041A6046
:10DA80002A6008601C60BDE8F8830B4B0B4D0C4905
:10DA9000F2E700BF001BB740006CDC026006F0003C
:10DAA00000800340048003400880034000800B4056
:10DAB00004800B4008800B4000900340049003401A
:10DAC00008900340212801D8FFF73CBD704700BFF4
:10DAD000212806D8044B53F8303093F80002C0B226
:10DAE00070470020704700BF20430100212801D863
:10DAF000FFF74ABD704700BF72B60C490C4B0D4A88
:10DB00001B680868126862B6520102D5322B88BFC2
:10DB100001300949C3F5BB334FF47A72FF33A1FBDF
:10DB2000031302FB00F000EB93107047A09FFF1F50
:10DB300018E000E004ED00E0ABAAAAAA2DE9F84342
:10DB4000054672B6204F214B214A1B683C6812687B
:10DB500062B6520102D5322B88BF013495B3C3F5AA
:10DB6000BB331C4EDFF86490DFF86480FF334FF462
:10DB70007A72A6FB031302FB04F404EB931472B64F
:10DB8000D9F800103A68D8F800E062B6C1F5BB33A6
:10DB9000FF33A6FB03031EF0806FC4EB93134FF417
:10DBA0007A7002D0322988BF013200FB0233B3F50C
:10DBB0007A7F04D3013D05D004F57A74DFE701F0E4
:10DBC00029FCDCE7BDE8F883A09FFF1F18E000E018
:10DBD00004ED00E0ABAAAAAAF8B52D4B2D49DFF859
:10DBE000D0E0DFF8D0C02C4E2C4D2D4C2D4A2E4FBE
:10DBF0004FF4000018604FF0807018604FF0007014
:10DC000018604FF0806018604FF0006018600020CE
:10DC1000086028234BF6FF71CCF80010CEF80030D6
:10DC2000336013602B6023603B60B3629362092210
:10DC300045F8242CC4F8D80F05F57F65C7F8D41F24
:10DC400007F5FF2707F5FA67C6F8F83F2B6006F5DA
:10DC5000FF26C4F8D42F05F5FD2504F5FF24386010
:10DC600006F2F4761148316005F5FF6504F5FD64B0
:10DC70002B6023600260FFF76BF91920FFF75EFF4E
:10DC800000F0B6FF40F21310BDE8F840FFF756BFB2
:10DC900008E100E004800340148003402480034036
:10DCA0002C8003401C8003403480034000800B40E4
:10DCB0000C800340088003402DE9F84F214B1B687E
:10DCC00007460BB101221A70DFF888901E4D99F8B3
:10DCD0000040DFF884801D4E0134272C8ABF4FF0AE
:10DCE000000A5FFA84FA5446AB462B78A34216D159
:10DCF000FFF7E2FB40281FDC33791B06F5D59BF8C4
:10DD000000300133272B86BF00221346DAB218F801
:10DD10000330DBB2F3712A702B78A342E8D00C49B0
:10DD20000A4BFFB208F804700120AC22087089F891
:10DD300000A0DA70BDE8F88FFF28D6DD01F06AFB9D
:10DD4000D3E700BF18A0FF1F15A0FF1F00C00640AB
:10DD500014A0FF1F1CA0FF1FAC9FFF1F1C4BDFF870
:10DD600094C01A681B49F0B542F480521A4D1A60EB
:10DD7000DFF884E0194F1A4E1A4C00238CF800305B
:10DD80004FF451722B701F2840F213358EF800307B
:10DD90003B70337025600A6012D819460124124A7C
:10DDA000124D11701248547000212C274026937296
:10DDB0004FF4003491701174D7702E700460F0BD70
:10DDC000C0F34431C0F3471400F01F03E7E700BF7E
:10DDD000348004400CC00440A99FFF1F15A0FF1F02
:10DDE00014A0FF1F08C0044000C0064031E400E05A
:10DDF00004E100E0A89FFF1F1CA0FF1F034B1B684E
:10DE0000DB0401D5FFF758BF704700BF34800440E2
:10DE100010B5044C237823B101F0FCFA2378002BD1
:10DE2000FAD110BD14A0FF1F054A064B10781B78CD
:10DE3000C0B2DBB2984238BF4030C01A704700BF52
:10DE4000A89FFF1FA99FFF1F30B42B4B1A79940680
:10DE50001FD52A48DA790378294901333F2B0978FD
:10DE6000C8BF00238B42D2B203D0264CD9B2E254B1
:10DE70000170254A116861B1244A1278D2B29342E6
:10DE800036BFC2F140029B1A9B18272BC4BF012347
:10DE90000B70194AD378DBB2180611D45A060DD587
:10DEA000154B1B795B0609D5194B1A491B680022D3
:10DEB0000A7003B11A70104B2C22DA7030BC704714
:10DEC00011790906EAD5144910480C780178C9B2CD
:10DED0008C420DD04A1C272A84BF00210A460F4DD0
:10DEE000054C98BFD1B2AA5CD2B2E2710170D5E7FD
:10DEF0006C21D170D2E700BF00C00640A89FFF1F71
:10DF0000A99FFF1FD49FFF1FA49FFF1F15A0FF1FE6
:10DF100018A0FF1F14A0FF1F1CA0FF1FAC9FFF1F16
:10DF200021282FD8184B195CFF292BD0174B184AE2
:10DF3000DFF870C003EBC000F0B54368DFF868E0BD
:10DF4000144F154D154E00241C60DEF800300120E2
:10DF500043F020038840CEF8003014604FF4A073E3
:10DF600038602E60C2F800C0013BFDD113689B05EC
:10DF7000FCD42023013BFDD1094B09B233F8110039
:10DF800080B2F0BD00207047304401002043010002
:10DF900000500440085004400450044000000203B4
:10DFA0000051044080014A0038800440431E032B86
:10DFB00014D872B60A4951F8230068B170B4094CFC
:10DFC000058834F81320466841F82360521B24F872
:10DFD000132062B670BC704762B67047002070476D
:10DFE00078A0FF1FBCA2FF1F013803280BD872B610
:10DFF000074B53F8203043B100205B680130002B01
:10E00000FBD162B67047002070471846F9E700BFA1
:10E01000CCA0FF1F30B472B62B4A13781D0706D56B
:10E020002A4B196A002936D0996A002941D05378C1
:10E030001C0706D5254B196C00293ED0996C002988
:10E0400039D09378190705D5204B196E002936D0A1
:10E05000996E89B1D3781B0707D51C4BD3F8802064
:10E060007AB3D3F8882011213AB162B6184B002256
:10E070001A7030BC00F04ABE0D21154C154D2278A7
:10E0800043F8315003EBC1030830013A5860227065
:10E0900062B630BC704704220D4C0F4D217843F816
:10E0A000325003EBC20308304A1E5860227062B639
:10E0B000EFE70521E1E70921DFE70822ECE70C2281
:10E0C000EAE71022E8E700BF544401000080FF1F88
:10E0D000F5A0FF1FC800400088004000431E032B2E
:10E0E0001DD81B4A400140F0100030B4104472B6F5
:10E0F000184CE25C032A1BD8DFE802F00212151765
:10E1000003220D88E25410F0080F14BFC82388239F
:10E1100043EA054308310360416062B630BC704792
:10E1200008300222EDE70522EBE708300422E8E799
:10E13000094A52F8230038B1084A52F823004160D6
:10E1400042F8231062B6E9E742F82310034AF7E7E2
:10E150000080FF1F04A1FF1FCCA0FF1FDCA0FF1F3A
:10E1600000BE70472DE9F04FDFF818B3DFF818A3B1
:10E1700087B044E0AD4F4FEA930807EBC809013E72
:10E18000D9F8042003F00803F6B2A2F1080003F066
:10E19000FF04002B40F0018157F838301B0C99B276
:10E1A00022F8081C002B00F0EF80A14B22F8064C4F
:10E1B00042F8044C53F82620002A00F0CF819D4DF0
:10E1C00055F8263058609C4C45F8260034F8163037
:10E1D000194424F8161000F079FD002800F0C281DF
:10E1E000964A974B19F0080F00F1080018BF134624
:10E1F000C9F8040047F8383008238BF800309BF842
:10E200000040E4B265071CD58E4B1B78B3B18E4934
:10E210000A7802F0FF0322B1013BDBB20B7003B9B5
:10E2200000BE8A490A7802F0FF032AB1013BDBB243
:10E230000B70002B00F0688100F066FE04238BF861
:10E24000003004F0080303F0FF02002B00F0C98047
:10E250009AF80030DBB21E098CD19A08DFF8CC9115
:10E2600059F8321009EBC200C1F38301013940684B
:10E270000C2900F28580DFE801F07A7A83838383BA
:10E2800083834683838307000168714D4068714F23
:10E29000714E6860296088B240F281610024674B4A
:10E2A00049F832304FF0010E88423C60C9F8104006
:10E2B000C9F8184086F800E05C4A00F2E780B0F543
:10E2C000D06F80F01B82B0F5817F00F0D98100F221
:10E2D0006981802800F02A82822840F0D781A988AD
:10E2E00001F07F01042900F2D1815C485C4A890079
:10E2F00008441470547001788C0740F1608382F8F0
:10E3000000E0022173E1534F3A682AB3554B524E55
:10E31000554819883478057840298E4645F002081A
:10E3200028BF4FF0400E002C84F001043470CEEB77
:10E3300001010CBF8824C82409EBC80689B285F006
:10E34000010544EA0E447260198049F8384072446D
:10E350000570002965D03A603D4B1A88B2F5A06F70
:10E360000ED100219A785970404B1A7008E0384954
:10E370003F4C0D68A54200F09880304949F83210B2
:10E380003C4A0123137037E72C4A2D4B19F0080F34
:10E3900018BF134647F838302EE700F0B7FC364A6E
:10E3A000364952F82630002B00F0E38058688C5D27
:10E3B00042F8260003F10802C9F80420032C05D80E
:10E3C000DFE804F02C02292602228A551A8819F067
:10E3D000080F0CBF8823C82343EA024347F83830AC
:10E3E0000AE7E00700F19380210600F1D180A2073F
:10E3F00006D5234A234913780220DBB21370087034
:10E40000E30602D51F4B10221A7007B0BDE8F08F4B
:10E4100004228A55DAE705228A55D7E703228A556E
:10E42000D4E7BEF1400F18BF002294E70080FF1F21
:10E4300078A0FF1F24A0FF1FBCA2FF1FC800400040
:10E440008800400000A1FF1F89A0FF1F74A1FF1FCB
:10E45000ECA0FF1F20A0FF1F88A0FF1FC0200740C7
:10E46000F8A0FF1F34A0FF1FF4A0FF1F9820074053
:10E470002109000394200740CCA0FF1F04A1FF1F27
:10E48000882007408020074090200740B0F5106F9B
:10E4900000F07C8140F2A38040F62112904240F0CF
:10E4A0007B82A54A012313706AE74C68A3498C421A
:10E4B0007FF463AF0178A9297FF45FAF41784529E4
:10E4C0007FF45BAF8178C2297FF457AFC1786B29A5
:10E4D0007FF453AF9A489B4E0178347881F0010560
:10E4E000002C41F0020105700CBF8820C82084F088
:10E4F000010449F8310009EBC1019348347000254B
:10E5000005244D60047038E700F064FF94E68F4BFB
:10E5100089488B491A614FF0020E80F800E08C4F59
:10E520000A708C49196099608B4E8C4D8C4C9A61A5
:10E530000D213970FF213170DFF84CE22970227013
:10E54000884D894A8EF800109F27012406F8047C24
:10E550005D600470DA6007B0BDE8F08F43F8260014
:10E56000824D30E6824A47F8380013780133137041
:10E5700042E68B5D032B00F2BA8001A252F823F031
:10E58000F9E10000F9E10000D9E50000D3E5000061
:10E590006F49724B80220D2008701A70A2077FF518
:10E5A0002FAF26E740F20232904240F0ED81AA8878
:10E5B00002F07F02042A69D86D88002D66D1644973
:10E5C000CDF804E0920011440A7842F002020A7089
:10E5D000C1E101238B550FE600238B550CE6B0F506
:10E5E000086F53D16349644A097811707146ED8808
:10E5F0008D4280F0E88252480478402DAE4644F0C7
:10E60000020C28BF4FF0400E02EB0E0309EBCC01C9
:10E61000029301234A604FEA0E48CEEB05010193B5
:10E620000025C82242EA080384F0010249F83C3080
:10E6300035700270DFF814C1424BDFF8048149BB2A
:10E64000BEF1400F7FF42DAF42F0020C09EBCC037A
:10E65000029ADFF8F8E05A608DBB0D0445F088059A
:10E660009DF804304EF83C500A4433700470134651
:10E6700040297FF416AF0021404A3B60118010E72B
:10E68000AA8802F07F02042A40F28B81304A0F23CD
:10E69000137006E74029D7D942F002020CEBC20002
:10E6A000029E4660BDB19DF8045035481D7033464A
:10E6B000403988F8004040334CF83200DCE79DF8E0
:10E6C000043033700D04029B047045F0C8050B4400
:10E6D0004EF83C50CCE79DF804501D70029B1D483D
:10E6E00088F80040403940334CF83200C4E719F054
:10E6F000080F0CBF022303238B557DE521494A688F
:10E70000002AC3D06C88B5F804E003E00C314A68F5
:10E71000002ABBD00B88A342F8D14B887345F5D1B2
:10E72000240A032C0CBF1178098960E7124A0221E0
:10E73000147054705BE700BF942007400100040090
:10E74000F4A0FF1F88A0FF1F89A0FF1F0080FF1FEC
:10E75000C0200740880040008820074080200740F4
:10E760009820074038A0FF1F8CA0FF1F24A0FF1F88
:10E77000F5A0FF1F00A1FF1FF8A0FF1F34A0FF1F7F
:10E78000C8004000584401008C200740B248116A7C
:10E79000AC7804700C0600F19881D9F82820AF49B4
:10E7A000100600F1DB81D9F83020AC49120600F1E7
:10E7B000D081D9F83820A949130600F1C581D9F8CC
:10E7C0004020A649150600F1BA81D9F84820A3498E
:10E7D000140600F1AF81D9F85020A049100600F1CD
:10E7E000A481D9F858209D49120600F19981D9F8E1
:10E7F00060209A49130600F18E81D9F86820974964
:10E80000150600F18381D9F870209449140600F1AF
:10E810007881D9F878209149100600F16D81D9F8F6
:10E8200080208E49120600F16181D9F888208B4939
:10E83000130600F15581D9F890208849150600F19A
:10E840004981D9F898208549140600F1FF80844851
:10E85000844A854901908548854D864C049700235C
:10E860000596029580460F4616461D46039430686D
:10E8700028B1446800F04AFA2046002CF9D1002360
:10E880003360029B38681A46002342F8253028B1CD
:10E89000446800F03BFA2046002CF9D100223A608F
:10E8A000019A98F800301146002241F8042B039A8F
:10E8B0000191023B4FF0000122F81510032B07D8FD
:10E8C000DFE803F05D025D024FF0010388F80030DD
:10E8D0000135042D06F1040607F1040708F10108CB
:10E8E000C5D1654C654D2278654B049F059E00217E
:10E8F000100729701A7000F19280624962780A70DC
:10E900000021C9F83010C9F838101107DFF84C8120
:10E910006ED4A2785C49DFF844810A7000211207A6
:10E92000C9F85010C9F858104BD4E27857494B4CED
:10E930000A7013074FF00001C9F87010C9F8781079
:10E9400000F1AE8033780193002283F00105C9F80D
:10E950009020C9F898200021029188468E460A46E8
:10E960004B48047844F0020C09EBCC030393019B61
:10E97000002B039B5A600CBF8822C82252E64FF03E
:10E98000000388F80030A3E7B0F5A06F7FF47EAEF7
:10E99000012300250193DEE740F621229042F7D0C3
:10E9A00074E66D88002D7FF471AE3A49CDF804E02D
:10E9B000920011440A7822F002020A70CBE7022189
:10E9C00015E600F083F9002800F0EB800830324AA9
:10E9D000C8F86400C8F8602000F078F9002800F05A
:10E9E000DA8008302D4AC9F86C00C9F868209CE725
:10E9F00000F06CF9002800F0E0800830264AC8F8E2
:10EA00004400C8F8402000F061F9002800F0CF80F1
:10EA10000830224AC9F84C00C9F8482079E700F0CC
:10EA200055F9002800F0A58008301B4AC9F82400D9
:10EA3000C9F8202000F04AF9002800F0948008303E
:10EA4000164AC9F82C00C9F8282056E7D1F89C00CE
:10EA5000083800F05BF9FAE600A1FF1F0080FF1FF5
:10EA6000DCA0FF1F78A0FF1FCCA0FF1F04A1FF1F89
:10EA700024A0FF1FBCA2FF1F54440100F5A0FF1FEC
:10EA8000C4200740C8200740CC200740D0200740C2
:10EA9000F4A0FF1FC020074088004000C8004000CD
:10EAA00000F014F9002870D008304F4AC4F88400F0
:10EAB000C4F8802000F00AF9002860D008304B4AE2
:10EAC000C9F88C00C9F888203CE7506A083800F083
:10EAD0001DF962E6D1F89400083800F017F9B0E6A5
:10EAE000D1F88C00083800F011F9A4E6D1F88400C0
:10EAF000083800F00BF998E6C86F083800F006F9FE
:10EB00008DE6486F083800F001F982E6C86E0838D3
:10EB100000F0FCF877E6486E083800F0F7F86CE68D
:10EB2000C86D083800F0F2F861E6486D083800F06A
:10EB3000EDF856E6C86C083800F0E8F84BE6486C8B
:10EB4000083800F0E3F840E6C86B083800F0DEF85B
:10EB500035E6486B083800F0D9F82AE6C86A083864
:10EB600000F0D4F81FE62A78C9F8280001322A708C
:10EB7000C3E62A78C9F8200001322A705AE72A78B9
:10EB8000C9F8880001322A70DCE62A78C4F88000CF
:10EB900001322A708EE72A78C9F8680001322A709B
:10EBA000C3E62A78C8F8600001322A7014E72A7890
:10EBB000C9F8480001322A70ABE62A78C8F840004C
:10EBC00001322A701FE740298E4628BF4FF0400EC1
:10EBD00002EB0E0302930123CEEB01014FEA0E4834
:10EBE00000250193BCE600BF88004000C80040003B
:10EBF000F8B500F08FFD294B29482A4C2A4F2B4DA0
:10EC0000DFF8BCC0DFF8BCE0294E00221A605A6071
:10EC10009A60DA601A615A619A61DA611A625A621C
:10EC20009A62DA621A635A639A63DA631A645A64FC
:10EC30009A64DA641A655A659A65DA651A665A66DC
:10EC40009A66DA661A675A679A67DA67C3F88020A5
:10EC50000168C3F8842041F480210160C3F30721D7
:10EC60002170C3F30740134938701B0E2B70FF232C
:10EC70008CF80030104D8EF8003010480B700123D6
:10EC8000337084F8642070264FF40074102207F863
:10EC90002C3C2E70046081F8F820F8BD0080FF1F26
:10ECA000348004409C200740B0200740B420074037
:10ECB000942007401020074049E400E008E100E00C
:10ECC0008020074088200740704700BF72B60D487B
:10ECD0000268B2FA82F30F2B10DC4FF00041D940EA
:10ECE00022EA0102026062B6074803EBC303DB00BD
:10ECF000C2180021C15010465160704762B6002012
:10ED0000704700BFB892FF1FBC83FF1F0D4B0E4A18
:10ED1000C31AA2FB03231B090F2B0CD80B4A127832
:10ED200052B972B60A484FF00041026821FA03F363
:10ED30001A43026062B67047064A1278002AF0D081
:10ED4000FFF768B9BC83FF1F398EE338F5A0FF1FBA
:10ED5000B892FF1F00A1FF1F38B50E4B0E4C1B6869
:10ED6000218805468BB1B1F5917F05D20B4A4B1C2A
:10ED700055549BB2238038BD002208489847002193
:10ED8000064A55540123238038BDB1F5917FEDD358
:10ED900038BD00BF2CA1FF1FC6A2FF1FCCA2FF1FC2
:10EDA0002DE9F843214E224F3168012380463B7004
:10EDB000B1B1204D4B8801EB8302013300240F2BAE
:10EDC000C2F808802C7004D84B8000233B70BDE84B
:10EDD000F88340230B800320FFF780F93460F4E7C9
:10EDE000DFF8549099F80030002BF0D0114D45F623
:10EDF000215408E0013C12D02B7883B900F00AFBC3
:10EE000099F800307BB10320FFF7EEF80528F1D820
:10EE1000FFF75CFF014630600028EBD0CAE7012312
:10EE20002B70BDE8F883BDE8F88300BF48A1FF1F41
:10EE30001CA1FF1F4CA1FF1F00A1FF1F1201F8B56D
:10EE4000D5B2A1B3012943D04378044600781B060C
:10EE500043EA004040F4704045F004068F1E304302
:10EE6000FFF79EFF022F04F1020314D9053414F8B2
:10EE7000023C14F8032C14F8010C1B0443EA02238F
:10EE8000334343EA0060033FFFF78AFF022F234624
:10EE900004F10304EBD8022F23D0012F0DD045F449
:10EEA000774040F00500BDE8F840FFF779BF14480F
:10EEB0002843BDE8F840FFF773BF187845F477059D
:10EEC00045F0060545EA0020BDE8F840FFF768BFB9
:10EED00003780C4845EA03452843BDE8F840FFF7AE
:10EEE0005FBF1A78587845F0774545F0070545EA41
:10EEF000022545EA0040BDE8F840FFF751BF00BFDA
:10EF000006F0F70007F000F738B5084B1C7824B975
:10EF1000074D296809B14B8803B938BD9B000B80A8
:10EF20000320FFF7DBF82C6038BD00BF1CA1FF1FDA
:10EF300048A1FF1F2DE9F041AD4E33680746002B75
:10EF400000F092801D885A88910803EB81010432F9
:10EF5000AA428C6842D25A8004F00F064FEA142865
:10EF6000A449A6F1080208F00F00C4F30313062A0F
:10EF700000F101050B701AD9B31E012B5FFA88F05E
:10EF80004ED9052E48D0042E00F0A481731F022B09
:10EF90007FD90F2E0ED1F72842D8F02802D0964BF9
:10EFA0001B883BB1FFF7D8FE0020BDE8F08127B1F8
:10EFB000BD4202D00020BDE8F081082EC4F3033327
:10EFC00000F08780092E11D00A2E40F094800A2B81
:10EFD000F0D18A4B8A4A1B68A02181E01846FFF7CE
:10EFE00095FE0420FEF7E2FF3060B5E7092BE1D182
:10EFF000270E00F07B81834B814A1B689021C4F36C
:10F0000007461170EDB2FCB2002B00F09D80224645
:10F0100031462846984797E0F02843D9F72841D051
:10F02000F1380E28C6D801A353F820F0E3F1000010
:10F03000C7F10000B5F10000B5EF0000B5EF00002A
:10F04000A7F10000B5EF000087F20000B5EF000067
:10F0500051F200006BF200008FF10000B5EF0000EC
:10F0600077F100005BF10000674B1B78002BA1D00B
:10F070000420FEF79BFF0346306000289AD00588E5
:10F08000002D7FF460AFFFF741FE35602846BDE8F4
:10F09000F081FFF761FEC4F30740FFF75DFE072E26
:10F0A00002D1200EFFF758FE534B584A1988584892
:10F0B0001468584D524A017000270E0AF0201F8034
:10F0C0002E7010700CB301225348A0470120BDE8F8
:10F0D000F081082B7FF46EAF504B494A1B688021AA
:10F0E000C4F307461170EDB2240E6BB328462246D6
:10F0F0003146984728E00B2E11D10B2B7FF45AAFE5
:10F10000474B3F4A1B68B021EAE7464B1B68002B80
:10F1100000F0FB80404898470120BDE8F0810C2EAC
:10F1200040F000810C2B7FF445AF3F4B344A1B6805
:10F13000C0211170EDB2C4F30746002B00F0C88067
:10F1400028463146240E98473849314A314B0D70D4
:10F1500016701C700120BDE8F081354B1B68002B38
:10F1600000F0D6809847C4F30746254BEDB2240E35
:10F1700083F80080E8E72F4B1B68002BF2D12E4B61
:10F180001B68A3B1FE209847C4F30746EDE72B4B5D
:10F190001B68002BE6D1284B1B6843B1FC20984725
:10F1A000C4F30746E1E7264B1B68002BDAD1C4F312
:10F1B0000746DAE7234B1B68C4F30746002BD4D07D
:10F1C00030469847D1E7204B1A68002AEFD0260C2A
:10F1D000630C06F07F0003F47E531843F6B29047A9
:10F1E000C3E71A4B1B68C4F30746002BE8D1BCE702
:10F1F00054A1FF1FCAA2FF1FC6A2FF1F30A1FF1FFD
:10F20000C4A2FF1F64A1FF1F00A1FF1F2CA1FF1FAD
:10F21000C8A2FF1FC9A2FF1FCCA2FF1F5CA1FF1F36
:10F2200060A1FF1F44A1FF1F20A1FF1FCBA2FF1F52
:10F230000CA1FF1F10A1FF1F14A1FF1F50A1FF1F52
:10F2400040A1FF1F58A1FF1F28A1FF1F3CA1FF1FC6
:10F250003F4B1B68002B85D13E4B1B68002BA6D073
:10F26000FA209847C4F307467FE73B4B1B68002B07
:10F270007FF478AF374B1B68002B98D0FB20984762
:10F28000C4F3074671E7354B1B68002B7FF46AAF68
:10F29000304B1B68002B8AD0F8209847C4F30746F0
:10F2A00063E70E2B7FF486AE2D4A2E4B1268E021C9
:10F2B0001970002A47D0260C610C06F07F0301F478
:10F2C0007E511943EDB2A1F5005128469047F6B2A0
:10F2D000240E39E7FFF740FDC4F30740FFF73CFD7C
:10F2E000200EFFF739FD0020BDE8F0811E4B1D4ABE
:10F2F0001B6880211170EDB2C4F3074683B131461B
:10F3000028463A4698473C461EE70120BDE8F08172
:10F31000104B1B68002B3FF44AAFFF20984746E78D
:10F320001C4611E70D2EBCD10D2B7FF443AE0F4BC5
:10F330000C4A1B68D0211170EDB2C4F30746002BB4
:10F340007FF4FEAEC4E7C4F30746EDB2240EFBE63D
:10F3500038A1FF1F14A1FF1F18A1FF1F08A1FF1F45
:10F3600024A1FF1FC4A2FF1F5CA1FF1F34A1FF1F28
:10F3700038B5164D2868E0B101884488A14213DDF4
:10F3800003191B7A83B104F10803C2180C1B002374
:10F3900002E012F8011F21B10133A342F9D1204646
:10F3A00038BD1C46204638BDFFF7B0FC0020286061
:10F3B00038BD074B1B780BB9002038BD0220FEF783
:10F3C000F5FD28600028D7D1F6E700BF70A1FF1F28
:10F3D00000A1FF1F0D4B1B78BBB910B50C4C216869
:10F3E00003F0FF024B883F2B07DC07330B4401F18E
:10F3F000470003F8012F8342FBD140230B800120FB
:10F40000FEF76CFE0023236010BD704768A1FF1F4C
:10F410006CA1FF1F38B5224C237803B138BD0123FE
:10F420002370FFF7A5FF70BB00F048F840BB00F069
:10F43000DBF810BBFEF7F8FCE0B900232370EFF314
:10F440000583002BEAD1EFF3108172B6154B1868D3
:10F45000E0B1154C2278CAB945691D6001232370BB
:10F46000C5B1AA6101B962B600254577836898479E
:10F470002570D3E700F020F8DFE700F01BF8D9E7AC
:10F4800000F016F8D3E7FFF71FFCCDE70029C5D140
:10F4900062B638BD054B1D600029E5D1E3E700BF2A
:10F4A00075A1FF1F8C9FFF1F909FFF1F889FFF1F4D
:10F4B000704700BF704700BF704700BF054A064B4A
:10F4C00010781B78C0B2DBB2984238BF4030C01A07
:10F4D000704700BF7CA1FF1F7DA1FF1FF0B4384B18
:10F4E0001A7912F0300F2CD072B6997D01F0FF021C
:10F4F00000293DD062B6334F334938780D78334E0A
:10F500001C46C0B2EDB2431C402BE17928BF00235A
:10F51000AB4202F1FF32C9B21CBFF154184612F0DF
:10F52000FF02F0D12A4B1B68C2B23A704BB1A8421D
:10F5300036BFC5F14005401B40192728C4BF012232
:10F540001A701F49CA78D2B2150616D452060DD5C4
:10F550001B4B1B795B0609D51E4B1F491B680022FC
:10F560000A7003B11A70164B3C22DA70F0BC704777
:10F570004022D9795A7462B6E3E70B791C06E5D5C7
:10F58000164B174E1C783378E4B2DBB29C420ED097
:10F59000144D01E0A3420AD00133402B28BF0023C1
:10F5A0000879E85CC0B2C871087D0728F2D9DBB2DF
:10F5B000034933700B79180644BF7C23CB70C5E731
:10F5C00000A006407CA1FF1F7DA1FF1FC0A1FF1F5F
:10F5D00078A1FF1F04A2FF1F00A2FF1F08A2FF1FA8
:10F5E00001A2FF1F80A1FF1F054A064B10781B7860
:10F5F000C0B2DBB2984238BF4030C01A704700BF7B
:10F600007CA2FF1F11A2FF1FF0B4384B1A7912F031
:10F61000300F2CD072B6997D01F0FF0200293DD049
:10F6200062B6334F334938780D78334E1C46C0B23A
:10F63000EDB2431C402BE17928BF0023AB4202F11D
:10F64000FF32C9B21CBFF154184612F0FF02F0D1CC
:10F650002A4B1B68C2B23A704BB1A84236BFC5F103
:10F660004005401B40192728C4BF01221A701F49BA
:10F67000CA78D2B2150616D452060DD51B4B1B798B
:10F680005B0609D51E4B1F491B6800220A7003B197
:10F690001A70164B3C22DA70F0BC70474022D979C0
:10F6A0005A7462B6E3E70B791C06E5D5164B174E84
:10F6B0001C783378E4B2DBB29C420ED0144D01E0EA
:10F6C000A3420AD00133282B28BF00230879E85C25
:10F6D000C0B2C871087D0728F2D9DBB20349337084
:10F6E0000B79180644BF7C23CB70C5E700B00640F9
:10F6F0007CA2FF1F11A2FF1F3CA2FF1F0CA2FF1F35
:10F7000080A2FF1F10A2FF1F84A2FF1F7DA2FF1F68
:10F7100014A2FF1F70B584B072B6194B194D1A4868
:10F72000702241260F2480211A702E701A46047010
:10F73000197013781B06FCD5144B186862B6144B6D
:10F74000144C984298BF00EB800001A998BF40007C
:10F750000A22FDF7CFFE01A92046002311F8012B54
:10F7600001333AB10A2B20F8022FF7D11623237068
:10F7700004B070BD5B00DBB2237004B070BD00BF8D
:10F78000000002400700024006000240080002405C
:10F790007F9698008493FF1F2DE9F043DFF8EC80FB
:10F7A0008BB006460F4600F073F898F9003001332D
:10F7B00004460D4637D03046394600F0DFF90028C0
:10F7C00031D02BA3D3E900233046394600F026FE82
:10F7D000814668BB28A3D3E900233046394600F0B0
:10F7E000FFFD00B398F90030254ACDF8209004249D
:10F7F00000200021022BCDE90467CDE902670094C7
:10F800000192CDE906012CD0684600F0BDF940B365
:10F81000089B1BB101F0AAF9089B0360DDE9060112
:10F820000BB0BDE8F083204629460BB0BDE8F0835D
:10F83000134A98F90030019203210022CDE90467B0
:10F84000CDE90267009108922BB90E4B4FF0604250
:10F85000CDE90623D8E70C490020022BCDE90601AB
:10F86000D2D101F083F922230360D1E7AFF3008006
:10F87000EF39FAFE422E864051302DD5104987C00F
:10F88000C4440100FFFFEF470000F07F9A93FF1F81
:10F890002DE9F04FB04F21F00042BA4283B00C4640
:10F8A0004FEAD17605460DD9AC4FBA4225D9C1F3FE
:10F8B0001303034340F0EF800EB10020014603B074
:10F8C000BDE8F08FA64B9A4200F2CC80A54B9A423D
:10F8D00000F2DE808AA3D3E9002300F05DF9002264
:10F8E000A14B00F09BFD002800F005812846214631
:10F8F00000229D4B00F050F9E1E783A3D3E90023F8
:10F9000000F08CFD002840F0CB802846214680A3E3
:10F91000D3E9002300F064FD0028CED1934B2846A4
:10F9200003EBC60821467CA3D3E9002300F0E6FAE6
:10F93000D8E9002300F030F900F07AFD804600F0AD
:10F9400077FA77A3D3E9002306460F4600F0D6FAEC
:10F9500002460B462846214600F01CF972A3D3E963
:10F960000023CDE900013046394600F0C7FA82464F
:10F970008B4652465B46DDE9000100F00BF9054677
:10F980000C462A4623462846214600F0B7FA68A3CB
:10F99000D3E9002306460F4600F0B0FA66A3D3E988
:10F9A000002300F0F7F832463B4600F0A7FA64A3C4
:10F9B000D3E9002300F0F0F832463B4600F09EFA0F
:10F9C00061A3D3E9002300F0E5F832463B4600F09E
:10F9D00095FA5FA3D3E9002300F0DEF832463B46F8
:10F9E00000F08CFA02460B462846214600F0D2F879
:10F9F00006460F462846214632463B46B8F1000FE0
:10FA000056D000F07BFA324604460D463B460020B5
:10FA10004FF0804100F0BEF802460B4620462946D2
:10FA200000F096FB02460B465046594600F0B2F8ED
:10FA3000DDE9002300F0AEF80B4602464A490020FB
:10FA400000F0A8F86FF47F7398454FDA08F57A78DC
:10FA500001EB085100224FF0B87300F04FFA03B0E9
:10FA6000BDE8F08F424B9A423FF658AF414BF4004D
:10FA70002344D3E9002300F08DF83F4BC6F1010881
:10FA80001C44CDE90001D4E900ABC6EB080870E7DF
:10FA90004FF0000875E702460B4600F07DF80EE7D0
:10FAA00017A3D3E900231046194600F027FA06E70A
:10FAB00000F024FA0022804689464FF08043304609
:10FAC000394600F067F802460B464046494600F0CA
:10FAD0003FFB2A46234600F05DF802460B46002015
:10FAE000214900F057F803B0BDE8F08F01EB085151
:10FAF00003B0BDE8F08F804643E700BFAFF300805E
:10FB00009C7500883CE4377EEF39FAFE422E864031
:10FB100051302DD5104987C0FE822B654715F73F20
:10FB20000000E0FE422EE63F763C7935EF39EA3DB3
:10FB3000D0A4BE726937663EF16BD2C541BDBB3EF3
:10FB40002CDE25AF6A56113F93BDBE166CC1663FD1
:10FB50003E5555555555C53F412E8640FFFFEF7F19
:10FB6000422ED63FFFFF2F3E0000F03FC844010069
:10FB7000B1A2F03FE8440100D844010041F0004147
:10FB800001F58010C00F70470020704781F00041E0
:10FB900002E000BF83F0004330B54FEA41044FEA72
:10FBA000430594EA050F08BF90EA020F1FBF54EA0D
:10FBB000000C55EA020C7FEA645C7FEA655C00F0A9
:10FBC000E2804FEA5454D4EB5555B8BF6D420CDD7A
:10FBD0002C4480EA020281EA030382EA000083EAFD
:10FBE000010180EA020281EA0303362D88BF30BD9D
:10FBF00011F0004F4FEA01314FF4801C4CEA1131F3
:10FC000002D0404261EB410113F0004F4FEA033351
:10FC10004CEA133302D0524263EB430394EA050FDC
:10FC200000F0A780A4F10104D5F1200E0DDB02FA4B
:10FC30000EFC22FA05F2801841F1000103FA0EF2DF
:10FC4000801843FA05F359410EE0A5F120050EF1A5
:10FC5000200E012A03FA0EFC28BF4CF0020C43FAD6
:10FC600005F3C01851EBE37101F0004507D54FF0E3
:10FC7000000EDCF1000C7EEB00006EEB0101B1F533
:10FC8000801F1BD3B1F5001F0CD349085FEA300079
:10FC90004FEA3C0C04F101044FEA445212F5800F84
:10FCA00080F09A80BCF1004F08BF5FEA500C50F121
:10FCB000000041EB045141EA050130BD5FEA4C0C04
:10FCC000404141EB010111F4801FA4F10104E9D18D
:10FCD00091F0000F04BF01460020B1FA81F308BF84
:10FCE0002033A3F10B03B3F120020CDA0C3208DD50
:10FCF00002F1140CC2F10C0201FA0CF021FA02F12B
:10FD00000CE002F11402D8BFC2F1200C01FA02F19A
:10FD100020FA0CFCDCBF41EA0C019040E41AA2BFBF
:10FD200001EB0451294330BD6FEA04041F3C1CDA87
:10FD30000C340EDC04F11404C4F1200220FA04F0A7
:10FD400001FA02F340EA030021FA04F345EA030151
:10FD500030BDC4F10C04C4F1200220FA02F001FA13
:10FD600004F340EA0300294630BD21FA04F0294695
:10FD700030BD94F0000F83F4801306BF81F480112E
:10FD80000134013D4EE77FEA645C18BF7FEA655CA1
:10FD900029D094EA050F08BF90EA020F05D054EA73
:10FDA000000C04BF1946104630BD91EA030F1EBF78
:10FDB0000021002030BD5FEA545C05D1400049417C
:10FDC00028BF41F0004130BD14F580043CBF01F56F
:10FDD000801130BD01F0004545F0FE4141F4700155
:10FDE0004FF0000030BD7FEA645C1ABF1946104630
:10FDF0007FEA655C1CBF0B46024650EA013406BF31
:10FE000052EA033591EA030F41F4002130BD00BFEF
:10FE100090F0000F04BF0021704730B54FF48064AC
:10FE200004F132044FF000054FF0000150E700BF2D
:10FE300090F0000F04BF0021704730B54FF480648C
:10FE400004F1320410F0004548BF40424FF0000179
:10FE50003EE700BF42004FEAE2014FEA31014FEABC
:10FE600002701FBF12F07F4393F07F4F81F060510B
:10FE7000704792F0000F14BF93F07F4F704730B57A
:10FE80004FF4607401F0004521F0004120E700BF0D
:10FE900050EA010208BF704730B54FF000050AE094
:10FEA00050EA010208BF704730B511F0004502D595
:10FEB000404261EB41014FF4806404F132045FEA97
:10FEC000915C3FF4DCAE4FF003025FEADC0C18BF3C
:10FED00003325FEADC0C18BF033202EBDC02C2F132
:10FEE000200300FA03FC20FA02F001FA03FE40EAC4
:10FEF0000E0021FA02F11444C1E600BF70B54FF0C4
:10FF0000FF0C4CF4E06C1CEA11541DBF1CEA1355A5
:10FF100094EA0C0F95EA0C0F00F0DEF82C4481EA0D
:10FF2000030621EA4C5123EA4C5350EA013518BF2D
:10FF300052EA033541F4801143F4801338D0A0FB1A
:10FF400002CE4FF00005E1FB02E506F00042E0FBC7
:10FF500003E54FF00006E1FB03569CF0000F18BFCD
:10FF60004EF0010EA4F1FF04B6F5007F64F5407475
:10FF700004D25FEA4E0E6D4146EB060642EAC62108
:10FF800041EA55514FEAC52040EA5E504FEACE2E75
:10FF9000B4F1FD0C88BFBCF5E06F1ED8BEF1004F78
:10FFA00008BF5FEA500E50F1000041EB045170BDF4
:10FFB00006F0004646EA010140EA020081EA030138
:10FFC000B4EB5C04C2BFD4EB0C0541EA045170BD34
:10FFD00041F480114FF0000E013C00F3AB8014F1AE
:10FFE000360FDEBF002001F0004170BDC4F10004F7
:10FFF000203C35DA0C341BDC04F11404C4F1200578
:020000021000EC
:1000000000FA05F320FA04F001FA05F240EA0200D2
:1000100001F0004221F0004110EBD37021FA04F608
:1000200042EB06015EEA430E08BF20EAD37070BDC2
:10003000C4F10C04C4F1200500FA04F320FA05F021
:1000400001FA04F240EA020001F0004110EBD37023
:1000500041F100015EEA430E08BF20EAD37070BD93
:10006000C4F1200500FA05F24EEA020E20FA04F36C
:1000700001FA05F243EA020321FA04F001F000411B
:1000800021FA04F220EA020000EBD3705EEA430E8C
:1000900008BF20EAD37070BD94F0000F0FD101F0BB
:1000A0000046400041EB010111F4801F08BF013CF4
:1000B000F7D041EA060195F0000F18BF704703F032
:1000C0000046520043EB030313F4801F08BF013DB9
:1000D000F7D043EA0603704794EA0C0F0CEA135575
:1000E00018BF95EA0C0F0CD050EA410618BF52EA2F
:1000F0004306D1D181EA030101F000414FF0000035
:1001000070BD50EA410606BF1046194652EA430642
:1001100019D094EA0C0F02D150EA013613D195EAB6
:100120000C0F05D152EA03361CBF104619460AD1FE
:1001300081EA030101F0004141F0FE4141F4700108
:100140004FF0000070BD41F0FE4141F4780170BDF8
:1001500070B54FF0FF0C4CF4E06C1CEA11541DBF5D
:100160001CEA135594EA0C0F95EA0C0F00F0A7F85F
:10017000A4EB050481EA030E52EA03354FEA01318C
:1001800000F088804FEA03334FF0805545EA13139F
:1001900043EA12634FEA022245EA111545EA106567
:1001A0004FEA00260EF000419D4208BF964244F1FE
:1001B000FD0404F5407402D25B084FEA3202B61A1D
:1001C00065EB03055B084FEA32024FF480104FF4F1
:1001D000002CB6EB020E75EB030E22BFB61A754665
:1001E00040EA0C005B084FEA3202B6EB020E75EBF8
:1001F000030E22BFB61A754640EA5C005B084FEA60
:100200003202B6EB020E75EB030E22BFB61A75462C
:1002100040EA9C005B084FEA3202B6EB020E75EB37
:10022000030E22BFB61A754640EADC0055EA060EF8
:1002300018D04FEA051545EA16754FEA06164FEA3B
:10024000C30343EA52734FEAC2025FEA1C1CC0D1E7
:1002500011F4801F0BD141EA00014FF000004FF074
:10026000004CB6E711F4801F04BF01430020B4F135
:10027000FD0C88BFBCF5E06F3FF6AFAEB5EB030CED
:1002800004BFB6EB020C5FEA500C50F1000041EBEA
:10029000045170BD0EF0004E4EEA113114EB5C04B7
:1002A000C2BFD4EB0C0541EA045170BD41F480118A
:1002B0004FF0000E013C90E645EA060E8DE60CEA92
:1002C000135594EA0C0F08BF95EA0C0F3FF43BAFAF
:1002D00094EA0C0F0AD150EA01347FF434AF95EA66
:1002E0000C0F7FF425AF104619462CE795EA0C0F4A
:1002F00006D152EA03353FF4FDAE1046194622E717
:1003000050EA410618BF52EA43067FF4C5AE50EAF0
:1003100041047FF40DAF52EA43057FF4EBAE12E7E0
:100320004FF0FF3C06E000BF4FF0010C02E000BFC1
:100330004FF0010C4DF804CD4FEA410C7FEA6C5CA4
:100340004FEA430C18BF7FEA6C5C1BD001B050EA47
:10035000410C0CBF52EA430C91EA030F02BF90EA32
:10036000020F0020704710F1000F91EA030F58BFF1
:10037000994208BF90422CBFD8176FEAE37040F053
:10038000010070474FEA410C7FEA6C5C02D150EAF1
:10039000013C07D14FEA430C7FEA6C5CD6D152EAAC
:1003A000033CD3D05DF8040B704700BF8446104671
:1003B00062468C461946634600E000BF01B5FFF770
:1003C000B7FF002848BF10F1000F01BD4DF808ED40
:1003D000FFF7F4FF0CBF012000205DF808FB00BF11
:1003E0004DF808EDFFF7EAFF34BF012000205DF86B
:1003F00008FB00BF4DF808EDFFF7E0FF94BF0120B8
:1004000000205DF808FB00BF4DF808EDFFF7CEFFB8
:1004100094BF012000205DF808FB00BF4DF808EDF7
:10042000FFF7C4FF34BF012000205DF808FB00BFC8
:100430004FEA410212F5001215D211D56FF478730C
:10044000B3EB625212D94FEAC12343F0004343EAAF
:10045000505311F0004F23FA02F018BF404270478A
:100460004FF00000704750EA013005D111F0004014
:1004700008BF6FF0004070474FF00000704700BFAA
:100480004FEA4102B2F1E04324BFB3F5001CDCF1B6
:10049000FE5C0DD901F0004C4FEAC0024CEA5070EE
:1004A000B2F1004F40EB830008BF20F0010070471D
:1004B00011F0804F21D113F13872BCBF01F0004020
:1004C000704741F480114FEA5252C2F11802C2F152
:1004D000200C10FA0CF320FA02F018BF40F00100D3
:1004E0004FEAC1234FEAD32303FA0CFC40EA0C0085
:1004F00023FA02F34FEA4303CCE77FEA625307D1C2
:1005000050EA01331EBF4FF0FE4040F440007047F8
:1005100001F0004040F0FE4040F40000704700BF92
:1005200080F0004002E000BF81F0004142001FBFA8
:100530005FEA410392EA030F7FEA226C7FEA236CB1
:100540006AD04FEA1262D2EB1363C1BFD2184140A6
:1005500048404140B8BF5B42192B88BF704710F03C
:10056000004F40F4000020F07F4018BF404211F0DF
:10057000004F41F4000121F07F4118BF494292EA47
:10058000030F3FD0A2F1010241FA03FC10EB0C0073
:10059000C3F1200301FA03F100F0004302D5494200
:1005A00060EB4000B0F5000F13D3B0F1807F06D3AD
:1005B00040084FEA310102F10102FE2A51D2B1F1A5
:1005C000004F40EBC25008BF20F0010040EA03009A
:1005D0007047490040EB000010F4000FA2F1010247
:1005E000EDD1B0FA80FCACF1080CB2EB0C0200FAD1
:1005F0000CF0AABF00EBC25052421843BCBFD0401F
:100600001843704792F0000F81F4000106BF80F498
:1006100000000132013BB5E74FEA41037FEA226C5B
:1006200018BF7FEA236C21D092EA030F04D092F026
:10063000000F08BF0846704790EA010F1CBF00205A
:10064000704712F07F4F04D1400028BF40F00040B7
:10065000704712F100723CBF00F50000704700F0D7
:10066000004343F0FE4040F4000070477FEA2262FE
:1006700016BF08467FEA23630146420206BF5FEACF
:10068000412390EA010F40F4800070474FF00003CF
:1006900004E000BF10F0004348BF40425FEA000C96
:1006A00008BF704743F0964301464FF000001CE03E
:1006B00050EA010208BF70474FF000030AE000BF94
:1006C00050EA010208BF704711F0004302D54042D2
:1006D00061EB41015FEA010C02BF84460146002044
:1006E00043F0B64308BFA3F18053A3F50003BCFA5F
:1006F0008CF2083AA3EBC25310DB01FA02FC63440C
:1007000000FA02FCC2F12002BCF1004F20FA02F212
:1007100043EB020008BF20F00100704702F1200205
:1007200001FA02FCC2F1200250EA4C0021FA02F266
:1007300043EB020008BF20EADC7070474FF0FF0C6B
:100740001CEAD0521EBF1CEAD15392EA0C0F93EA66
:100750000C0F6FD01A4480EA010C400218BF5FEA08
:1007600041211ED04FF0006343EA501043EA51117B
:10077000A0FB01310CF00040B1F5000F3EBF490075
:1007800041EAD3715B0040EA010062F17F02FD2A79
:100790001DD8B3F1004F40EBC25008BF20F001005C
:1007A000704790F0000F0CF0004C08BF49024CEA73
:1007B000502040EA51207F3AC2BFD2F1FF0340EA05
:1007C000C250704740F400004FF00003013A5DDC76
:1007D00012F1190FDCBF00F000407047C2F10002B7
:1007E000410021FA02F1C2F1200200FA02FC5FEAA4
:1007F000310040F1000053EA4C0308BF20EADC70EE
:10080000704792F0000F00F0004C02BF400010F45F
:10081000000F013AF9D040EA0C0093F0000F01F00C
:10082000004C02BF490011F4000F013BF9D041EA2E
:100830000C018FE70CEAD15392EA0C0F18BF93EA30
:100840000C0F0AD030F0004C18BF31F0004CD8D15A
:1008500080EA010000F00040704790F0000F17BFE1
:1008600090F0004F084691F0000F91F0004F14D027
:1008700092EA0C0F01D142020FD193EA0C0F03D17F
:100880004B0218BF084608D180EA010000F0004082
:1008900040F0FE4040F40000704740F0FE4040F45D
:1008A000400070474FF0FF0C1CEAD0521EBF1CEAFC
:1008B000D15392EA0C0F93EA0C0F69D0A2EB03021A
:1008C00080EA010C49024FEA402037D04FF08053B4
:1008D00043EA111143EA10130CF000408B4238BF79
:1008E0005B0042F17D024FF4000C8B4224BF5B1A87
:1008F00040EA0C00B3EB510F24BFA3EB510340EAD5
:100900005C00B3EB910F24BFA3EB910340EA9C0082
:10091000B3EBD10F24BFA3EBD10340EADC001B01F2
:1009200018BF5FEA1C1CE0D1FD2A3FF650AF8B4296
:1009300040EBC25008BF20F0010070470CF0004CA3
:100940004CEA50207F32C2BFD2F1FF0340EAC250CE
:10095000704740F400004FF00003013A37E792F08F
:10096000000F00F0004C02BF400010F4000F013AED
:10097000F9D040EA0C0093F0000F01F0004C02BFE8
:10098000490011F4000F013BF9D041EA0C0195E751
:100990000CEAD15392EA0C0F08D142027FF47DAFEA
:1009A00093EA0C0F7FF470AF084676E793EA0C0FDA
:1009B00004D14B023FF44CAF08466EE730F0004CD8
:1009C00018BF31F0004CCAD130F000427FF45CAF68
:1009D00031F000437FF43CAF5FE700BF4FF0FF3CD6
:1009E00006E000BF4FF0010C02E000BF4FF0010C29
:1009F0004DF804CD4FEA40024FEA41037FEA226CF2
:100A000018BF7FEA236C11D001B052EA530C18BF13
:100A100090EA010F58BFB2EB030088BFC81738BF78
:100A20006FEAE17018BF40F0010070477FEA226C66
:100A300002D15FEA402C05D17FEA236CE4D15FEA62
:100A4000412CE1D05DF8040B704700BF8446084696
:100A50006146FFE70FB5FFF7C9FF002848BF10F157
:100A6000000F0FBD4DF808EDFFF7F4FF0CBF01209C
:100A700000205DF808FB00BF4DF808EDFFF7EAFF26
:100A800034BF012000205DF808FB00BF4DF808EDE1
:100A9000FFF7E0FF94BF012000205DF808FB00BFD6
:100AA0004DF808EDFFF7D2FF94BF012000205DF85C
:100AB00008FB00BF4DF808EDFFF7C8FF34BF012069
:100AC00000205DF808FB00BF4FEA4002B2F1FE4F84
:100AD0000FD34FF09E03B3EB12620DD94FEA002300
:100AE00043F0004310F0004F23FA02F018BF4042D9
:100AF00070474FF00000704712F1610F01D14202C0
:100B000005D110F0004008BF6FF0004070474FF073
:100B10000000704742000ED2B2F1FE4F0BD34FF0EF
:100B20009E03B3EB126209D44FEA002343F0004363
:100B300023FA02F070474FF00000704712F1610F86
:100B400001D1420202D14FF0FF3070474FF0000058
:100B5000704700BF0B460146184600F001B800BFC1
:100B600013460A460146022000F0BCBE014B18683D
:100B7000704700BFC897FF1F70B50F4E0F4D761B13
:100B8000B61018BF002405D0013455F8043B98472F
:100B9000A642F9D10A4E0B4D761B03F0AFFCB610FE
:100BA00018BF002406D0013455F8043B9847A642EC
:100BB000F9D170BD70BD00BF0845010008450100B6
:100BC0001C45010008450100024B0146186800F071
:100BD0000BB800BFC897FF1F024B0146186800F012
:100BE00045BF00BFC897FF1F2DE9F04F01F10B056E
:100BF000162D83B0064640F29F8035F0070500F1C0
:100C0000BF80A94200F2BC8000F058FBB5F5FC7F24
:100C1000C0F09C826B0A00F0BA80042B00F2838142
:100C2000A80900F1390E4FEA4E033830C44F07EBE4
:100C30008303A3F108015C68A14207D1ACE0002A5C
:100C400080F2AC80E468A14200F0A680636823F0E3
:100C500003035A1B0F2AF2DDB9493C6901F1080E62
:100C6000744500F0B381636823F003035A1B0F2A15
:100C700000F39981002AC1F814E0C1F810E080F275
:100C80009E80B3F5007F80F06781DB0803F1010CE3
:100C900001229B1002FA03F34A6851F83C80C4F821
:100CA000088001EBCC091A43A9F10803E3604A600C
:100CB00041F83C40C8F80C40831001249C40944209
:100CC00000F28A80144206D120F00300640014422E
:100CD00000F10400FAD007EBC009CC468046DCF8EE
:100CE0000C108C4507D173E1002A80F28181C9681C
:100CF0008C4500F06D814B6823F003035A1B0F2ACB
:100D0000F2DD0C46D1F80CC054F8088F4B1945F0B1
:100D100001054D6042F00101C8F80CC03046CCF826
:100D200008807B613B61C3F80CE0C3F808E05960C0
:100D30009A5000F0C5FA1FE0102921D800F0BEFA41
:100D40001025062302207E4F07EB8303A3F1080240
:100D50005C68944200F045816368E168A56823F00F
:100D60000303234430465A68E96042F001028D6073
:100D70005A6000F0A5FA0834204603B0BDE8F08FB1
:100D800000240C232046336003B0BDE8F08F80239D
:100D90004FF0400E3F2049E770465DE72344E1688D
:100DA0005A68A56842F00102E96030468D605A60D9
:100DB00000F086FA0834204603B0BDE8F08F2344E3
:100DC00030465A6842F001025A6000F079FA08345D
:100DD000204603B0BDE8F08FBC68636823F00308C9
:100DE000A84504D3C5EB08030F2B00F38C80554BAB
:100DF000DFF860911A68D9F8003001332A4404EB17
:100E0000080A00F0608102F580520F3222F47F62FE
:100E100022F00F0211463046019200F04BFCB0F177
:100E2000FF3F8346019A00F05881824500F2FC8022
:100E3000454B1968DA451144196000F05381D9F81F
:100E40000000DFF810E101301BBFCAEB0B0A514470
:100E5000CEF800B019601BF0070100F01781C1F156
:100E60000800C1F58051834408315A44C2F30B0293
:100E7000C2EB010949463046019300F01BFC431CBC
:100E8000019B00F03F81CBEB00024A4442F001029B
:100E90001968C7F808B04944BC42CBF8042019606F
:100EA000DFF8A49016D0B8F10F0F40F2FD80626811
:100EB000A8F10C0323F00703E01802F001024FF041
:100EC000050E1A430F2B6260C0F804E0C0F808E07A
:100ED00000F21C811D4BBC681A68914288BF1960E2
:100EE0001B4B1A689142626888BF196022F00302A6
:100EF0009542A2EB050301D80F2B04DC304600F02D
:100F0000DFF9002438E7621943F0010345F00105D9
:100F100065603046BA60536000F0D2F9083420466C
:100F200003B0BDE8F08F142B71D9542B00F2A480CC
:100F3000280B00F16F0E4FEA4E036E3076E600BFCD
:100F4000CC97FF1F90A2FF1F94A2FF1F8CA2FF1F30
:100F500088A2FF1FD89BFF1F5A0A042A5ED9142AB1
:100F600000F2B38002F15C0149005B3207EB810CB7
:100F700057F82110DFF8DC81ACF1080C8C4500F04B
:100F800088804A6822F00302934202D289688C4525
:100F9000F7D1D1F80CC07A68C4F80CC0A160CCF8C5
:100FA0000840CC6088E6631942F0010745F001056E
:100FB000656030464B610B61C3F80CE0C3F808E094
:100FC0005F609A50083400F07BF9D5E64A6873E612
:100FD00008F1010818F0030F0CF1080C7FF47FAE44
:100FE00030E0DC68A34208BF02303FF435AEB3E620
:100FF0000B440C465A68C96854F8085F42F0010275
:101000005A603046E9608D6000F05AF9B4E603F1A9
:101010005C0E03F15B004FEA4E0307E69A0902F10A
:10102000390149003832A1E7BC424A4B3FF400AFD6
:101030009C68626822F003025AE759F8083999451A
:1010400040F0828010F0030F00F1FF30F5D17B6893
:1010500023EA04037B6064009C423FF6BDAE002C93
:101060003FF4BAAE1C4240467FF435AE64001C42E9
:1010700000F10400FAD02EE6B3F5AA7F18D8E80BE9
:1010800000F1780E4FEA4E037730CFE54FF48051F0
:10109000EBE60121D8F80430921001FA02F21A436B
:1010A000C8F80420614677E70123CBF8043025E730
:1010B00040F25452934220D8A80C00F17D0E4FEA22
:1010C0004E037C30B2E51032A4E6542A26D81A0B1F
:1010D00002F16F0149006E3248E7BC68626822F095
:1010E000030205E7CAF30B0000287FF4A8AE4244D0
:1010F000BB6842F001025A60ECE6FE234FF07F0E1F
:101100007E2093E501224FF00009C1E604F10801B9
:10111000304600F0ABFCD9F80010DBE6B2F5AA7F50
:1011200005D8DA0B02F17801490077321EE740F268
:1011300054518A4205D89A0C02F17D0149007C3253
:1011400014E7FE217E2211E77B6884E7E808431C50
:101150005B00F8E5CC97FF1F8842F0B50DD98B18DE
:1011600098420AD28118002A51D09A1A13F8014DD8
:1011700001F8014D9342F9D1F0BD0F2A48D941EA57
:1011800000039B0746D100F1100401F1100315463E
:1011900053F8106C44F8106C53F80C6C44F80C6C59
:1011A00053F8086C44F8086C103D53F8046C44F88C
:1011B000046C0F2D03F1100304F11004E8D8A2F120
:1011C000100323F00F0302F00F0E1033BEF1030FD4
:1011D0001944034421D91E1F0D467446043C55F89A
:1011E000047B46F8047F032CF8D8AEF1040424F005
:1011F000030404342344214402F0030262B1013B9E
:101200000A4411F8014B03F8014F8A42F9D1F0BDAD
:101210000346F3E70346F2E7F0BD7246EEE700BF90
:1012200070B4840746D0541E002A41D0CDB2034684
:1012300002E0621EE4B3144603F8015B9A07F8D19A
:10124000032C2ED9CDB245EA05250F2C45EA0545DC
:1012500019D903F110022646103E0F2E42F8105CF9
:1012600042F80C5C42F8085C42F8045C02F110029F
:10127000F2D8A4F1100222F00F0204F00F04103291
:10128000032C13440DD91E462246043A032A46F87D
:10129000045BFAD8221F22F003020432134404F044
:1012A00003042CB1C9B21C4403F8011BA342FBD1B7
:1012B00070BC704714460346C2E700BF704700BFCA
:1012C000704700BF024B0A460146186800F002B89A
:1012D000C897FF1F2DE9F04F174683B0002900F093
:1012E000C1800E46814607F10B05FFF7E7FF56F870
:1012F00004EC162D2EF00304A6F1080840D81022A5
:101300001546AF4241D8944275DAC94B996808EB4B
:1013100004008842416800F0D98021F001030344B1
:101320005B68DB077DD51EF0010F35D03946484696
:10133000FFF75AFC0746E0B156F8043C23F00103DE
:101340004344A0F108029A4200F04481221F242A5B
:1013500000F23181132A00F20481034632461168FB
:1013600019605168596092689A603146484600F0A9
:101370007DFB4846FFF7A4FF384603B0BDE8F08F79
:1013800025F00705002D2A46BBDA0C230020C9F8FA
:10139000003003B0BDE8F08F56F8083CC3EB080AF4
:1013A000DAF8043023F0030C04EB0C039342BDDBAA
:1013B0005746DAF80C1057F8080F221F242AC1608C
:1013C000886000F21781132A40F212813168CAF84E
:1013D00008107168CAF80C101B2A00F22B8108361D
:1013E0000AF110023168116071685160B168916052
:1013F0003E461C46D046631B0F2B1DD8D8F8043040
:1014000003F0010323434444C8F80430636843F005
:10141000010363604846FFF753FF304603B0BDE861
:10142000F08F21F003012144914221DBC3688268DF
:101430000C46D3609A60DEE7D8F8042008EB05017B
:1014400002F00102154343F001020B44C8F80450B6
:101450004A605A6842F0010208315A60484600F07A
:1014600005FBD7E7114603B0BDE8F04FFFF7BCBB63
:101470001EF0010F7FF45AAF56F8083CC3EB080A80
:10148000DAF8043023F0030C01EB0C0E96458BDBED
:10149000C36882685746D3609A6057F8081FDAF825
:1014A0000C30CB60221F242A996000F29980132A05
:1014B00062D93368CAF808307368CAF80C301B2A3E
:1014C00000F2A08008360AF1100356E021F0030B69
:1014D000A34405F11000834559DA1EF0010F7FF493
:1014E00025AF56F8081CC1EB080ADAF8041021F001
:1014F000030CE34458453FF757AF5746DAF80C1052
:1015000057F8080F221F242AC160886000F2B480B7
:10151000132A40F2A5803168CAF808107168CAF829
:101520000C101B2A00F2AF8008360AF11002316855
:10153000116071685160B16891600AEB0501C5EBFB
:101540000B0242F0010299604A60DAF8043003F0BD
:1015500001031D434846CAF80450FFF7B1FE384660
:101560005CE733680360736843601B2A27D800F187
:10157000080306F10802F2E63B4632681A60726818
:101580005A60B2689A603E467446D04633E708EB2C
:101590000501C5EB0B0B4BF0010299604A6056F850
:1015A000043C03F001031D43484646F8045CFFF782
:1015B00087FE304632E73146FFF7CEFDD5E6B36809
:1015C0008360F368C360242A28D000F1100306F179
:1015D0001002C4E650F8043C23F003031C440AE75D
:1015E000314638467446D046FFF7B6FD3E4602E720
:1015F0003A46F7E6314638461C46D046FFF7ACFD82
:101600003E46F8E6B368CAF81030F368CAF81430FA
:10161000242A1BD010360AF11803AEE733690361A0
:101620007369436106F1180200F1180397E600BFE1
:10163000CC97FF1FB168CAF81010F168CAF81410EF
:10164000242A0FD010360AF11802CBE63369CAF803
:1016500018307369CAF81C3018360AF120038CE779
:101660003A4664E73269CAF818207269CAF81C2041
:1016700018360AF12002B5E6314638460193FFF7E5
:101680006BFD019B59E7B168CAF81010F168CAF800
:101690001410242A03D010360AF1180247E73269E1
:1016A000CAF818207269CAF81C2018360AF12002FC
:1016B0003DE700BF38B5074C0023054608462360C8
:1016C000FBF7E2FE431C00D038BD2368002BFBD0A3
:1016D0002B6038BDF0A3FF1FFFFFFFFFFFFFFFFFE1
:1016E000FFFFFFFFFFFFFFFFFFFFFFFFFFFFFFFF0A
:1016F000FFFFFFFFFFFFFFFFFFFFFFFFFFFFFFFFFA
:1017000090F800F06DE9024520F007016FF0000C41
:1017100010F0070491F820F040F049804FF00004E9
:101720006FF00700D1E9002391F840F000F10800C4
:1017300082FA4CF2A4FA8CF283FA4CF3A2FA8CF3FC
:101740004BBBD1E9022382FA4CF200F10800A4FA63
:101750008CF283FA4CF3A2FA8CF3E3B9D1E90423B7
:1017600082FA4CF200F10800A4FA8CF283FA4CF3EE
:10177000A2FA8CF37BB9D1E9062301F1200182FAA8
:101780004CF200F10800A4FA8CF283FA4CF3A2FAAE
:101790008CF3002BC6D0002A04BF04301A4612BABC
:1017A000B2FA82F2FDE8024500EBD2007047D1E9BF
:1017B000002304F00305C4F100004FEAC50514F04E
:1017C000040F91F840F00CFA05F562EA05021CBF1F
:1017D00063EA050362464FF00004A9E7002A41D0FE
:1017E00040EA010313F00303F0B425D1032A23D9FF
:1017F00004680D68AC421FD1043A35D0A4F101351C
:1018000025EA040414F0803F31D1071D0D1D0DE0C1
:1018100057F8043B0E68A3F10134B34224EA0304F1
:101820000AD1043A20D014F0803F23D1032A29465C
:10183000384605F10405EBD803780C789C4202F198
:10184000FF320CD182B114B916E06AB17BB110F845
:10185000013F11F8014FA34202F1FF32F5D0181BEE
:10186000F0BC7047104670471046F0BC70471846F1
:10187000F0BC70470020F3E72046F1E740EA01039F
:101880009B0770B42BD1032A29D90C460346214665
:1018900054F8046BA6F1013525EA060515F0803FE2
:1018A00006D1043A032A43F8046B2146EFD8A2B1CB
:1018B0000C781C70013A013301313CB16AB111F866
:1018C000014B03F8014B013A002CF7D12AB11A441D
:1018D000002103F8011B9A42FBD170BC70470346FC
:1018E000E5E700BF2DE9F047254C2568D5F84841CC
:1018F0000646884692469946C4B360681F2817DC9E
:10190000431C76B104EB80050122C5F888A0D4F809
:10191000881182401143022EC4F88811C5F808913D
:101920001ED00230636044F820800020BDE8F087BC
:10193000144B03B34FF4C870FFF746F90446D0B117
:10194000D5F84831002780E88800C5F84841384676
:101950000123C4F88871C4F88C71002EE1D0D1E75E
:10196000D4F88C110A43C4F88C21DAE705F5A67483
:10197000C5F84841C1E74FF0FF30BDE8F08700BF30
:10198000F8440100C90B0100024B13B1024800F0FA
:1019900005B8704700000000A919010000230146A6
:1019A0001A461846FFF79EBF38B5074D074C2C1B4B
:1019B000A41005D0013C55F8043D9847002CF9D1FE
:1019C000BDE8384002F0AABD0000000000000000A1
:1019D000F8B5234F0C460646FFF770FCBB685D6800
:1019E00025F00305291B01F6EF7121F47F6121F039
:1019F0000F01A1F58054B4F5805F07DB002130466C
:101A0000FFF758FEBB682B44984204D03046FFF7DE
:101A100057FC0020F8BD61423046FFF74BFE013015
:101A20000DD0104BBA6819682D1B45F001053046E2
:101A3000091B55601960FFF743FC0120F8BD002128
:101A40003046FFF737FEBA68831A0F2BDEDD064CEF
:101A50000449246843F00103001B53600860D5E784
:101A6000CC97FF1F94A2FF1FD89BFF1F002945D0D2
:101A70002DE9F0410D468046FFF720FC55F8047C27
:101A80006A4927F00103A5F10804E2188E6850683E
:101A9000B24220F0030062D0FE0750600BD455F82C
:101AA000087CE41B01F1080EA56875453B446FD026
:101AB000E768EF60BD6015186D68ED0742D543F02B
:101AC00001026260E350B3F5007F18D2DB085A1CB4
:101AD0004D6851F83270A76001209B1000FA03F3A3
:101AE00001EBC2001D430838E0604D6041F8324010
:101AF000FC604046BDE8F041FFF7E2BB70475A0A80
:101B0000042A53D89A0902F139077F0002F13805F7
:101B100001EB870051F827204449083890424DD006
:101B2000516821F003018B4202D292689042F7D1B2
:101B3000D068E060A2608460D4604046BDE8F041B7
:101B4000FFF7BEBB95683A4FBD4203443FD0D06813
:101B5000E86043F0010285606260E350B3E7FF078D
:101B6000034407D455F8082CA41A1344A068E2686B
:101B7000C26090602F4A126843F001009342606097
:101B80008C60B6D32C4B40461968FFF721FFB0E7B5
:101B900011184968C90744D49168D268CA600344DF
:101BA00043F0010091606060E350A2E7142A17D867
:101BB00002F15C077F0002F15B05A9E7AA104B6800
:101BC000012505FA02F213434B600246B1E743F0E8
:101BD00001024C610C61E560A5606260E35088E73A
:101BE000542A06D81A0B02F16F077F0002F16E0526
:101BF0008EE7B2F5AA7F06D8DA0B02F178077F00EC
:101C000002F1770584E740F25450824206D89A0CDC
